:10000000F8FF0220A99501008D950100459501009A
:100010004595010045950100459501004595010074
:100020004595010045950100459501008D9501001C
:100030008D950100459501000DC5010085C70100A2
:100040008D9501008D9501008D9501008D95010024
:100050008D9501008D9501008D9501008D95010014
:100060008D9501008D9501008D9501008D95010004
:100070008D9501008D9501008D9501008D950100F4
:100080008D9501008D9501008D9501008D950100E4
:100090008D9501008D9501008D9501008D950100D4
:1000A000A1850100FD8601008D9501008D9501005F
:1000B0008D9501008D9501008D95010059DB0100A2
:1000C0008D950100B5DC01008D95010011DE010068
:1000D0008D95010041DF01008D9501008D95010096
:1000E0008D9501008D9501008D9501008D95010084
:1000F0008D9501008D9501008D9501008D95010074
:100100008D9501008D9501008D9501008D95010063
:100110008D95010049A001008D9501008D9501008C
:100120008D9501008D9501008D9501008D95010043
:100130008D9501008D9501008D9501008D95010033
:1001400059C201008D95010071E001008D950100FB
:10015000A1E101008D9501008D9501008D950100B3
:100160008D9501008D950100598801008D95010044
:100170008D9501008D9501008D9501008D950100F3
:100180008D9501008D9501008D9501008D950100E3
:100190008D9501008D950100FFFFFFFFFFFFFFFF21
:1001A000FFFFFFFFFFFFFFFFFFFFFFFFFFFFFFFF5F
:1001B000FFFFFFFFFFFFFFFFFFFFFFFFFFFFFFFF4F
:1001C000FFFFFFFFFFFFFFFFFFFFFFFFFFFFFFFF3F
:1001D000FFFFFFFFFFFFFFFFFFFFFFFFFFFFFFFF2F
:10040000FFFFFFFFFFFFFFFFFFFFFFFFDEF9FFFF23
:1004100010B5054C237833B9044B13B10448AFF33E
:1004200000800123237010BDF4EB002000000000C9
:10043000844C0200084B10B51BB108490848AFF3C3
:1004400000800848036803B910BD074B002BFBD0A0
:10045000BDE81040184700BF00000000F8EB002086
:10046000844C0200F4EB002000000000704700BF45
:1004700010B54FF4097104461CF0EAFB204610BD8C
:1004800070B54FF06A522DED028B064642F6585376
:1004900008EE902A40F6DB72C0F202034FF20E45DE
:1004A00040F6DA70C4F24902C2F20005C3F64920F0
:1004B00008EE102A336000240FE007EE904AF8EEB1
:1004C000E77A77EE807A67EEA87A67EE887A27EE89
:1004D000800A1EF08DF910EE100A21F04BF941EC64
:1004E000100B1DF0EDFF00230022CCF2900351EC25
:1004F000100B21F093F941EC100B1DF0F5FF51ECBE
:10050000100B21F063FC0134B4F5806FB6EE000AE5
:1005100025F8020FD1D14FF06A534EF60E4508EE82
:10052000103AC2F20005002407EE904AF8EEE77A8E
:10053000013467EE887A17EE900A21F01BF99FEDDF
:10054000140B41EC110B1EF053FA002351EC100B6D
:100550000022C3F6F07320F0ADFF00230022C4F2A6
:10056000B00321F05BF921F051FC21F003F941ECDB
:10057000100B1DF0B9FF51EC100B21F027FCB4F566
:10058000806F25F8020FCFD1BDEC028B304670BDD5
:100590000000000000000040704700BF10B54FF49D
:1005A000097104461CF054FB204610BD2DE9F04FA4
:1005B0004DF68466C2F200060A9D0B989DF83070D5
:1005C000B6F800C042F67054C0F20204C5EB000A4F
:1005D000002F18BF0C466FEA0C0B0AF1200A4DF6EB
:1005E00084294DF68448043A271FA1F1040E0FFA1E
:1005F0008BFB4FEAAA1AC2F20009C2F200080026D9
:1006000027E0B4F5007F02D08CB3C943C9B239F8F2
:1006100011104CEA010101EBC00080B20BEA0004AA
:10062000E143C9B2241238F8111001F58061490084
:10063000E14010EA0C0F18BFC94357F8044F09985E
:1006400009B2013604EB8131402E03444EF8041FF9
:1006500010D052F8041F1944891301F44074554412
:10066000B4F5807FC9B2A8B2CBD1C943C9B239F8B9
:100670001110D0E7BDE8F08F2DE9F04F4DF68465FD
:10068000C2F2000509982E880A9D9DF82C7042F64A
:100690007054C0F20204C0EB050E002F14BF0F46C9
:1006A00027466FEA06090EF1200E4DF684284DF616
:1006B000844C3C1F0D1F0FFA89F9FC374FEAAE1E20
:1006C000C2F20008C2F2000C2AE0BBF5007F04D0A1
:1006D000BBF1000F30D0C943C9B238F81110314313
:1006E00001EBCA0A1FFA8AFA09EA0A0B6FEA0B0140
:1006F000C9B24FEA2B2B3CF8111001F5806149007B
:100700001AEA060F21FA0BF154F804AF18BFC943D7
:1007100009B20AEB8131BC421A4445F8041F0ED0DD
:10072000911301F4407B7044BBF5807F1FFA80FA7F
:10073000C9B2CAD1C943C9B238F81110D0E7BDE86F
:10074000F08F00BF2DE9F04F4DF6846083B0C2F208
:1007500000000D9EB0F800C00C9C9DF840A00F9FBB
:100760000E980E9D019342F6705EC0F2020EC4EB2D
:10077000060B6FEA0C06BAF1000F14BF8A46F24668
:1007800033B20BF1200B4DF684294DF68448AAF1C3
:10079000040600686D680093A1F1040E0AF1FC0ADA
:1007A0004FEAAB1B0137C2F20009C2F2000829E090
:1007B000B0F5007F02D098B3DB43DBB239F81330D9
:1007C0004CEA030303EBC101009B89B203EA010079
:1007D000C343DBB2001238F8133003F580635B00CB
:1007E000C34011EA0C0F18BFDB4356F8041F0198F1
:1007F0001BB29B031944564502444EF8041F284679
:1008000011D01D4643193B4113449B1303F4407020
:100810005C44B0F5807FDBB2A1B2C9D1DB43DBB26F
:1008200039F81330CEE70E9A1560536003B0BDE877
:10083000F08F00BF2DE9F04F43F6EC6403EB430368
:10084000C0F2020404EBC3050646144689460FCDE8
:1008500091B00AAF0FC795E80300002387E80300B3
:10086000012704F160088DF8247007978DF8253072
:100870008DF826300AAD48E00AF1FF3101EB011195
:1008800006EB0111133121F00F0194E80140C0146F
:10089000C0F500706060BEF1000F3FD0BEF5FE7F76
:1008A0003EDA10AFBA441AF81CCCBCF1000F04D0E9
:1008B00012F1000C18BF4FF0010CC3F301123AB152
:1008C00010AF07EB020B1BF81CBCBBF1000F34D1BF
:1008D00003F0C003C02B02D11B9B0F2B41DDA3688B
:1008E000E2680190CDF808C0CDF800E03046FFF78F
:1008F000C3FE9DF81C300AF81C3CE368A26803EBB9
:100900008213E3601034A04514D055F8043B13F073
:10091000030A03F00402AFD14946B6E740F2FF1ED6
:10092000B0F5FE7FBDDB002AE7D110AB9A440AF890
:100930001C2CE2E711B0BDE8F08F013A02EB021285
:10094000E368CDF80CC006EB02120290CDF804E08B
:10095000A0680090133222F00F023046FFF726FE07
:10096000C7E71F46E268A36803971A9F0190CDF876
:1009700010C00297CDF800E03046FFF7E3FEB8E77D
:1009800000207047704700BF704700BF10B5044695
:100990001BF0E4FB204610BD10B5044621F010FF0B
:1009A00001462046BDE810401BF0D0B842F6EC608E
:1009B00008B51021C0F202001BF0C8F84FF60F2056
:1009C0001AF03AFA42F60070C0F202000F211BF052
:1009D000BDF84EF20020C2F20000BDE808401BF056
:1009E000C7BF00BF42F6107008B51621C0F2020062
:1009F0001BF0ACF84FF20F601AF01EFA42F60070CE
:100A0000C0F202000F211BF0A1F84EF20020C2F24A
:100A10000000BDE808401BF0ABBF00BF42F62870E5
:100A200008B51321C0F202001BF090F84FF60F300A
:100A30001AF002FA42F60070C0F202000F211BF019
:100A400085F84EF20020C2F20000BDE808401BF01D
:100A50008FBF00BF42F63C7008B50F21C0F2020004
:100A60001BF074F84FF60F401AF0E6F942F60070EA
:100A7000C0F202000F211BF069F84EF20020C2F212
:100A80000000BDE808401BF073BF00BF42F64C7089
:100A900008B51821C0F202001BF058F84FF60F609D
:100AA0001AF0CAF942F60070C0F202000F211BF0E2
:100AB0004DF84EF20020C2F20000BDE808401BF0E5
:100AC00057BF00BF38B542F668704EF2002540F6B9
:100AD00064541021C2F20104C2F20005C0F2020007
:100AE0001BF034F828461BF043FF20680FF0EEF8A7
:100AF00020680EF0F7FF20680FF008F842F67C70CF
:100B00001621C0F202001BF021F84FF60F701AF008
:100B100093F942F60070C0F202000F211BF016F8A4
:100B20002846BDE838401BF023BF00BF42F6947052
:100B300008B51021C0F202001BF008F840F67473EB
:100B4000C2F20103FA21986C03681B68984742F6C9
:100B5000A870C0F202000F211AF0F8FF4EF2002038
:100B6000C2F20000BDE808401BF002BF42F6B870B8
:100B700008B51321C0F202001AF0E8FF40F67473C2
:100B8000C2F20103FB21986C03681B68984742F688
:100B9000A870C0F202000F211AF0D8FF4EF2002018
:100BA000C2F20000BDE808401BF0E2BE42F6CC7085
:100BB00008B50F21C0F202001AF0C8FF40F67473A6
:100BC000C2F20103FC21986C03681B68984742F647
:100BD000A870C0F202000F211AF0B8FF4EF20020F8
:100BE000C2F20000BDE808401BF0C2BE42F6DC7055
:100BF00008B51821C0F202001AF0A8FF40F674737D
:100C0000C2F20103FE21986C03681B68984742F604
:100C1000A870C0F202000F211AF098FF4EF20020D7
:100C2000C2F20000BDE808401BF0A2BE38B542F693
:100C300068704EF2002540F664541021C2F201049F
:100C4000C2F20005C0F202001AF080FF28461BF035
:100C50008FFE20680FF03AF820680EF043FF2068FE
:100C60000EF054FF42F6F8701621C0F202001AF09E
:100C70006DFF40F67473C2F20103FF21986C0368A4
:100C80001B68984742F6A870C0F202000F211AF0C4
:100C90005DFF2846BDE838401BF06ABE10B504462B
:100CA00043F210001521C0F202001AF04FFF200499
:100CB00000F4FE0040F4734040F002001AF0BCF86B
:100CC00042F60070C0F202000F211AF03FFF4EF210
:100CD0000020C2F20000BDE810401BF049BE00BF7A
:100CE00010B5044643F228001F21C0F2020004F0B0
:100CF0000F041AF02BFF44F010044FF2021040EAE8
:100D000004401AF099F842F60070C0F202000F2178
:100D10001AF01CFF4EF20020C2F20000BDE81040A5
:100D20001BF026BE43F2480008B51621C0F20200AF
:100D30001AF00CFF40F67473C2F20103F621986CAE
:100D40000368DB6C984742F6A870C0F202000F21DE
:100D50001AF0FCFE4EF20020C2F20000BDE808408E
:100D60001BF006BE1F2938B50C46054608D84DF6BF
:100D70008863C2F2000318790FF01AFF0BF0B2FD7E
:100D800043F260000D21C0F202001AF0DFFE2304DE
:100D9000681E03F4FE0343F44043000243F00C03D7
:100DA00000F4706018431AF047F842F60070C0F281
:100DB00002000F211AF0CAFE4EF20020C2F200001B
:100DC000BDE838401BF0D4BD70B5064643F2700054
:100DD0000C46C0F20200122115461AF0B7FE6EB999
:100DE000681E0002240400F4706004F4FE04204332
:100DF00040F4504040F00D001AF01EF842F600702A
:100E0000C0F202000F211AF0A1FE4EF20020C2F241
:100E10000000BDE870401BF0ABBD00BF38B540F628
:100E200074740546C2F2010443F284001F21C0F22B
:100E300002001AF08BFEA06C0368F1211B68984732
:100E4000A06C036829461B68984742F6A870C0F258
:100E500002000F211AF07AFE4EF20020C2F20000CA
:100E6000BDE838401BF084BD38B540F674740546C3
:100E7000C2F2010443F2A4001521C0F202001AF0EC
:100E800065FEA06C0368F3211B689847A06C03689B
:100E900005F07F01DB6C984742F6A870C0F20200B3
:100EA0000F211AF053FE4EF20020C2F20000BDE8FE
:100EB00038401BF05DBD00BF38B540F66453C2F248
:100EC000010301F500521B6805460C4643F2BC00C5
:100ED000C3F884200D21C0F2020004F30D041AF0BF
:100EE00035FE04F50054681E2304000203F4FE03DB
:100EF00000F47060184340F46040640404F0FE4461
:100F000040F00E00204319F097FF42F60070C0F247
:100F100002000F211AF01AFE4EF20020C2F2000069
:100F2000BDE838401BF024BDF0B548F29042C2F253
:100F3000010283B040F2442311680091C2F2010320
:100F400000991E681268019240F65C55C2F20105D4
:100F500040F62852C2F20102891B43F2CC004EF245
:100F60000024C2F20004019F298000260C21C0F257
:100F7000020016701F601AF0E9FD2B8820464EF61D
:100F8000602191FBF3F11BF095FC43F2DC0005219D
:100F9000C0F202001AF0DAFD298820461BF08AFC14
:100FA00043F2E4000F21C0F202001AF0CFFD204608
:100FB0001BF0DEFC03B0F0BD08B540F62851C2F2CC
:100FC00001014AF6AB230A780132D2B2CAF6AA234B
:100FD000A3FB02031B0903EB4303A2EBC30313F0C0
:100FE000FF0F0A7001D1FFF79FFF43F2F4001021B9
:100FF000C0F202001AF0AAFD4FF60F0019F01CFF14
:1010000042F60070C0F202000F211AF09FFD4EF26E
:101010000020C2F20000BDE808401BF0A9BC00BFE0
:1010200008B540F62851C2F201014AF6AB230A780E
:101030000132D2B2CAF6AA23A3FB02031B0903EBB7
:101040004303A2EBC30313F0FF0F0A7001D1FFF7B4
:101050006BFF43F208101021C0F202001AF076FD77
:1010600040F67473C2F20103F821986C03681B68A0
:10107000984742F6A870C0F202000F211AF066FDF0
:101080004EF20020C2F20000BDE808401BF070BC28
:101090001F2938B50D46044608D84DF68863C2F2BC
:1010A000000318790FF084FD0BF01CFC43F21C10B8
:1010B0000D21C0F202001AF049FD611EC9B20F29CC
:1010C0000FD840F67474C2F2010441F0C001A06C64
:1010D00003681B689847A06C036805F07F011B68D4
:1010E000984742F6A870C0F202000F211AF02EFDB8
:1010F0004EF20020C2F20000BDE838401BF038BCC0
:1011000048F28C33C2F2010310B41A6813685068B5
:1011100019780478507A137A044201EA03011AD04C
:10112000937A03F0030309B143F0040343F0080387
:101130009910082B91722AD8072B22D2032B2ED07C
:1011400011D9042B13D0062B14D1D3685DF8044BAE
:10115000023BD3607047937A03F003030029E7D082
:1011600043F00403E4E7012B0BD0022B02D1D36838
:10117000013BD3605DF8044B70470D2BF7D00E2B6D
:10118000F8D1D3685DF8044B0133D36070470C2B62
:1011900005D0F2D8092BD8D00B2BE8D0EAE7D368DA
:1011A0005DF8044B0233D360704700BF48F28C33C4
:1011B000C2F2010310B45A681368506819780478B1
:1011C000507A137A044201EA03011AD0937A03F0A9
:1011D000030309B143F0040343F008039910082BFB
:1011E00091722AD8072B22D2032B2ED011D9042B8F
:1011F00013D0062B14D1D3685DF8044B023BD360A7
:101200007047937A03F003030029E7D043F0040307
:10121000E4E7012B0BD0022B02D1D368013BD36052
:101220005DF8044B70470D2BF7D00E2BF8D1D36827
:101230005DF8044B0133D36070470C2B05D0F2D816
:10124000092BD8D00B2BE8D0EAE7D3685DF8044B24
:101250000233D360704700BF48F28C33C2F20103FF
:1012600010B49A681368506819780478507A137A21
:10127000044201EA03011AD0937A03F0030309B18F
:1012800043F0040343F008039910082B91722AD805
:10129000072B22D2032B2ED011D9042B13D0062BCF
:1012A00014D1D3685DF8044B023BD3607047937A46
:1012B00003F003030029E7D043F00403E4E7012B24
:1012C0000BD0022B02D1D368013BD3605DF8044BF5
:1012D00070470D2BF7D00E2BF8D1D3685DF8044B77
:1012E0000133D36070470C2B05D0F2D8092BD8D02E
:1012F0000B2BE8D0EAE7D3685DF8044B0233D360E8
:10130000704700BF48F28C33C2F2010310B4DA68B0
:101310001368506819780478507A137A044201EA05
:1013200003011AD0937A03F0030309B143F00403D5
:1013300043F008039910082B91722AD8072B22D268
:10134000032B2ED011D9042B13D0062B14D1D36824
:101350005DF8044B023BD3607047937A03F00303BC
:101360000029E7D043F00403E4E7012B0BD0022B64
:1013700002D1D368013BD3605DF8044B70470D2B5D
:10138000F7D00E2BF8D1D3685DF8044B0133D3604E
:1013900070470C2B05D0F2D8092BD8D00B2BE8D0F6
:1013A000EAE7D3685DF8044B0233D360704700BFAF
:1013B00048F28C33C2F2010310B41A691368506802
:1013C00019780478507A137A044201EA03011AD09A
:1013D000937A03F0030309B143F0040343F00803D5
:1013E0009910082B91722AD8072B22D2032B2ED0CA
:1013F00011D9042B13D0062B14D1D3685DF8044BFC
:10140000023BD3607047937A03F003030029E7D0CF
:1014100043F00403E4E7012B0BD0022B02D1D36885
:10142000013BD3605DF8044B70470D2BF7D00E2BBA
:10143000F8D1D3685DF8044B0133D36070470C2BAF
:1014400005D0F2D8092BD8D00B2BE8D0EAE7D36827
:101450005DF8044B0233D360704700BF48F28C3311
:10146000C2F2010310B45A691368506819780478FD
:10147000507A137A044201EA03011AD0937A03F0F6
:10148000030309B143F0040343F008039910082B48
:1014900091722AD8072B22D2032B2ED011D9042BDC
:1014A00013D0062B14D1D3685DF8044B023BD360F4
:1014B0007047937A03F003030029E7D043F0040355
:1014C000E4E7012B0BD0022B02D1D368013BD360A0
:1014D0005DF8044B70470D2BF7D00E2BF8D1D36875
:1014E0005DF8044B0133D36070470C2B05D0F2D864
:1014F000092BD8D00B2BE8D0EAE7D3685DF8044B72
:101500000233D360704700BF48F28C33C2F201034C
:1015100010B49A691368506819780478507A137A6D
:10152000044201EA03011AD0937A03F0030309B1DC
:1015300043F0040343F008039910082B91722AD852
:10154000072B22D2032B2ED011D9042B13D0062B1C
:1015500014D1D3685DF8044B023BD3607047937A93
:1015600003F003030029E7D043F00403E4E7012B71
:101570000BD0022B02D1D368013BD3605DF8044B42
:1015800070470D2BF7D00E2BF8D1D3685DF8044BC4
:101590000133D36070470C2B05D0F2D8092BD8D07B
:1015A0000B2BE8D0EAE7D3685DF8044B0233D36035
:1015B000704700BF48F28C33C2F2010310B4DA69FD
:1015C0001368506819780478507A137A044201EA53
:1015D00003011AD0937A03F0030309B143F0040323
:1015E00043F008039910082B91722AD8072B22D2B6
:1015F000032B2ED011D9042B13D0062B14D1D36872
:101600005DF8044B023BD3607047937A03F0030309
:101610000029E7D043F00403E4E7012B0BD0022BB1
:1016200002D1D368013BD3605DF8044B70470D2BAA
:10163000F7D00E2BF8D1D3685DF8044B0133D3609B
:1016400070470C2B05D0F2D8092BD8D00B2BE8D043
:10165000EAE7D3685DF8044B0233D360704700BFFC
:1016600048F28C33C2F2010310B41A6E136850684A
:1016700019780478507A137A044201EA03011AD0E7
:10168000937A03F0030309B143F0040343F0080322
:101690009910082B91722AD8072B22D2032B2ED017
:1016A00011D9042B13D0062B14D1D3685DF8044B49
:1016B000023BD3607047937A03F003030029E7D01D
:1016C00043F00403E4E7012B0BD0022B02D1D368D3
:1016D000013BD3605DF8044B70470D2BF7D00E2B08
:1016E000F8D1D3685DF8044B0133D36070470C2BFD
:1016F00005D0F2D8092BD8D00B2BE8D0EAE7D36875
:101700005DF8044B0233D360704700BF48F28C335E
:10171000C2F2010310B45A6E136850681978047845
:10172000507A137A044201EA03011AD0937A03F043
:10173000030309B143F0040343F008039910082B95
:1017400091722AD8072B22D2032B2ED011D9042B29
:1017500013D0062B14D1D3685DF8044B023BD36041
:101760007047937A03F003030029E7D043F00403A2
:10177000E4E7012B0BD0022B02D1D368013BD360ED
:101780005DF8044B70470D2BF7D00E2BF8D1D368C2
:101790005DF8044B0133D36070470C2B05D0F2D8B1
:1017A000092BD8D00B2BE8D0EAE7D3685DF8044BBF
:1017B0000233D360704700BF48F28C33C2F201039A
:1017C00010B49A6E1368506819780478507A137AB6
:1017D000044201EA03011AD0937A03F0030309B12A
:1017E00043F0040343F008039910082B91722AD8A0
:1017F000072B22D2032B2ED011D9042B13D0062B6A
:1018000014D1D3685DF8044B023BD3607047937AE0
:1018100003F003030029E7D043F00403E4E7012BBE
:101820000BD0022B02D1D368013BD3605DF8044B8F
:1018300070470D2BF7D00E2BF8D1D3685DF8044B11
:101840000133D36070470C2B05D0F2D8092BD8D0C8
:101850000B2BE8D0EAE7D3685DF8044B0233D36082
:10186000704700BF48F28C33C2F2010310B4DA6E45
:101870001368506819780478507A137A044201EAA0
:1018800003011AD0937A03F0030309B143F0040370
:1018900043F008039910082B91722AD8072B22D203
:1018A000032B2ED011D9042B13D0062B14D1D368BF
:1018B0005DF8044B023BD3607047937A03F0030357
:1018C0000029E7D043F00403E4E7012B0BD0022BFF
:1018D00002D1D368013BD3605DF8044B70470D2BF8
:1018E000F7D00E2BF8D1D3685DF8044B0133D360E9
:1018F00070470C2B05D0F2D8092BD8D00B2BE8D091
:10190000EAE7D3685DF8044B0233D360704700BF49
:1019100048F28C33C2F2010310B41A6F1368506896
:1019200019780478507A137A044201EA03011AD034
:10193000937A03F0030309B143F0040343F008036F
:101940009910082B91722AD8072B22D2032B2ED064
:1019500011D9042B13D0062B14D1D3685DF8044B96
:10196000023BD3607047937A03F003030029E7D06A
:1019700043F00403E4E7012B0BD0022B02D1D36820
:10198000013BD3605DF8044B70470D2BF7D00E2B55
:10199000F8D1D3685DF8044B0133D36070470C2B4A
:1019A00005D0F2D8092BD8D00B2BE8D0EAE7D368C2
:1019B0005DF8044B0233D360704700BF48F28C33AC
:1019C000C2F2010310B45A6F136850681978047892
:1019D000507A137A044201EA03011AD0937A03F091
:1019E000030309B143F0040343F008039910082BE3
:1019F00091722AD8072B22D2032B2ED011D9042B77
:101A000013D0062B14D1D3685DF8044B023BD3608E
:101A10007047937A03F003030029E7D043F00403EF
:101A2000E4E7012B0BD0022B02D1D368013BD3603A
:101A30005DF8044B70470D2BF7D00E2BF8D1D3680F
:101A40005DF8044B0133D36070470C2B05D0F2D8FE
:101A5000092BD8D00B2BE8D0EAE7D3685DF8044B0C
:101A60000233D360704700BF48F28C33C2F20103E7
:101A700010B49A6F1368506819780478507A137A02
:101A8000044201EA03011AD0937A03F0030309B177
:101A900043F0040343F008039910082B91722AD8ED
:101AA000072B22D2032B2ED011D9042B13D0062BB7
:101AB00014D1D3685DF8044B023BD3607047937A2E
:101AC00003F003030029E7D043F00403E4E7012B0C
:101AD0000BD0022B02D1D368013BD3605DF8044BDD
:101AE00070470D2BF7D00E2BF8D1D3685DF8044B5F
:101AF0000133D36070470C2B05D0F2D8092BD8D016
:101B00000B2BE8D0EAE7D3685DF8044B0233D360CF
:101B1000704700BF48F28C33C2F2010310B4DA6F91
:101B20001368506819780478507A137A044201EAED
:101B300003011AD0937A03F0030309B143F00403BD
:101B400043F008039910082B91722AD8072B22D250
:101B5000032B2ED011D9042B13D0062B14D1D3680C
:101B60005DF8044B023BD3607047937A03F00303A4
:101B70000029E7D043F00403E4E7012B0BD0022B4C
:101B800002D1D368013BD3605DF8044B70470D2B45
:101B9000F7D00E2BF8D1D3685DF8044B0133D36036
:101BA00070470C2B05D0F2D8092BD8D00B2BE8D0DE
:101BB000EAE7D3685DF8044B0233D360704700BF97
:101BC00048F28C33C2F2010310B4D3F880201368BA
:101BD000506819780478507A137A044201EA0301B4
:101BE0001AD0937A03F0030309B143F0040343F0DE
:101BF00008039910082B91722AD8072B22D2032BA5
:101C00002ED011D9042B13D0062B14D1D3685DF834
:101C1000044B023BD3607047937A03F0030300291F
:101C2000E7D043F00403E4E7012B0BD0022B02D1F1
:101C3000D368013BD3605DF8044B70470D2BF7D0A0
:101C40000E2BF8D1D3685DF8044B0133D360704795
:101C50000C2B05D0F2D8092BD8D00B2BE8D0EAE713
:101C6000D3685DF8044B0233D360704748F28C337D
:101C7000C2F2010310B4D3F88420136850681978B5
:101C80000478507A137A044201EA03011AD0937A55
:101C900003F0030309B143F0040343F00803991070
:101CA000082B91722AD8072B22D2032B2ED011D9C0
:101CB000042B13D0062B14D1D3685DF8044B023BE0
:101CC000D3607047937A03F003030029E7D043F011
:101CD0000403E4E7012B0BD0022B02D1D368013BB4
:101CE000D3605DF8044B70470D2BF7D00E2BF8D165
:101CF000D3685DF8044B0133D36070470C2B05D0DB
:101D0000F2D8092BD8D00B2BE8D0EAE7D3685DF8DE
:101D1000044B0233D360704748F28C33C2F20103A4
:101D200010B4D3F888201368506819780478507A72
:101D3000137A044201EA03011AD0937A03F00303F1
:101D400009B143F0040343F008039910082B917282
:101D50002AD8072B22D2032B2ED011D9042B13D033
:101D6000062B14D1D3685DF8044B023BD360704757
:101D7000937A03F003030029E7D043F00403E4E778
:101D8000012B0BD0022B02D1D368013BD3605DF84D
:101D9000044B70470D2BF7D00E2BF8D1D3685DF8AC
:101DA000044B0133D36070470C2B05D0F2D8092BBC
:101DB000D8D00B2BE8D0EAE7D3685DF8044B0233A8
:101DC000D360704748F28C33C2F2010310B4D3F8E9
:101DD0008C201368506819780478507A137A04427A
:101DE00001EA03011AD0937A03F0030309B143F027
:101DF000040343F008039910082B91722AD8072B8B
:101E000022D2032B2ED011D9042B13D0062B14D1A0
:101E1000D3685DF8044B023BD3607047937A03F0BC
:101E200003030029E7D043F00403E4E7012B0BD0C0
:101E3000022B02D1D368013BD3605DF8044B70479D
:101E40000D2BF7D00E2BF8D1D3685DF8044B01337E
:101E5000D36070470C2B05D0F2D8092BD8D00B2BB0
:101E6000E8D0EAE7D3685DF8044B0233D3607047EB
:101E700048F28C33C2F2010310B4D3F890201368F7
:101E8000506819780478507A137A044201EA030101
:101E90001AD0937A03F0030309B143F0040343F02B
:101EA00008039910082B91722AD8072B22D2032BF2
:101EB0002ED011D9042B13D0062B14D1D3685DF882
:101EC000044B023BD3607047937A03F0030300296D
:101ED000E7D043F00403E4E7012B0BD0022B02D13F
:101EE000D368013BD3605DF8044B70470D2BF7D0EE
:101EF0000E2BF8D1D3685DF8044B0133D3607047E3
:101F00000C2B05D0F2D8092BD8D00B2BE8D0EAE760
:101F1000D3685DF8044B0233D360704748F28C33CA
:101F2000C2F2010310B4D3F89420136850681978F2
:101F30000478507A137A044201EA03011AD0937AA2
:101F400003F0030309B143F0040343F008039910BD
:101F5000082B91722AD8072B22D2032B2ED011D90D
:101F6000042B13D0062B14D1D3685DF8044B023B2D
:101F7000D3607047937A03F003030029E7D043F05E
:101F80000403E4E7012B0BD0022B02D1D368013B01
:101F9000D3605DF8044B70470D2BF7D00E2BF8D1B2
:101FA000D3685DF8044B0133D36070470C2B05D028
:101FB000F2D8092BD8D00B2BE8D0EAE7D3685DF82C
:101FC000044B0233D360704748F28C33C2F20103F2
:101FD00010B4D3F898201368506819780478507AB0
:101FE000137A044201EA03011AD0937A03F003033F
:101FF00009B143F0040343F008039910082B9172D0
:102000002AD8072B22D2032B2ED011D9042B13D080
:10201000062B14D1D3685DF8044B023BD3607047A4
:10202000937A03F003030029E7D043F00403E4E7C5
:10203000012B0BD0022B02D1D368013BD3605DF89A
:10204000044B70470D2BF7D00E2BF8D1D3685DF8F9
:10205000044B0133D36070470C2B05D0F2D8092B09
:10206000D8D00B2BE8D0EAE7D3685DF8044B0233F5
:10207000D360704748F28C33C2F2010310B4D3F836
:102080009C201368506819780478507A137A0442B7
:1020900001EA03011AD0937A03F0030309B143F074
:1020A000040343F008039910082B91722AD8072BD8
:1020B00022D2032B2ED011D9042B13D0062B14D1EE
:1020C000D3685DF8044B023BD3607047937A03F00A
:1020D00003030029E7D043F00403E4E7012B0BD00E
:1020E000022B02D1D368013BD3605DF8044B7047EB
:1020F0000D2BF7D00E2BF8D1D3685DF8044B0133CC
:10210000D36070470C2B05D0F2D8092BD8D00B2BFD
:10211000E8D0EAE7D3685DF8044B0233D360704738
:1021200048F28C33C2F2010310B4D3F8A020136834
:10213000506819780478507A137A044201EA03014E
:102140001AD0937A03F0030309B143F0040343F078
:1021500008039910082B91722AD8072B22D2032B3F
:102160002ED011D9042B13D0062B14D1D3685DF8CF
:10217000044B023BD3607047937A03F003030029BA
:10218000E7D043F00403E4E7012B0BD0022B02D18C
:10219000D368013BD3605DF8044B70470D2BF7D03B
:1021A0000E2BF8D1D3685DF8044B0133D360704730
:1021B0000C2B05D0F2D8092BD8D00B2BE8D0EAE7AE
:1021C000D3685DF8044B0233D360704748F28C3318
:1021D000C2F2010310B4D3F8A42013685068197830
:1021E0000478507A137A044201EA03011AD0937AF0
:1021F00003F0030309B143F0040343F0080399100B
:10220000082B91722AD8072B22D2032B2ED011D95A
:10221000042B13D0062B14D1D3685DF8044B023B7A
:10222000D3607047937A03F003030029E7D043F0AB
:102230000403E4E7012B0BD0022B02D1D368013B4E
:10224000D3605DF8044B70470D2BF7D00E2BF8D1FF
:10225000D3685DF8044B0133D36070470C2B05D075
:10226000F2D8092BD8D00B2BE8D0EAE7D3685DF879
:10227000044B0233D360704748F28C33C2F201033F
:1022800010B4D3F8A8201368506819780478507AED
:10229000137A044201EA03011AD0937A03F003038C
:1022A00009B143F0040343F008039910082B91721D
:1022B0002AD8072B22D2032B2ED011D9042B13D0CE
:1022C000062B14D1D3685DF8044B023BD3607047F2
:1022D000937A03F003030029E7D043F00403E4E713
:1022E000012B0BD0022B02D1D368013BD3605DF8E8
:1022F000044B70470D2BF7D00E2BF8D1D3685DF847
:10230000044B0133D36070470C2B05D0F2D8092B56
:10231000D8D00B2BE8D0EAE7D3685DF8044B023342
:10232000D360704748F28C33C2F2010310B4D3F883
:10233000AC201368506819780478507A137A0442F4
:1023400001EA03011AD0937A03F0030309B143F0C1
:10235000040343F008039910082B91722AD8072B25
:1023600022D2032B2ED011D9042B13D0062B14D13B
:10237000D3685DF8044B023BD3607047937A03F057
:1023800003030029E7D043F00403E4E7012B0BD05B
:10239000022B02D1D368013BD3605DF8044B704738
:1023A0000D2BF7D00E2BF8D1D3685DF8044B013319
:1023B000D36070470C2B05D0F2D8092BD8D00B2B4B
:1023C000E8D0EAE7D3685DF8044B0233D360704786
:1023D00048F28C33C2F2010310B4D3F8B020136872
:1023E000506819780478507A137A044201EA03019C
:1023F0001AD0937A03F0030309B143F0040343F0C6
:1024000008039910082B91722AD8072B22D2032B8C
:102410002ED011D9042B13D0062B14D1D3685DF81C
:10242000044B023BD3607047937A03F00303002907
:10243000E7D043F00403E4E7012B0BD0022B02D1D9
:10244000D368013BD3605DF8044B70470D2BF7D088
:102450000E2BF8D1D3685DF8044B0133D36070477D
:102460000C2B05D0F2D8092BD8D00B2BE8D0EAE7FB
:10247000D3685DF8044B0233D360704748F28C3365
:10248000C2F2010310B4D3F8B4201368506819786D
:102490000478507A137A044201EA03011AD0937A3D
:1024A00003F0030309B143F0040343F00803991058
:1024B000082B91722AD8072B22D2032B2ED011D9A8
:1024C000042B13D0062B14D1D3685DF8044B023BC8
:1024D000D3607047937A03F003030029E7D043F0F9
:1024E0000403E4E7012B0BD0022B02D1D368013B9C
:1024F000D3605DF8044B70470D2BF7D00E2BF8D14D
:10250000D3685DF8044B0133D36070470C2B05D0C2
:10251000F2D8092BD8D00B2BE8D0EAE7D3685DF8C6
:10252000044B0233D360704748F28C33C2F201038C
:1025300010B4D3F8B8201368506819780478507A2A
:10254000137A044201EA03011AD0937A03F00303D9
:1025500009B143F0040343F008039910082B91726A
:102560002AD8072B22D2032B2ED011D9042B13D01B
:10257000062B14D1D3685DF8044B023BD36070473F
:10258000937A03F003030029E7D043F00403E4E760
:10259000012B0BD0022B02D1D368013BD3605DF835
:1025A000044B70470D2BF7D00E2BF8D1D3685DF894
:1025B000044B0133D36070470C2B05D0F2D8092BA4
:1025C000D8D00B2BE8D0EAE7D3685DF8044B023390
:1025D000D360704748F28C33C2F2010310B4D3F8D1
:1025E000BC201368506819780478507A137A044232
:1025F00001EA03011AD0937A03F0030309B143F00F
:10260000040343F008039910082B91722AD8072B72
:1026100022D2032B2ED011D9042B13D0062B14D188
:10262000D3685DF8044B023BD3607047937A03F0A4
:1026300003030029E7D043F00403E4E7012B0BD0A8
:10264000022B02D1D368013BD3605DF8044B704785
:102650000D2BF7D00E2BF8D1D3685DF8044B013366
:10266000D36070470C2B05D0F2D8092BD8D00B2B98
:10267000E8D0EAE7D3685DF8044B0233D3607047D3
:1026800048F28C33C2F2010310B4D3F8C0201368AF
:10269000506819780478507A137A044201EA0301E9
:1026A0001AD0937A03F0030309B143F0040343F013
:1026B00008039910082B91722AD8072B22D2032BDA
:1026C0002ED011D9042B13D0062B14D1D3685DF86A
:1026D000044B023BD3607047937A03F00303002955
:1026E000E7D043F00403E4E7012B0BD0022B02D127
:1026F000D368013BD3605DF8044B70470D2BF7D0D6
:102700000E2BF8D1D3685DF8044B0133D3607047CA
:102710000C2B05D0F2D8092BD8D00B2BE8D0EAE748
:10272000D3685DF8044B0233D360704748F28C33B2
:10273000C2F2010310B4D3F8C420136850681978AA
:102740000478507A137A044201EA03011AD0937A8A
:1027500003F0030309B143F0040343F008039910A5
:10276000082B91722AD8072B22D2032B2ED011D9F5
:10277000042B13D0062B14D1D3685DF8044B023B15
:10278000D3607047937A03F003030029E7D043F046
:102790000403E4E7012B0BD0022B02D1D368013BE9
:1027A000D3605DF8044B70470D2BF7D00E2BF8D19A
:1027B000D3685DF8044B0133D36070470C2B05D010
:1027C000F2D8092BD8D00B2BE8D0EAE7D3685DF814
:1027D000044B0233D360704748F28C33C2F20103DA
:1027E00010B4D3F8C8201368506819780478507A68
:1027F000137A044201EA03011AD0937A03F0030327
:1028000009B143F0040343F008039910082B9172B7
:102810002AD8072B22D2032B2ED011D9042B13D068
:10282000062B14D1D3685DF8044B023BD36070478C
:10283000937A03F003030029E7D043F00403E4E7AD
:10284000012B0BD0022B02D1D368013BD3605DF882
:10285000044B70470D2BF7D00E2BF8D1D3685DF8E1
:10286000044B0133D36070470C2B05D0F2D8092BF1
:10287000D8D00B2BE8D0EAE7D3685DF8044B0233DD
:10288000D360704748F28C33C2F2010310B4D3F81E
:10289000CC201368506819780478507A137A04426F
:1028A00001EA03011AD0937A03F0030309B143F05C
:1028B000040343F008039910082B91722AD8072BC0
:1028C00022D2032B2ED011D9042B13D0062B14D1D6
:1028D000D3685DF8044B023BD3607047937A03F0F2
:1028E00003030029E7D043F00403E4E7012B0BD0F6
:1028F000022B02D1D368013BD3605DF8044B7047D3
:102900000D2BF7D00E2BF8D1D3685DF8044B0133B3
:10291000D36070470C2B05D0F2D8092BD8D00B2BE5
:10292000E8D0EAE7D3685DF8044B0233D360704720
:1029300048F28C33C2F2010310B4D3F8D0201368EC
:10294000506819780478507A137A044201EA030136
:102950001AD0937A03F0030309B143F0040343F060
:1029600008039910082B91722AD8072B22D2032B27
:102970002ED011D9042B13D0062B14D1D3685DF8B7
:10298000044B023BD3607047937A03F003030029A2
:10299000E7D043F00403E4E7012B0BD0022B02D174
:1029A000D368013BD3605DF8044B70470D2BF7D023
:1029B0000E2BF8D1D3685DF8044B0133D360704718
:1029C0000C2B05D0F2D8092BD8D00B2BE8D0EAE796
:1029D000D3685DF8044B0233D360704748F28C3300
:1029E000C2F2010310B4D3F8D420136850681978E8
:1029F0000478507A137A044201EA03011AD0937AD8
:102A000003F0030309B143F0040343F008039910F2
:102A1000082B91722AD8072B22D2032B2ED011D942
:102A2000042B13D0062B14D1D3685DF8044B023B62
:102A3000D3607047937A03F003030029E7D043F093
:102A40000403E4E7012B0BD0022B02D1D368013B36
:102A5000D3605DF8044B70470D2BF7D00E2BF8D1E7
:102A6000D3685DF8044B0133D36070470C2B05D05D
:102A7000F2D8092BD8D00B2BE8D0EAE7D3685DF861
:102A8000044B0233D360704748F28C33C2F2010327
:102A900010B4D3F8D8201368506819780478507AA5
:102AA000137A044201EA03011AD0937A03F0030374
:102AB00009B143F0040343F008039910082B917205
:102AC0002AD8072B22D2032B2ED011D9042B13D0B6
:102AD000062B14D1D3685DF8044B023BD3607047DA
:102AE000937A03F003030029E7D043F00403E4E7FB
:102AF000012B0BD0022B02D1D368013BD3605DF8D0
:102B0000044B70470D2BF7D00E2BF8D1D3685DF82E
:102B1000044B0133D36070470C2B05D0F2D8092B3E
:102B2000D8D00B2BE8D0EAE7D3685DF8044B02332A
:102B3000D360704748F28C33C2F2010310B4D3F86B
:102B4000DC201368506819780478507A137A0442AC
:102B500001EA03011AD0937A03F0030309B143F0A9
:102B6000040343F008039910082B91722AD8072B0D
:102B700022D2032B2ED011D9042B13D0062B14D123
:102B8000D3685DF8044B023BD3607047937A03F03F
:102B900003030029E7D043F00403E4E7012B0BD043
:102BA000022B02D1D368013BD3605DF8044B704720
:102BB0000D2BF7D00E2BF8D1D3685DF8044B013301
:102BC000D36070470C2B05D0F2D8092BD8D00B2B33
:102BD000E8D0EAE7D3685DF8044B0233D36070476E
:102BE00048F28C33C2F2010310B41A6A13685068B9
:102BF00019780478507A137A044201EA03011AD052
:102C0000937A03F0030309B143F0040343F008038C
:102C10009910082B91722AD8072B22D2032B2ED081
:102C200011D9042B13D0062B14D1D3685DF8044BB3
:102C3000023BD3607047937A03F003030029E7D087
:102C400043F00403E4E7012B0BD0022B02D1D3683D
:102C5000013BD3605DF8044B70470D2BF7D00E2B72
:102C6000F8D1D3685DF8044B0133D36070470C2B67
:102C700005D0F2D8092BD8D00B2BE8D0EAE7D368DF
:102C80005DF8044B0233D360704700BF48F28C33C9
:102C9000C2F2010310B45A6A1368506819780478B4
:102CA000507A137A044201EA03011AD0937A03F0AE
:102CB000030309B143F0040343F008039910082B00
:102CC00091722AD8072B22D2032B2ED011D9042B94
:102CD00013D0062B14D1D3685DF8044B023BD360AC
:102CE0007047937A03F003030029E7D043F004030D
:102CF000E4E7012B0BD0022B02D1D368013BD36058
:102D00005DF8044B70470D2BF7D00E2BF8D1D3682C
:102D10005DF8044B0133D36070470C2B05D0F2D81B
:102D2000092BD8D00B2BE8D0EAE7D3685DF8044B29
:102D30000233D360704700BF48F28C33C2F2010304
:102D400010B49A6A1368506819780478507A137A24
:102D5000044201EA03011AD0937A03F0030309B194
:102D600043F0040343F008039910082B91722AD80A
:102D7000072B22D2032B2ED011D9042B13D0062BD4
:102D800014D1D3685DF8044B023BD3607047937A4B
:102D900003F003030029E7D043F00403E4E7012B29
:102DA0000BD0022B02D1D368013BD3605DF8044BFA
:102DB00070470D2BF7D00E2BF8D1D3685DF8044B7C
:102DC0000133D36070470C2B05D0F2D8092BD8D033
:102DD0000B2BE8D0EAE7D3685DF8044B0233D360ED
:102DE000704700BF48F28C33C2F2010310B4DA6AB4
:102DF0001368506819780478507A137A044201EA0B
:102E000003011AD0937A03F0030309B143F00403DA
:102E100043F008039910082B91722AD8072B22D26D
:102E2000032B2ED011D9042B13D0062B14D1D36829
:102E30005DF8044B023BD3607047937A03F00303C1
:102E40000029E7D043F00403E4E7012B0BD0022B69
:102E500002D1D368013BD3605DF8044B70470D2B62
:102E6000F7D00E2BF8D1D3685DF8044B0133D36053
:102E700070470C2B05D0F2D8092BD8D00B2BE8D0FB
:102E8000EAE7D3685DF8044B0233D360704700BFB4
:102E900048F28C33C2F2010310B41A6B1368506805
:102EA00019780478507A137A044201EA03011AD09F
:102EB000937A03F0030309B143F0040343F00803DA
:102EC0009910082B91722AD8072B22D2032B2ED0CF
:102ED00011D9042B13D0062B14D1D3685DF8044B01
:102EE000023BD3607047937A03F003030029E7D0D5
:102EF00043F00403E4E7012B0BD0022B02D1D3688B
:102F0000013BD3605DF8044B70470D2BF7D00E2BBF
:102F1000F8D1D3685DF8044B0133D36070470C2BB4
:102F200005D0F2D8092BD8D00B2BE8D0EAE7D3682C
:102F30005DF8044B0233D360704700BF48F28C3316
:102F4000C2F2010310B45A6B136850681978047800
:102F5000507A137A044201EA03011AD0937A03F0FB
:102F6000030309B143F0040343F008039910082B4D
:102F700091722AD8072B22D2032B2ED011D9042BE1
:102F800013D0062B14D1D3685DF8044B023BD360F9
:102F90007047937A03F003030029E7D043F004035A
:102FA000E4E7012B0BD0022B02D1D368013BD360A5
:102FB0005DF8044B70470D2BF7D00E2BF8D1D3687A
:102FC0005DF8044B0133D36070470C2B05D0F2D869
:102FD000092BD8D00B2BE8D0EAE7D3685DF8044B77
:102FE0000233D360704700BF48F28C33C2F2010352
:102FF00010B49A6B1368506819780478507A137A71
:10300000044201EA03011AD0937A03F0030309B1E1
:1030100043F0040343F008039910082B91722AD857
:10302000072B22D2032B2ED011D9042B13D0062B21
:1030300014D1D3685DF8044B023BD3607047937A98
:1030400003F003030029E7D043F00403E4E7012B76
:103050000BD0022B02D1D368013BD3605DF8044B47
:1030600070470D2BF7D00E2BF8D1D3685DF8044BC9
:103070000133D36070470C2B05D0F2D8092BD8D080
:103080000B2BE8D0EAE7D3685DF8044B0233D3603A
:10309000704700BF48F28C33C2F2010310B4DA6B00
:1030A0001368506819780478507A137A044201EA58
:1030B00003011AD0937A03F0030309B143F0040328
:1030C00043F008039910082B91722AD8072B22D2BB
:1030D000032B2ED011D9042B13D0062B14D1D36877
:1030E0005DF8044B023BD3607047937A03F003030F
:1030F0000029E7D043F00403E4E7012B0BD0022BB7
:1031000002D1D368013BD3605DF8044B70470D2BAF
:10311000F7D00E2BF8D1D3685DF8044B0133D360A0
:1031200070470C2B05D0F2D8092BD8D00B2BE8D048
:10313000EAE7D3685DF8044B0233D360704700BF01
:1031400048F28C33C2F2010310B41A6C1368506851
:1031500019780478507A137A044201EA03011AD0EC
:10316000937A03F0030309B143F0040343F0080327
:103170009910082B91722AD8072B22D2032B2ED01C
:1031800011D9042B13D0062B14D1D3685DF8044B4E
:10319000023BD3607047937A03F003030029E7D022
:1031A00043F00403E4E7012B0BD0022B02D1D368D8
:1031B000013BD3605DF8044B70470D2BF7D00E2B0D
:1031C000F8D1D3685DF8044B0133D36070470C2B02
:1031D00005D0F2D8092BD8D00B2BE8D0EAE7D3687A
:1031E0005DF8044B0233D360704700BF48F28C3364
:1031F000C2F2010310B45A6C13685068197804784D
:10320000507A137A044201EA03011AD0937A03F048
:10321000030309B143F0040343F008039910082B9A
:1032200091722AD8072B22D2032B2ED011D9042B2E
:1032300013D0062B14D1D3685DF8044B023BD36046
:103240007047937A03F003030029E7D043F00403A7
:10325000E4E7012B0BD0022B02D1D368013BD360F2
:103260005DF8044B70470D2BF7D00E2BF8D1D368C7
:103270005DF8044B0133D36070470C2B05D0F2D8B6
:10328000092BD8D00B2BE8D0EAE7D3685DF8044BC4
:103290000233D360704700BF48F28C33C2F201039F
:1032A00010B49A6C1368506819780478507A137ABD
:1032B000044201EA03011AD0937A03F0030309B12F
:1032C00043F0040343F008039910082B91722AD8A5
:1032D000072B22D2032B2ED011D9042B13D0062B6F
:1032E00014D1D3685DF8044B023BD3607047937AE6
:1032F00003F003030029E7D043F00403E4E7012BC4
:103300000BD0022B02D1D368013BD3605DF8044B94
:1033100070470D2BF7D00E2BF8D1D3685DF8044B16
:103320000133D36070470C2B05D0F2D8092BD8D0CD
:103330000B2BE8D0EAE7D3685DF8044B0233D36087
:10334000704700BF48F28C33C2F2010310B4DA6C4C
:103350001368506819780478507A137A044201EAA5
:1033600003011AD0937A03F0030309B143F0040375
:1033700043F008039910082B91722AD8072B22D208
:10338000032B2ED011D9042B13D0062B14D1D368C4
:103390005DF8044B023BD3607047937A03F003035C
:1033A0000029E7D043F00403E4E7012B0BD0022B04
:1033B00002D1D368013BD3605DF8044B70470D2BFD
:1033C000F7D00E2BF8D1D3685DF8044B0133D360EE
:1033D00070470C2B05D0F2D8092BD8D00B2BE8D096
:1033E000EAE7D3685DF8044B0233D360704700BF4F
:1033F00048F28C33C2F2010310B41A6D136850689E
:1034000019780478507A137A044201EA03011AD039
:10341000937A03F0030309B143F0040343F0080374
:103420009910082B91722AD8072B22D2032B2ED069
:1034300011D9042B13D0062B14D1D3685DF8044B9B
:10344000023BD3607047937A03F003030029E7D06F
:1034500043F00403E4E7012B0BD0022B02D1D36825
:10346000013BD3605DF8044B70470D2BF7D00E2B5A
:10347000F8D1D3685DF8044B0133D36070470C2B4F
:1034800005D0F2D8092BD8D00B2BE8D0EAE7D368C7
:103490005DF8044B0233D360704700BF48F28C33B1
:1034A000C2F2010310B45A6D136850681978047899
:1034B000507A137A044201EA03011AD0937A03F096
:1034C000030309B143F0040343F008039910082BE8
:1034D00091722AD8072B22D2032B2ED011D9042B7C
:1034E00013D0062B14D1D3685DF8044B023BD36094
:1034F0007047937A03F003030029E7D043F00403F5
:10350000E4E7012B0BD0022B02D1D368013BD3603F
:103510005DF8044B70470D2BF7D00E2BF8D1D36814
:103520005DF8044B0133D36070470C2B05D0F2D803
:10353000092BD8D00B2BE8D0EAE7D3685DF8044B11
:103540000233D360704700BF48F28C33C2F20103EC
:1035500010B49A6D1368506819780478507A137A09
:10356000044201EA03011AD0937A03F0030309B17C
:1035700043F0040343F008039910082B91722AD8F2
:10358000072B22D2032B2ED011D9042B13D0062BBC
:1035900014D1D3685DF8044B023BD3607047937A33
:1035A00003F003030029E7D043F00403E4E7012B11
:1035B0000BD0022B02D1D368013BD3605DF8044BE2
:1035C00070470D2BF7D00E2BF8D1D3685DF8044B64
:1035D0000133D36070470C2B05D0F2D8092BD8D01B
:1035E0000B2BE8D0EAE7D3685DF8044B0233D360D5
:1035F000704700BF48F28C33C2F2010310B4DA6D99
:103600001368506819780478507A137A044201EAF2
:1036100003011AD0937A03F0030309B143F00403C2
:1036200043F008039910082B91722AD8072B22D255
:10363000032B2ED011D9042B13D0062B14D1D36811
:103640005DF8044B023BD3607047937A03F00303A9
:103650000029E7D043F00403E4E7012B0BD0022B51
:1036600002D1D368013BD3605DF8044B70470D2B4A
:10367000F7D00E2BF8D1D3685DF8044B0133D3603B
:1036800070470C2B05D0F2D8092BD8D00B2BE8D0E3
:10369000EAE7D3685DF8044B0233D360704700BF9C
:1036A00048F28C33C2F2010310B4D3F8E02013685F
:1036B000506819780478507A137A044201EA0301B9
:1036C0001AD0937A03F0030309B143F0040343F0E3
:1036D00008039910082B91722AD8072B22D2032BAA
:1036E0002ED011D9042B13D0062B14D1D3685DF83A
:1036F000044B023BD3607047937A03F00303002925
:10370000E7D043F00403E4E7012B0BD0022B02D1F6
:10371000D368013BD3605DF8044B70470D2BF7D0A5
:103720000E2BF8D1D3685DF8044B0133D36070479A
:103730000C2B05D0F2D8092BD8D00B2BE8D0EAE718
:10374000D3685DF8044B0233D360704748F28C3382
:10375000C2F2010310B4D3F8E4201368506819785A
:103760000478507A137A044201EA03011AD0937A5A
:1037700003F0030309B143F0040343F00803991075
:10378000082B91722AD8072B22D2032B2ED011D9C5
:10379000042B13D0062B14D1D3685DF8044B023BE5
:1037A000D3607047937A03F003030029E7D043F016
:1037B0000403E4E7012B0BD0022B02D1D368013BB9
:1037C000D3605DF8044B70470D2BF7D00E2BF8D16A
:1037D000D3685DF8044B0133D36070470C2B05D0E0
:1037E000F2D8092BD8D00B2BE8D0EAE7D3685DF8E4
:1037F000044B0233D360704748F28C33C2F20103AA
:1038000010B4D3F8E8201368506819780478507A17
:10381000137A044201EA03011AD0937A03F00303F6
:1038200009B143F0040343F008039910082B917287
:103830002AD8072B22D2032B2ED011D9042B13D038
:10384000062B14D1D3685DF8044B023BD36070475C
:10385000937A03F003030029E7D043F00403E4E77D
:10386000012B0BD0022B02D1D368013BD3605DF852
:10387000044B70470D2BF7D00E2BF8D1D3685DF8B1
:10388000044B0133D36070470C2B05D0F2D8092BC1
:10389000D8D00B2BE8D0EAE7D3685DF8044B0233AD
:1038A000D360704748F28C33C2F2010310B4D3F8EE
:1038B000EC201368506819780478507A137A04421F
:1038C00001EA03011AD0937A03F0030309B143F02C
:1038D000040343F008039910082B91722AD8072B90
:1038E00022D2032B2ED011D9042B13D0062B14D1A6
:1038F000D3685DF8044B023BD3607047937A03F0C2
:1039000003030029E7D043F00403E4E7012B0BD0C5
:10391000022B02D1D368013BD3605DF8044B7047A2
:103920000D2BF7D00E2BF8D1D3685DF8044B013383
:10393000D36070470C2B05D0F2D8092BD8D00B2BB5
:10394000E8D0EAE7D3685DF8044B0233D3607047F0
:10395000F0B540F66453C2F201034DF20A721B68DF
:10396000C3F6234206EE102A93F89D2093F89F6039
:1039700007EE102A93F89620B8EEC77A07EE902A41
:1039800027EE067AF8EEE76A83B067EE267A0D46F0
:10399000FCEEE77A0021CDED017A044683F89350DE
:1039A0009DF8042083F8921083F8911083F890100A
:1039B0000EB183F8902093F89E1009B183F89120FE
:1039C00093F8A01009B183F8922093F8A52093F8FA
:1039D000A70007EE102A4DF20A72C3F6234206EE44
:1039E000102A93F89420B8EEC77A07EE902A27EEB3
:1039F000067AF8EEE76A67EE267AFCEEE77ACDED16
:103A0000017A9DF8042030B193F89000904238BFBD
:103A1000104683F8900093F8A60030B193F8910017
:103A2000904238BF104683F8910093F8A80030B157
:103A300093F89260B24238BF324683F8922093F8EE
:103A4000A12093F8A36007EE102A4DF20A72C3F684
:103A5000234206EE102A93F89520B8EEC77A07EEB7
:103A6000902A27EE067AF8EEE76A67EE267AFCEEF1
:103A7000E77ACDED017A9DF8042036B193F8906095
:103A8000964238BF164683F8906093F8A26036B12C
:103A900093F89160964238BF164683F8916093F888
:103AA000A46036B193F89270BA4238BF3A4683F8B0
:103AB000922093F8A92093F8AB7007EE902A4DF26C
:103AC0000A72C3F6234207EE102AF8EEE77A67EE91
:103AD000877A07EE105AB8EEC77A67EE877AFCEE5F
:103AE000E77ACDED017A9DF8042037B193F8907014
:103AF000974238BF174683F8907093F8AA7037B191
:103B000093F89170974238BF174683F8917093F8F5
:103B1000AC7037B193F892E0724538BF724683F8C3
:103B2000922029B926B918B917B97F2283F89220B3
:103B300043F22C100D21C0F2020018F007F8611EAC
:103B4000C9B20F290FD840F67474C2F2010441F0D3
:103B5000D001A06C03681B689847A06C036805F04F
:103B60007F011B68984742F6A8700F21C0F202003F
:103B700017F0ECFF4EF20020C2F2000003B0BDE8E7
:103B8000F04018F0F5BE00BFF0B540F66453C2F245
:103B900001034DF20A721B68C3F6234206EE102A97
:103BA00093F89D2093F89F6007EE102A93F89620D3
:103BB000B8EEC77A07EE902A27EE067AF8EEE76AA3
:103BC00083B067EE267A0C46FCEEE77A0021CDED55
:103BD000017A054683F893409DF8042083F89210FB
:103BE00083F8911083F890100EB183F8902093F829
:103BF0009E1009B183F8912093F8A01009B183F8C1
:103C0000922093F8A52093F8A70007EE102A4DF212
:103C10000A72C3F6234206EE102A93F89420B8EEF7
:103C2000C77A07EE902A27EE067AF8EEE76A67EE83
:103C3000267AFCEEE77ACDED017A9DF8042030B1CA
:103C400093F89000904238BF104683F8900093F8A4
:103C5000A60030B193F89100904238BF104683F827
:103C6000910093F8A80030B193F89260B24238BF47
:103C7000324683F8922093F8A12093F8A36007EED0
:103C8000102A4DF20A72C3F6234206EE102A93F868
:103C90009520B8EEC77A07EE902A27EE067AF8EE5E
:103CA000E76A67EE267AFCEEE77ACDED017A9DF8B9
:103CB000042036B193F89060964238BF164683F8D8
:103CC000906093F8A26036B193F89160964238BF45
:103CD000164683F8916093F8A46036B193F8927019
:103CE000BA4238BF3A4683F8922093F8A92093F855
:103CF000AB7007EE902A4DF20A72C3F6234207EE2C
:103D0000102AF8EEE77A67EE877A07EE104AB8EEE7
:103D1000C77A67EE877AFCEEE77ACDED017A9DF8F7
:103D2000042037B193F89070974238BF174683F854
:103D3000907093F8AA7037B193F89170974238BF9A
:103D4000174683F8917093F8AC7037B193F892E00E
:103D5000724538BF724683F8922029B926B918B93E
:103D600017B97F2283F8922043F23C100D21C0F254
:103D70000200240417F0EAFE04F4FE04681E44F472
:103D80005044000244F00D0400F47060204317F02A
:103D900053F842F600700F21C0F2020017F0D6FE71
:103DA0004EF20020C2F2000003B0BDE8F04018F06F
:103DB000DFBD00BF70B5044643F24C100E46C0F2A2
:103DC00002001221154617F0C1FE611EC9B20F296B
:103DD00015D840F67474C2F2010441F0A001A06C41
:103DE00003681B689847A06C036806F07F011B6896
:103DF0009847A06C036805F07F011B68984743F261
:103E00006010C0F202000A2117F0A0FE4EF200205E
:103E1000C2F20000BDE8704018F0AABDF8B54DF63A
:103E20008867C2F2000705463B7C0E4614467BB30A
:103E300098422DD043F26C101E21C0F2020017F000
:103E400085FE4EF2002000230A222946C2F200001D
:103E500018F0A0FD43F28C100E21C0F2020017F002
:103E600075FE4EF20020397C00230A22C2F20000C7
:103E700018F090FD43F29C100121C0F2020017F0EF
:103E800065FE4EF20020C2F2000018F071FD08E05D
:103E900040F66453C2F201032246186831460BF023
:103EA0006BFB43F2A0101121C0F2020017F04EFE8E
:103EB000230603F0FE43300443F41043013D43F076
:103EC000090300F4FE002D02184305F47065284331
:103ED00016F0B2FF42F60070C0F202000F2117F098
:103EE00035FE4EF20020C2F20000BDE8F84018F0A6
:103EF0003FBD00BFF8B54DF68867C2F20007054622
:103F00003B7C0E4614467BB398422DD043F26C1096
:103F10001E21C0F2020017F019FE4EF2002000230D
:103F20000A222946C2F2000018F034FD43F28C1038
:103F30000E21C0F2020017F009FE4EF20020397C7B
:103F400000230A22C2F2000018F024FD43F29C1064
:103F50000121C0F2020017F0F9FD4EF20020C2F27A
:103F6000000018F005FD07E040F66453C2F20103BB
:103F7000314618680BF0C8FC43F2B4101221C0F2AD
:103F8000020017F0E3FD230603F0FE43300443F480
:103F90000043013D43F0080300F4FE002D021843E6
:103FA00005F47065284316F047FF42F60070C0F232
:103FB00002000F2117F0CAFD4EF20020C2F20000ED
:103FC000BDE8F84018F0D4BCF8B54DF68865C2F2EB
:103FD000000504462B7C0E4617467BB398422DD035
:103FE00043F26C101E21C0F2020017F0AFFD4EF23A
:103FF000002000230A222146C2F2000018F0CAFC69
:1040000043F28C100E21C0F2020017F09FFD4EF219
:104010000020297C00230A22C2F2000018F0BAFC1A
:1040200043F29C100121C0F2020017F08FFD4EF206
:104030000020C2F2000018F09BFC08E040F6645338
:10404000C2F201033A46186831460BF095FA43F282
:10405000C8101121C0F20200013C17F077FDE1B257
:104060000F2915D840F67475C2F2010541F0900190
:10407000A86C03681B689847A86C036806F07F016A
:104080001B689847A86C036807F07F011B68984776
:1040900042F6A870C0F202000F2117F057FD4EF251
:1040A0000020C2F20000BDE8F84018F061BC00BF7B
:1040B000F8B54DF68865C2F2000504462B7C0E4625
:1040C00017467BB398422DD043F26C101E21C0F2EC
:1040D000020017F03BFD4EF2002000230A22214689
:1040E000C2F2000018F056FC43F28C100E21C0F210
:1040F000020017F02BFD4EF20020297C00230A223B
:10410000C2F2000018F046FC43F29C100121C0F2FC
:10411000020017F01BFD4EF20020C2F2000018F062
:1041200027FC07E040F66453C2F2010331461868E9
:104130000BF0EAFB43F2DC101221C0F20200013C5A
:1041400017F004FDE1B20F2915D840F67475C2F2DC
:10415000010541F08001A86C03681B689847A86CB2
:10416000036806F07F011B689847A86C036807F096
:104170007F011B68984742F6A870C0F202000F2129
:1041800017F0E4FC4EF20020C2F20000BDE8F84057
:1041900018F0EEBB38B540F66453C2F20103044692
:1041A0001B6801F5005543F2F0100D21C3F884504F
:1041B000C0F2020017F0CAFC611EC9B20F2915D85F
:1041C00040F67474C2F2010441F0E001A06C03688F
:1041D0001B689847A06C036805F07F011B6898472F
:1041E000A06C0368C5F3C6111B68984742F6A87017
:1041F000C0F202000F2117F0A9FC4EF20020C2F21B
:104200000000BDE8384018F0B3BB00BF10B442F660
:1042100090640023C0F202044172026104600372E0
:10422000C36041B1194600E0026942F82310427AA6
:1042300001339A42F8DC48F23463C2F201031A688F
:104240000AB90CE01A465369002BFBD150610023D8
:1042500043618380C38083725DF8044B70471860AC
:10426000F5E700BFF8B540F67474C2F2010447F6F2
:104270001221A06C0368DB69984743F6F5670320B9
:1042800043F61D6346F6711143F6893640F6B9626E
:1042900084F86400C0F20003C0F20007C0F200011D
:1042A000C0F20006C0F2000240F66550636027606D
:1042B000E1606661A261C0F2000045F65D4340F630
:1042C000E14740F6C95140F69D4640F6E5122061AF
:1042D000C0F20003C0F20007C0F20001C0F2000605
:1042E000C0F2000240F6B970E3612762A160A662E5
:1042F000E262C0F2000040F6AD1340F61D2740F622
:10430000552140F68D2640F6C522C0F200022063FA
:10431000C0F20003C0F20007C0F20001C0F20006C4
:104320004EF2002543F200206264C2F2000563638E
:10433000A76300234FF6FF77E16326641721C0F2DD
:10434000020084F84C3084F84E3084F84D30A36578
:10435000636584F8E93084F8663084F8653084F861
:10436000673084F86830E765276617F0EFFB28466A
:1043700018F0FEFA48F21C61C2F2010143F6C97E50
:10438000C0F2000E48F21464C1F800E0C2F2010469
:1043900044F2B10EC0F2000E48F21863C4F800E017
:1043A000C2F2010346F6950EC0F2000E48F2EC5739
:1043B000C3F800E0C2F2010743F6511EC0F2000E3E
:1043C00048F2DC50C7F800E0C2F2010044F2951E4A
:1043D000C0F2000E48F2D856C0F800E0C2F2010662
:1043E00041F2910EC0F2000E48F2FC52C6F800E015
:1043F000C2F2010245F69D4EC0F2000E48F2F451A1
:10440000C2F800E0C2F2010140F61D6EC0F2000EDB
:1044100048F2E854C1F800E0C2F2010443F6B55E88
:10442000C0F2000E48F21063C4F800E0C2F20103CB
:1044300040F6696EC0F2000E48F2F857C3F800E08B
:10444000C2F2010740F6255EC0F2000E48F2C050ED
:10445000C7F800E0C2F2010041F22107C0F20007F4
:1044600048F2F0560760C2F2010648F2D05240F618
:104470002D37C2F20102C0F2000748F2086140F68F
:104480006D303760C2F20101C0F2000048F2C8543A
:1044900048F2C45340F6AD37C2F201031060C2F2D5
:1044A0000104C0F2000740F6ED3640F62D4243F21B
:1044B00018200F60C0F20006C0F20002C0F2020035
:1044C000182126601A6017F041FB2846BDE8F84025
:1044D00018F04EBA4DF20A73C3F6234306EE103AB3
:1044E000437EC17E07EE103A837CB8EEC77A07EEB2
:1044F000903A70B4F8EEE76A27EE067A83B067EE7A
:10450000267A0022FCEEE77A8273CDED017A4273BF
:104510009DF80430027301B10373827E02B14373CC
:10452000027F02B1837390F8213090F8231007EED8
:10453000103A4DF20A73C3F6234306EE103A037C99
:10454000B8EEC77A07EE903A27EE067AF8EEE76AF9
:1045500067EE267AFCEEE77ACDED017A9DF804301D
:1045600021B1017B994238BF1946017390F822109E
:1045700021B1417B994238BF1946417390F82440DC
:1045800024B1817B8B4238BF0B468373437FC17F4D
:1045900007EE103A4DF20A73C3F6234306EE103AC3
:1045A000437CB8EEC77A07EE903A27EE067AF8EE2B
:1045B000E76A67EE267AFCEEE77ACDED017A9DF8A0
:1045C000043021B1017B994238BF19460173817FC4
:1045D00021B1417B994238BF1946417390F82010B0
:1045E00021B1857BAB4238BF2B46837390F82530D1
:1045F00090F8275007EE103A4DF20A73C3F62343A2
:1046000006EE103AC37BB8EEC77A07EE903A27EE73
:10461000067AF8EEE76A67EE267AFCEEE77ACDEDE9
:10462000017A9DF8043025B1057B9D4238BF1D46B7
:10463000057390F8265025B1457B9D4238BF1D4635
:10464000457390F8285025B1867BB34238BF334676
:10465000837322B919B914B90DB97F23837303B0D9
:1046600070BC70471D2810B50B4600F0E983024668
:1046700022D92C2800F064813FD8242800F0EE8352
:1046800040F2A880282800F0748300F2D680262803
:1046900000F0F58140F2D58248F28C34C2F2010478
:1046A00042F27501C0F2000104222720C4F89C30B8
:1046B00015F0F4F8012010BD0E2800F097833AD8C9
:1046C000062800F0A1836CD90A2800F0058300F2C7
:1046D0000781082800F07E8140F2758248F28C3410
:1046E000C2F2010442F68D41C0F200010422092009
:1046F000636215F0D3F8012010BD342800F0BD83AB
:1047000036D8302800F0638300F2D6802E2800F0DF
:10471000528140F2018248F28C34C2F2010442F22A
:10472000D551C0F2000104222F20C4F8BC3015F08E
:10473000B5F8012010BD152800F0748364D919283C
:1047400000F0FA8100F2A580172800F08A8140F27B
:10475000D18248F28C34C2F2010441F26161C0F2AC
:10476000000104221820236615F098F8012010BDDE
:10477000382800F0CE8275D8362800F0398140F212
:104780007F8248F28C34C2F2010442F63531C0F225
:10479000000104223720C4F8DC3015F07FF8012036
:1047A00010BD022800F0018240F27881042800F058
:1047B0004B8140F2BD8248F28C34C2F2010441F2D6
:1047C0005D41C0F2000104220520636115F066F826
:1047D000012010BD202800F0448240F28981222867
:1047E00000F0238140F2D48248F28C34C2F20104FA
:1047F00041F6C551C0F2000104222320C4F88C30D8
:1048000015F04CF8012010BD112800F0B18140F2E4
:104810005A81132800F0FB8040F2B88148F28C34B2
:10482000C2F2010443F2F131C0F20001042214206B
:10483000236515F033F8012010BD2A2800F0AC8064
:1048400040F2E08148F28C34C2F2010442F2253198
:10485000C0F2000104222B20C4F8AC3015F01EF881
:10486000012010BD3A2800F08880C0F072823B28F9
:1048700040F06D8248F28C34C2F2010443F6A50187
:10488000C0F200010422C4F8EC3015F007F8012052
:1048900010BD1B2863D040F28B8248F28C34C2F2E8
:1048A000010441F61111C0F2000104221C2023670B
:1048B00014F0F4FF012010BD322824D040F2928180
:1048C00048F28C34C2F2010442F68501C0F20001C4
:1048D00004223320C4F8CC3014F0E0FF012010BDD6
:1048E0000C281FD040F29E8148F28C34C2F20104A1
:1048F00042F63D71C0F2000104220D20636314F002
:10490000CDFF012010BD48F28C34C2F2010442F206
:10491000D971C0F200010422C4F8C83014F0BEFFFF
:10492000012010BD48F28C34C2F2010442F69161BC
:10493000C0F200010422236314F0B0FF012010BD77
:1049400048F28C34C2F2010442F2D131C0F20001CB
:104950000422C4F8B03014F0A1FF012010BD48F2C9
:104960008C34C2F2010441F66501C0F20001042258
:10497000E36614F093FF012010BD48F28C34C2F2BC
:10498000010443F2F971C0F200010422C4F8E830D6
:1049900014F084FF012010BD48F28C34C2F20104EF
:1049A00042F27921C0F200010422C4F8A83014F0C8
:1049B00075FF012010BD48F28C34C2F2010442F2AE
:1049C0002951C0F200010422C4F8B83014F066FF87
:1049D000012010BD48F28C34C2F2010442F6E131EC
:1049E000C0F200010422236214F058FF012010BD20
:1049F00048F28C34C2F2010442F68921C0F200016F
:104A00000422C4F8D83014F049FF012010BD48F248
:104A10008C34C2F2010443F24531C0F20001042299
:104A2000E36414F03BFF012010BD48F28C34C2F265
:104A3000010441F61951C0F200010422C4F8883083
:104A400014F02CFF012010BD48F28C34C2F2010496
:104A500041F2B131C0F20001236114F01FFF0120C7
:104A600010BD48F28C34C2F2010443F2F551C0F299
:104A700000010422E36514F011FF012010BD48F28B
:104A80008C34C2F2010441F6C971C0F20001042263
:104A9000C4F8983014F002FF012010BD002800F087
:104AA000FF80012840F0538148F28C34C2F20104A7
:104AB00041F2AD11C0F2000104220120636014F044
:104AC000EDFE012010BD0F2800F0F880102840F006
:104AD0003E8148F28C34C2F2010443F24111C0F22B
:104AE000000104221020236414F0D8FE012010BD20
:104AF0001E282FD01F2840F02A8148F28C34C2F2A1
:104B0000010441F61531C0F2000104221F20E367C1
:104B100014F0C4FE012010BD48F28C34C2F201042E
:104B200042F27D41C0F2000104222D20C4F8B430CD
:104B300014F0B4FE012010BD48F28C34C2F201041E
:104B400041F20D71C0F200010422636614F0A6FE6A
:104B5000012010BD48F28C34C2F2010441F66921F3
:104B6000C0F200010422A36714F098FE012010BDDA
:104B700048F28C34C2F2010443F2ED11C0F200019C
:104B80000422636414F08AFE012010BD48F28C34C4
:104B9000C2F2010443F29921C0F200010422122062
:104BA000A36414F07BFE012010BD48F28C34C2F2E5
:104BB000010441F25921C0F200010422A36014F063
:104BC0006DFE012010BD48F28C34C2F2010441F2A6
:104BD000B551C0F2000104220720E36114F05EFE2B
:104BE000012010BD48F28C34C2F2010442F22D7152
:104BF000C0F2000104223120C4F8C43014F04EFE8B
:104C0000012010BD48F28C34C2F2010442F2CD11F1
:104C1000C0F2000104222920C4F8A43014F03EFEA2
:104C2000012010BD48F28C34C2F2010442F6E55175
:104C3000C0F2000104220B20E36214F02FFE0120D9
:104C400010BD48F28C34C2F2010441F61D71C0F26D
:104C5000000104222520C4F8943014F01FFE012026
:104C600010BD48F28C34C2F2010441F6C131C0F2E9
:104C700000010422C4F8803014F010FE012010BDA1
:104C800048F28C34C2F2010442F6DD11C0F2000198
:104C900004223520C4F8D43014F000FE012010BDE9
:104CA00048F28C34C2F2010441F20111C0F2000159
:104CB0000422236014F0F2FD012010BD48F28C3470
:104CC000C2F2010443F29501C0F200010422E36341
:104CD00014F0E4FD012010BD48F28C34C2F201044E
:104CE00042F63951C0F200010422A36214F0D6FD4D
:104CF000012010BD48F28C34C2F2010443F2495144
:104D0000C0F2000104221620A36514F0C7FD0120A3
:104D100010BD48F28C34C2F2010443F2A161C0F22A
:104D200000010422C4F8E03014F0B8FD012010BDE9
:104D300048F28C34C2F2010441F20531C0F20001A4
:104D400004220320E36014F0A9FD012010BD00201F
:104D500010BD48F28C34C2F2010443F24D71C0F22E
:104D6000000104223920C4F8E43014F097FD01203A
:104D700010BD48F28C34C2F2010442F22111C0F29B
:104D800000010422C4F8A03014F088FD012010BDF9
:104D900048F28C34C2F2010441F66D41C0F20001C8
:104DA00004222120C4F8843014F078FD012010BDC5
:104DB00048F28C34C2F2010441F2B971C0F2000130
:104DC00004221A20A36614F069FD012010BD48F2E8
:104DD0008C34C2F2010442F28161C0F2000104226B
:104DE000C4F8C03014F05AFD012010BD48F28C34D4
:104DF000C2F2010442F6E971C0F200010422A36389
:104E000014F04CFD012010BD48F28C34C2F20104B4
:104E100041F20951C0F200010422A36114F03EFDE9
:104E2000012010BD48F28C34C2F2010443F29D41CE
:104E3000C0F200010422636514F030FD012010BDB2
:104E400048F28C34C2F2010441F6BD11C0F20001F7
:104E50000422636714F022FD012010BD48F28C3457
:104E6000C2F2010441F67161C0F200010422C4F8EB
:104E7000903014F013FD012010BD48F28C34C2F2C2
:104E8000010442F63111C0F200010422C4F8D0300E
:104E900014F004FD012010BDF8B5044616460D4679
:104EA0000846022114F03EFF3046022114F03AFF7A
:104EB00044F2B443C0F20203012253F835002272D7
:104EC00000F50071216053F8361062724FF462539E
:104ED00001F5007762F31F4300226760E260013B47
:104EE000FDD190F8003291F8002203F00103D207BF
:104EF00044BF43F00203DBB21D2DA37200F00F8408
:104F000022D92C2D00F070813FD8242D00F016847A
:104F100040F2A880282D00F0968300F2D680262D3E
:104F200000F00D8240F2F28248F28C33C2F20103AB
:104F300042F27501C0F2000104222720C3F89C4010
:104F400014F0ACFC012326E10E2D00F0BB833AD80F
:104F5000062D00F0C6836CD90A2D00F0258300F2DF
:104F60000881082D00F08F8140F2928248F28C3344
:104F7000C2F2010342F68D41C0F200010422092071
:104F80005C6214F08BFC012305E1342D00F0E68314
:104F900036D8302D00F0868300F2D7802E2D00F019
:104FA000628140F21A8248F28C33C2F2010342F26B
:104FB000D551C0F2000104222F20C3F8BC4014F0E8
:104FC0006DFC0123E7E0152D00F09A8364D9192DBB
:104FD00000F0138200F2A680172D00F0A18140F2AC
:104FE000F28248F28C33C2F2010341F26161C0F2F5
:104FF0000001042218201C6614F050FC0123CAE0B2
:10500000382D00F0EF8275D8362D00F04B8140F23C
:105010009D8248F28C33C2F2010342F63531C0F270
:10502000000104223720C3F8DC4014F037FC0123D0
:10503000B1E0022D00F01D8240F29181042D00F0BC
:10504000608140F2DF8248F28C33C2F2010341F208
:105050005D41C0F20001042205205C6114F01EFCD9
:10506000012398E0202D00F0618240F2A281222DE0
:1050700000F0378140F2F78248F28C33C2F201032C
:1050800041F6C551C0F2000104222320C3F88C4030
:1050900014F004FC01237EE0112D00F0CC8140F2DD
:1050A0007381132D00F00E8140F2D48148F28C33CD
:1050B000C2F2010343F2F131C0F2000104221420D4
:1050C0001C6514F0EBFB012365E02A2D00F0BB808A
:1050D00040F2FD8148F28C33C2F2010342F22531E5
:1050E000C0F2000104222B20C3F8AC4014F0D6FB20
:1050F000012350E03A2D00F09680C0F094823B2DC1
:1051000040F08F8248F28C33C2F2010343F6A501CE
:105110002846C0F200010422C3F8EC4014F0BEFBA4
:10512000012338E01B2D6FD040F2AD8248F28C3362
:10513000C2F2010341F61111C0F2000104221C2049
:105140001C6714F0ABFB012325E0322D2DD040F27B
:10515000AE8148F28C33C2F2010342F68501C0F2FF
:10516000000104223320C3F8CC4014F097FB012344
:1051700011E00C2D29D040F2BA8148F28C33C2F2F2
:10518000010342F63D71C0F2000104220D205C6370
:1051900014F084FB0123237430462146FFF762FAA2
:1051A000237C184420742046F8BD48F28C33C2F2A8
:1051B000010342F2D9712846C0F200010422C3F86B
:1051C000C84014F06BFB0123E5E748F28C33C2F2D0
:1051D000010342F691612846C0F2000104221C63DB
:1051E00014F05CFB0123D6E748F28C33C2F20103D2
:1051F00042F2D1312846C0F200010422C3F8B04087
:1052000014F04CFB0123C6E748F28C33C2F20103D1
:1052100041F665012846C0F200010422DC6614F064
:105220003DFB0123B7E748F28C33C2F2010343F29E
:10523000F9712846C0F200010422C3F8E84014F0D6
:105240002DFB0123A7E748F28C33C2F2010342F29F
:1052500079212846C0F200010422C3F8A84014F0C6
:105260001DFB012397E748F28C33C2F2010342F29F
:1052700029512846C0F200010422C3F8B84014F0B6
:105280000DFB012387E748F28C33C2F2010342F69B
:10529000E1312846C0F2000104221C6214F0FEFA3B
:1052A000012378E748F28C33C2F2010342F68921E8
:1052B0002846C0F200010422C3F8D84014F0EEFAE8
:1052C000012368E748F28C33C2F2010343F245310F
:1052D0002846C0F200010422DC6414F0DFFA012346
:1052E00059E748F28C33C2F2010341F619512846BE
:1052F000C0F200010422C3F8884014F0CFFA012361
:1053000049E748F28C33C2F2010341F2B131C0F2F5
:1053100000012A4628461C6114F0C0FA01233AE72E
:1053200048F28C33C2F2010343F2F5512846C0F231
:1053300000010422DC6514F0B1FA01232BE748F2E6
:105340008C33C2F2010341F6C9712846C0F2000154
:105350000422C3F8984014F0A1FA01231BE7002DA2
:1053600000F00481012D40F05C8148F28C33C2F2E0
:10537000010341F2AD11C0F20001042201205C6082
:1053800014F08CFA012306E70F2D00F0FE80102D9B
:1053900040F0478148F28C33C2F2010343F24111DD
:1053A000C0F20001042210201C6414F077FA0123DB
:1053B000F1E61E2D30D01F2D40F0338148F28C33A2
:1053C000C2F2010341F61531C0F2000104221F2090
:1053D000DC6714F063FA0123DDE648F28C33C2F295
:1053E000010342F27D41C0F2000104222D20C3F8E6
:1053F000B44014F053FA0123CDE648F28C33C2F2E4
:10540000010341F20D712846C0F2000104225C66DE
:1054100014F044FA0123BEE648F28C33C2F20103D1
:1054200041F669212846C0F2000104229C6714F06D
:1054300035FA0123AFE648F28C33C2F2010343F29E
:10544000ED112846C0F2000104225C6414F026FA33
:105450000123A0E648F28C33C2F2010343F2992102
:10546000C0F20001042212209C6414F017FA0123F8
:1054700091E648F28C33C2F2010341F259212846E9
:10548000C0F2000104229C6014F008FA012382E6B5
:1054900048F28C33C2F2010341F2B551C0F200016F
:1054A00004220720DC6114F0F9F9012373E648F2C5
:1054B0008C33C2F2010342F22D71C0F200010422CA
:1054C0003120C3F8C44014F0E9F9012363E648F23F
:1054D0008C33C2F2010342F2CD11C0F2000104226A
:1054E0002920C3F8A44014F0D9F9012353E648F267
:1054F0008C33C2F2010342F6E551C0F200010422EE
:105500000B20DC6214F0CAF9012344E648F28C3324
:10551000C2F2010341F61D71C0F2000104222520F0
:10552000C3F8944014F0BAF9012334E648F28C33FE
:10553000C2F2010341F6C1312846C0F20001042243
:10554000C3F8804014F0AAF9012324E648F28C3312
:10555000C2F2010342F6DD11C0F20001042235203F
:10556000C3F8D44014F09AF9012314E648F28C33BE
:10557000C2F2010341F201112846C0F200010422E7
:105580001C6014F08BF9012305E648F28C33C2F25B
:10559000010343F295012846C0F200010422DC63B6
:1055A00014F07CF90123F6E548F28C33C2F20103D2
:1055B00042F639512846C0F2000104229C6214F0E0
:1055C0006DF90123E7E548F28C33C2F2010343F29F
:1055D0004951C0F20001042216209C6514F05EF9C6
:1055E0000123D8E548F28C33C2F2010343F2A161F2
:1055F0002846C0F200010422C3F8E04014F04EF93E
:105600000123C8E548F28C33C2F2010341F20531AF
:10561000C0F2000104220320DC6014F03FF90123F2
:10562000B9E50023B7E548F28C33C2F2010343F237
:105630004D71C0F2000104223920C3F8E44014F097
:105640002DF90123A7E548F28C33C2F2010342F29F
:1056500021112846C0F200010422C3F8A04014F032
:105660001DF9012397E548F28C33C2F2010341F69C
:105670006D41C0F2000104222120C3F8844014F0DF
:105680000DF9012387E548F28C33C2F2010341F2A0
:10569000B971C0F2000104221A209C6614F0FEF8D1
:1056A000012378E548F28C33C2F2010342F28161B2
:1056B0002846C0F200010422C3F8C04014F0EEF8FE
:1056C000012368E548F28C33C2F2010342F6E97126
:1056D0002846C0F2000104229C6314F0DFF8012385
:1056E00059E548F28C33C2F2010341F209512846D0
:1056F000C0F2000104229C6114F0D0F801234AE5B5
:1057000048F28C33C2F2010343F29D412846C0F2B5
:10571000000104225C6514F0C1F801233BE548F266
:105720008C33C2F2010341F6BD112846C0F20001DC
:1057300004225C6714F0B2F801232CE548F28C33A4
:10574000C2F2010341F671612846C0F20001042251
:10575000C3F8904014F0A2F801231CE548F28C3302
:10576000C2F2010342F631112846C0F200010422C0
:10577000C3F8D04014F092F801230CE5F0B50746C9
:1057800043F23420A9B00E46C0F202000B2116F0FD
:10579000DDF94EF200203146C2F2000000230A2259
:1057A00017F0F8F843F24020C0F20200012116F091
:1057B000CDF9B6B100252C4643F20C600121C0F2B0
:1057C000020016F0C3F901344EF20020795DE4B214
:1057D000C2F2000000230A2217F0DCF8A642254698
:1057E000EAD84DF688644EF20020C2F20004C2F2FC
:1057F000000017F0BDF8237CBBB3BD7805F00F05A2
:105800000135AB4231D043F26C101E21C0F20200D0
:1058100016F09CF94EF2002000230A222946C2F21B
:10582000000017F0B7F843F28C100E21C0F202000E
:1058300016F08CF94EF2002000230A22217CC2F2DD
:10584000000017F0A7F843F29C100121C0F20200FB
:1058500016F07CF94EF20020C2F2000017F088F832
:1058600043F24420C0F2020006E07B78432B0ED0C6
:1058700043F26020C0F202001B2116F067F94EF2DD
:105880000020C2F2000017F073F829B0F0BD43F217
:105890007C200C21C0F2020016F058F9B9784EF2C3
:1058A0000020C1F30211C2F2000017F003F843F226
:1058B00040200121C0F2020016F048F94EF200200B
:1058C000C2F2000017F054F8072E32D0A32E0ED0EB
:1058D00043F2E8302021C0F2020016F037F94EF210
:1058E0000020C2F2000017F043F829B0F0BD43F2E7
:1058F0001C301321C0F2020097F8A14016F026F9DF
:105900004EF20020C2F2000017F032F897F8A230F1
:10591000F72B00F0048143F230301D21C0F2020069
:1059200016F014F94EF20020C2F2000017F020F831
:10593000ABE7FB78C3F38403002B6ED1BB79F72B65
:1059400040F005813A797B7940F66454C2F2010453
:1059500002F07F0203F07F0320683A717B710AF046
:10596000B5F9FA783B792068797902F0030203EB04
:10597000C213034483F830110AF09CF8FC783B7999
:1059800003EBC41404F0FF0443F2EC20C0F2020065
:10599000052116F0DBF8FB7813F07C0F06D143F2FB
:1059A000F420C0F20200092116F0D0F843F20030D2
:1059B0000B21C0F2020016F0C9F84EF200200023BD
:1059C0000A223979C2F2000016F0E4FF43F21830DF
:1059D0000321C0F2020016F0B9F84EF200207979E6
:1059E00000230A22C2F2000016F0D4FF43F20C306A
:1059F0000F21C0F2020016F0A9F84EF20020214655
:105A000000230A22C2F2000016F0C4FF4EF200206A
:105A1000C2F2000016F0ACFF37E7022B40F0A58081
:105A2000BB79F72B40F0938040F66453C2F2010338
:105A300039791B687A794AF6AB2001F07F01C3F609
:105A4000AA5007EE100A581802F07F0239717A71D5
:105A500080F88C2193F8CE4193F8CB5193F8D00184
:105A600093F8CC61C3F8885093F8CD5193F8D221C4
:105A700093F8D411C3F88C6083F89D5004F00106AC
:105A8000C4F34005C4F3800493F8CFE183F89E602B
:105A900083F89F5000F0010683F8A040C0F3400552
:105AA00093F8D14183F8A1E0C0F3800083F8A260AD
:105AB00002F0010E83F8A35083F8A40093F8D351A9
:105AC00083F8A540C1F3400001F00104C2F3400691
:105AD000C2F3800283F8A82083F8AA4083F8A6E0E6
:105AE00083F8A76083F8A95083F8AB0093F8D52119
:105AF000520607EE902AF8EEE77AC1F3800167EECE
:105B0000877A83F8AC10FDEEE77A03F18400C3EDE9
:105B1000267AFEF7DFFC3C795C34E4B234E7FB78AC
:105B200013F07F0362D139797A7942EAC1129B2A54
:105B300020D043F27430C0F20200362116F006F88D
:105B40004EF20020C2F2000016F012FF9DE643F272
:105B5000C4202621C0F2020015F0F8FF4EF200200A
:105B6000C2F2000016F004FF8FE643F28C20C0F270
:105B70000200E2E71A4607F1A0007B1D13F8011F9F
:105B80009842A2EB0102F9D165B202F07F04AC4267
:105B90003AD043F2AC30C0F20200FAF7FDFE4EF20A
:105BA0000020294600231022C2F2000016F0F2FE67
:105BB00043F2D0300321C0F2020015F0C7FF4EF2CD
:105BC0000020214600231022C2F2000016F0E2FE5F
:105BD00043F240200121C0F2020015F0B7FF4EF25F
:105BE0000020C2F2000016F0C3FE4EE643F2503031
:105BF0002121C0F2020015F0A9FF4EF20020C2F2EE
:105C0000000016F0B5FE40E6B91D01A89B2213F076
:105C100049FA40F650700DF195010A22C2F20100D6
:105C20001CF03CFE43F2D430C0F20200FAF7B4FE9E
:105C300040F65070C2F20100FAF7AEFE43F2DC30DB
:105C4000C0F20200FAF7A8FE40F66453C2F2010364
:105C500001A918680AF080F917E600BF38B50446B4
:105C60000D46FFF78BFD43F20C401021C0F20200FD
:105C700015F06CFF29462046002215F031F942F656
:105C80000070C0F202000F2115F060FF4EF20020FC
:105C9000C2F20000BDE8384016F06ABE70B540F6AA
:105CA00074750E460446C2F20105FFF767FD43F224
:105CB00020401021C0F2020015F048FFA86C0368D4
:105CC000F021DB6C984746B12644A86C14F8011B00
:105CD00003681B689847A642F7D1A86C0368F721B0
:105CE000DB6C984742F6A870C0F202000F2115F055
:105CF0002DFF4EF20020C2F20000BDE8704016F009
:105D000037BE00BFFFFFFFFF38B543F2344010EE4F
:105D1000105A4DF688642DED048BC2F20004142154
:105D2000C0F20200B0EE608AC4ED030A84ED020AFC
:105D300015F00CFF28461BF01DFD41EC100B4EF238
:105D400000200A21C2F2000016F064FE43F24C402B
:105D50000121C0F2020015F0F9FE40F6DB73C4F237
:105D60004903A06809EE103A1BF004FD41EC100B4A
:105D70004EF200200A21C2F2000016F04BFE43F260
:105D800050400621C0F2020015F0E0FE43F24C4004
:105D90000121C0F2020015F0D9FEE0681BF0EAFC18
:105DA00041EC100B4EF200200A21C2F2000016F066
:105DB00031FE43F258400221C0F2020015F0C6FE47
:105DC000E36807EE903A27EE890AF6EE008A20EEA5
:105DD000280A18F00DFDA36807EE903A60EE277AC6
:105DE00017EE900A1BF0C6FC9FED511B41EC100B07
:105DF00018F0FEFD4EF200200321C2F2000016F062
:105E000009FE43F25C400121C0F2020015F09EFE43
:105E1000E36807EE903A27EE890A20EE280A18F088
:105E200097FCA36807EE903A60EE277A17EE900A87
:105E30001BF0A0FC9FED3E1B41EC100B18F0D8FDB1
:105E40004EF200200321C2F2000016F0E3FD4EF2F4
:105E50000020C2F2000016F08BFD40F6645328EEDD
:105E6000098AC2F2010328EE288A1B68B0EE480AAC
:105E7000C3F82C5118F0BCFC4FF47E43C4F2FF630E
:105E800007EE903AB4EEE70AF1EE10FA0EDC4FF4AA
:105E90007E43CCF2FF6307EE903AB4EEE70AF1EEF0
:105EA00010FA30D50023C8F2010302E00023C7F640
:105EB000FF7340F60852C2F20102B0EE480A936145
:105EC00018F046FC4FF47E43C4F2FF6307EE903AAD
:105ED000B4EEE70AF1EE10FA23DC4FF47E43CCF285
:105EE000FF6307EE903AB4EEE70AF1EE10FA11D52F
:105EF0000023C8F20103BDEC048B40F63842C2F225
:105F00000102936138BDF0EE407AFEEEC87A17EEDA
:105F1000903ACEE7F0EE407AFEEEC87A17EE903A6D
:105F2000E9E70023C7F6FF73E5E700BFAFF30080A2
:105F30000000002085EBB13F2DE9F041054643F21A
:105F4000604082B00C46C0F20200032115F0FEFD55
:105F50004EF2002000230A222946C2F2000016F069
:105F600019FD43F264400121C0F2020015F0EEFD7C
:105F70004EF20020214600230A22C2F2000016F051
:105F800009FD4EF20020C2F2000016F0F1FC672D70
:105F900000F093824DD9782D00F0A08000F2898026
:105FA000692D00F0C180C0F0DE836A2D00F0A0836F
:105FB0006B2D40F0FC81002301EE903A04EB440489
:105FC0000023C4F2482304EB041401EE103AC4F396
:105FD000C71307EE903A40F67072C2F20102B8EEB3
:105FE000670AF0EE610AB7EE002A137004F0DAF8DF
:105FF0004FF47E43C4F2FF6307EE903AB4EEE70A33
:10600000F1EE10FA00F3D8834FF47E43CCF2FF6335
:1060100007EE903AB4EEE70AF1EE10FA40F126846A
:106020000023C8F2010340F69042C2F20102D3619C
:1060300067E2042D00F06A8240F2C5800A2D61D02B
:1060400040F2C481202D00F0DE81402D40F0AF8170
:1060500040F66456C2F201063F2C94BF0021012194
:10606000306809F033FD306809F038FD0546002836
:1060700040F09D813068374609F092FEEBB203EBA9
:10608000430498424FEA840440F291813068031936
:106090000135DA78002AEFD093F80280B8F1000FCA
:1060A000EAD198680BF08CF93868044484F80380CE
:1060B000E2E77B2D1CD040F27D817E2D00F09D819A
:1060C0007F2D40F0748140F66453C2F20103002139
:1060D000186802B0BDE8F04109F0F0BC40F6645326
:1060E000C2F20103186802B0BDE8F04109F0FABC41
:1060F00040F66453C2F20103186802B0BDE8F041F3
:1061000009F0E4BD4DF68863C2F2000300EE904A48
:106110009A68FBEEEC0A00EE102AC3ED030A02B007
:10612000BDE8F041FFF7F0BD002301EE903A0023F7
:10613000C4F2964302EE103A04EB44040023C4F286
:10614000482304EB041401EE103AC4F3C71307EE1E
:10615000903A40F24012C2F20102B8EE670AF0EE45
:10616000610A137004F01EF8B5EEC00AF1EE10FAE1
:1061700000F1268347F67903C4F2302307EE103A84
:10618000F6EE007AE0EE077A4FF4FC53C0F201031A
:10619000FCEEE77A17EE902A9A4240F276831A468E
:1061A0004FF4107040F2F423C2F20103197ECC07C1
:1061B00000F10983DC8B1A62A04241F0010188BF23
:1061C000D88319769DE1012D00F02B81C0F021814B
:1061D000022D40F0EC8040F66453C2F201034DF210
:1061E0000A721B68C3F6234206EE102A93F89D201C
:1061F00093F89F0083F8944007EE902A93F8962036
:10620000B8EEE77A06EE902A67EE067AF8EEE66ACE
:10621000002167EEA67A83F89210FCEEE77A83F805
:106220009110CDED017A9DF8042083F8901008B10B
:1062300083F8902093F89E1009B183F8912093F889
:10624000A01009B183F8922093F8A52093F8A70035
:1062500007EE902A4DF20A72B8EEE77A07EE904AFE
:10626000C3F6234206EE102AF8EEE76A67EE067AD6
:1062700067EEA67AFCEEE77ACDED017A9DF8042070
:1062800030B193F89000904238BF104683F89000E8
:1062900093F8A60030B193F89100904238BF1046B1
:1062A00083F8910093F8A84034B193F892008242A9
:1062B00038BF024683F8922093F8A12093F8A300F8
:1062C00007EE902A4DF20A72C3F6234206EE102A18
:1062D00093F89520B8EEE77A06EE902A67EE067AF4
:1062E000F8EEE66A67EEA67AFCEEE77ACDED017A83
:1062F0009DF8042030B193F89000904238BF1046CA
:1063000083F8900093F8A20030B193F89100904286
:1063100038BF104683F8910093F8A40030B193F889
:106320009250AA4238BF2A4683F8922093F8A920B7
:1063300093F8AB5007EE902A4DF20A72C3F623424F
:1063400006EE102A93F89320B8EEE77A06EE902A2C
:1063500067EE067AF8EEE66A67EEA67AFCEEE77A72
:10636000CDED017A9DF8042035B193F89050954217
:1063700038BF154683F8905093F8AA5035B193F87A
:106380009150954238BF154683F8915093F8AC5020
:1063900035B193F89260B24238BF324683F892200A
:1063A00029B920B91CB915B97F2283F8922002B00F
:1063B000BDE8F081792DFAD140F66453C2F20103B1
:1063C000186802B0BDE8F04109F0A0BB072DEED17E
:1063D00007EE904A0023C4F2FE23B8EE677A07EE78
:1063E000903A87EE270A4DF68863C2F20003DA6816
:1063F00000EE902A83ED020A91E640F66453C2F261
:106400000103012164E64DF68863C2F200031C71AA
:10641000CDE7632CCBD84DF68863C2F200031C7124
:106420006FE040F66453C2F201034DF20A721B683A
:10643000C3F6234206EE102A93F89D2093F89F009E
:1064400083F8964007EE902AB8EEE77A07EE904A76
:10645000F8EEE76A67EE067A002167EEA67A83F81F
:106460009210FCEEE77A83F89110CDED017A9DF859
:10647000042083F8901008B183F8902093F89E10C0
:1064800009B183F8912093F8A01009B183F8922004
:1064900093F8A52093F8A70007EE902A4DF20A7210
:1064A000C3F6234206EE102A93F8942006EE902AB3
:1064B000B8EEE77AF8EEE66AD8E624B204EB840395
:1064C00003EB830304EB8304C4F3C71407EE904A81
:1064D0000023C4F2C823F8EE676A07EE903A86EE0E
:1064E000A77A40F66452C2F2010240F6ED531268F8
:1064F000C2F201031C70F7EE007A77EEC77AC2EDA4
:106500004A7A02B0BDE8F04106F0ECB940F66453B7
:10651000C2F201034DF20A721B68C3F6234206EE73
:10652000102A93F89D2093F89F0083F8954007EE7A
:10653000902A93F89620B8EEE77A06EE902A67EE56
:10654000067AF8EEE66A002167EEA67A83F89210E2
:10655000FCEEE77A83F89110CDED017A9DF80420E6
:1065600083F8901008B183F8902093F89E1009B139
:1065700083F8912093F8A01009B183F8922093F842
:10658000A52093F8A70007EE902A4DF20A72C3F6F1
:10659000234206EE102A93F89420B8EEE77A06EE2E
:1065A000902A67EE067AF8EEE66A67EEA67AFCEEC7
:1065B000E77ACDED017A9DF8042030B193F8900090
:1065C000904238BF104683F8900093F8A60030B18F
:1065D00093F89100904238BF104683F8910093F8E9
:1065E000A85035B193F89200824238BF024683F832
:1065F000922093F8A12093F8A30007EE902A4DF281
:106600000A72C3F6234206EE102AB8EEE77A07EEC6
:10661000904AF8EEE76A67EE067A67EEA67AFCEE35
:10662000E77ACDED017A9DF8042030B193F890001F
:10663000904238BF104683F8900093F8A20030B122
:1066400093F89100904238BF104683F8910093F878
:10665000A40030B193F89240A24238BF224683F89A
:10666000922093F8A92093F8AB4007EE902A4DF2C0
:106670000A72C3F6234206EE102A93F89320B8EE6E
:10668000E77A06EE902A67EE067AF8EEE66A67EE9B
:10669000A67AFCEEE77ACDED017A9DF8042034B1BC
:1066A00093F89040944238BF144683F8904093F892
:1066B000AA4034B193F89140944238BF144683F80D
:1066C000914093F8AC4034B193F89260B24238BF35
:1066D000324683F8922000297FF469AE00287FF4C7
:1066E00066AE002D7FF463AE002C3FF45DAE5EE637
:1066F00004EBC4040022C4F3471401EE902A07EE11
:10670000904A40F6EC530022C2F20103C4F20C227C
:10671000B8EE670A01EE102AF0EE610AB7EE002A21
:106720001C7003F03FFD4FF47E43C4F2FF6307EE9D
:10673000903AB4EEE70AF1EE10FA39DC4FF47E43FA
:10674000CCF2FF6307EE903AB4EEE70AF1EE10FAEE
:1067500040F194800023C8F2010340F65842C2F28F
:106760000102D361CDE624B204EB840303EB83037F
:1067700004EB8304C4F3C71407EE904A0023C4F269
:10678000C823F8EE676A07EE903A86EEA77A40F6DD
:106790006452C2F201024FF610431268C2F20003C3
:1067A0001C70F7EE007A77EEC77AC2ED497AA8E658
:1067B0000023C7F6FF73D0E70023C7F6FF7332E468
:1067C00001200022EEE41C6AA24205D9D98B1A628C
:1067D000884288BFD88394E602F17F00C009013067
:1067E00000281A62024638BF0022880706D5586A78
:1067F0007F30C0090130824238BF02464F0706D5BC
:10680000986A7F30C0090130824238BF02460E07C5
:1068100006D5D86A7F30C0090130824238BF0246AF
:10682000CD0606D5186B7F30C0090130824238BFD3
:1068300002468C0606D5586B7F30C0090130824273
:1068400038BF0246480606D5986B7F30C009013034
:10685000824238BF0246C90906D0D96B7F31C909C7
:1068600001318A4238BF0A46DA834AE6F0EE407ABE
:10687000FEEEC87A17EE903AFFF7D5BBF0EE407AFD
:10688000FEEEC87A17EE903A67E702F17F00C00982
:10689000013087E4F8B54DF68865C2F2000504467C
:1068A0002B7C0E4617467BB398422DD043F26C10DA
:1068B0001E21C0F2020015F049F94EF2002000231B
:1068C0000A222146C2F2000016F064F843F28C104E
:1068D0000E21C0F2020015F039F94EF20020297C99
:1068E00000230A22C2F2000016F054F843F29C1072
:1068F0000121C0F2020015F029F94EF20020C2F287
:10690000000016F035F803E039463046FFF714FB77
:1069100043F268400D21C0F20200013C15F016F967
:10692000E1B20F2915D840F67475C2F2010541F0A5
:10693000B001A86C03681B689847A86C036806F050
:106940007F011B689847A86C036807F07F011B68EC
:10695000984742F6A870C0F202000F2115F0F6F831
:106960004EF20020C2F20000BDE8F84016F000B878
:10697000F8B54DF68867C2F2000705463B7C0E4627
:1069800014467BB398422DD043F26C101E21C0F206
:10699000020015F0DBF84EF2002000230A222946FF
:1069A000C2F2000015F0F6FF43F28C100E21C0F287
:1069B000020015F0CBF84EF20020397C00230A22A9
:1069C000C2F2000015F0E6FF43F29C100121C0F274
:1069D000020015F0BBF84EF20020C2F2000015F0E4
:1069E000C7FF03E021463046FFF7A6FA43F278409E
:1069F0000D21C0F2020015F0A9F8230603F0FE43B2
:106A0000681E43F43043360406F4FE0643F00B03DD
:106A10000002334300F47060184314F00DFA42F69C
:106A20000070C0F202000F2115F090F84EF2002025
:106A3000C2F20000BDE8F84015F09ABF48F290435A
:106A4000C2F2010382B01B68019340F66C72C2F27D
:106A5000010240F2A013C2F2010301991160012268
:106A60001A7002B0704700BF42F6AC632DE9F04FD8
:106A7000C0F202031C460FCCB1B020AD0FC50FCC45
:106A80000FC50FCC0FC594E80F0010944DF6886722
:106A900040F2A014C2F20007C2F201044FF0000E4F
:106AA00084F800E01F9585E80F00BD7A0395FD7A14
:106AB0003B7904953D7B05957D7B06956FEA03093F
:106AC000BD7B079509F00F0930AD05EB8909BA794F
:106AD00097F80580787A02901D1159F8403C11957D
:106AE0001146FA79139183F070431446DB433A7AE6
:106AF000019283EA05020DF1C00E02F00F020EEBC7
:106B000082024FEA281E52F8402C82EA1313DB431C
:106B100083EA0802754602F00F020DF1C00E0EEB7B
:106B200082020DF1C00E52F8402C129582EA131326
:106B300083EA050202F00F020EEB82020DF1C00E95
:106B400052F8402C82EA1313DB4383EA010202F07D
:106B50000F020EEB8202081152F8402C01990646F2
:106B600082EA131383EA06020DF1C00E02F00F024F
:106B70000EEB8202081114960990029852F8402CEC
:106B8000159482EA1313DB4383EA04020DF1C00E6D
:106B900002F00F020EEB8202251152F8402C039CEA
:106BA000169582EA131383EA05020DF1C00E02F076
:106BB0000F020EEB82020DF1C00E52F8402C82EA59
:106BC00013136FEA030C8CEA010202F00F0205991D
:106BD0000EEB82020B1152F8402C0C93099B82EAB7
:106BE0001C1C8CEA03020DF1C00E02F00F020EEB2A
:106BF0008202069B52F8402C1B110D9382EA1C1353
:106C0000DB4383EA0002061102F00F0207980A969E
:106C10000DF1C00E0EEB820E02110E925EF8402CAA
:106C200082EA13130A9A5A4002F00F020DF1C00EC5
:106C30000EEB820E109AA2F1300C5EF8402C82EA24
:106C40001313DB4383EA04020DF1C00E02F00F02BE
:106C50000EEB820226110B9652F8402C0B9C049EE0
:106C600082EA131383EA04020DF1C00A02F00F0254
:106C70000AEB8202351152F8402C179582EA131361
:106C8000DB4383EA060202F00F020AEB82020DF1F7
:106C9000C00A52F8402C0C9E82EA131383EA0502C4
:106CA00002F00F020AEB82020DF1C00A52F8402CEA
:106CB00082EA1313DB4383EA010202F00F020AEBBC
:106CC00082020DF1C00A52F8402C82EA131383EAC3
:106CD000060202F00F020AEB82020DF1C00A52F81E
:106CE000402C069E0E9D97F813B082EA1313DB43E7
:106CF00083EA060202F00F020AEB82020D9E52F8AE
:106D0000402C82EA131383EA06020DF1C00A02F056
:106D10000F020AEB82020DF1C00A52F8402C82EAFF
:106D20001313DB4383EA000202F00F020AEB820234
:106D30000DF1C00A52F8402C82EA131383EA0502CF
:106D400002F00F020AEB820297F80FA052F8402CD3
:106D5000564697F810A01896514697F811A01A9128
:106D600082EA13135046DB4397F812A083EA060227
:106D7000554602F00F020DF1C00A0AEB82023611ED
:106D800052F8402C199682EA131383EA06020DF199
:106D9000C00A02F00F020AEB82020DF1C00A52F89B
:106DA000402C1D9582EA1313DB4383EA010202F0B3
:106DB0000F020AEB82020E1152F8402C0F9682EA63
:106DC00013130F9A5A400DF1C00A02F00F020AEB9A
:106DD0008202064652F8402C1B9682EA1313DB43CC
:106DE00083EA06020DF1C00A02F00F020AEB8202EA
:106DF000011152F8402C1C9182EA131383EA01021C
:106E00004FEA2B1ACDF820A002F00F020DF1C00AB4
:106E10000AEB82020DF1C00A52F8402C82EA1313E9
:106E2000DB4383EA050202F00F020AEB820228111B
:106E300052F8402C1E9082EA131383EA00020DF1EF
:106E4000C00A02F00F020AEB820230AE52F8402C68
:106E500082EA1313DB438BEA030202F00F020AEB10
:106E600082020DF1800E52F8402C82EA131A089B20
:106E700055468AEA030ABCE80F000AF00F0A06EB3F
:106E80008A0A3C465AF840ACAEE80F00BCE80F0056
:106E9000AEE80F00BCE80F00AEE80F0059F8402C38
:106EA0008AEA151A82F07042119DD24382EA0503E4
:106EB00003F00F0306EB83030DF1C00E53F8403CC3
:106EC00083EA1212D24382EA080303F00F0306EBAF
:106ED00083036FEA0A0A53F8403CC7F800A083EA2C
:106EE0001212129B534003F00F030EEB83030DF1BC
:106EF000C00E53F8403C1398019983EA1212D24312
:106F000082EA000303F00F030EEB8303149853F897
:106F1000403C83EA121282EA00030DF1C00E03F036
:106F20000F030EEB8303159853F8403C83EA1212CB
:106F3000D24382EA00030DF1C00E03F00F030EEB03
:106F40008303169853F8403C83EA121282EA000346
:106F50000DF1C00E03F00F030EEB83030DF1C00E15
:106F600053F8403C099883EA1212D24382EA0103A3
:106F700003F00F030EEB83030DF1C00E53F8403CFA
:106F8000059983EA121282EA000303F00F030EEB65
:106F90008303029853F8403C83EA1212D24382EAF8
:106FA00000030DF1C00E03F00F030EEB83030A98EC
:106FB00053F8403C83EA121282EA00030DF1C00E3E
:106FC00003F00F030EEB83030DF1C00E53F8403CAA
:106FD0000B9883EA1212039BD243534003F00F0332
:106FE0000EEB83030DF1C00E53F8403C83EA1212FE
:106FF00082EA000303F00F030EEB83030DF1C00ED2
:1070000053F8403C179883EA1212049BD243534032
:1070100003F00F030EEB83030DF1C00E53F8403C59
:1070200083EA121282EA000303F00F030EEB8303DC
:107030000DF1C00E53F8403C0C9883EA1212D24373
:1070400082EA010303F00F030EEB83030DF1C00E80
:1070500053F8403C83EA121282EA000303F00F0364
:107060000EEB83030DF1C00E53F8403C0D9883EAFC
:107070001212069BD243534003F00F030EEB83031F
:107080000DF1C00E53F8403C83EA121282EA00036D
:1070900003F00F030EEB83030DF1C00E53F8403CD9
:1070A00007981A9983EA1212D24382EA000303F086
:1070B0000F030EEB83030E9853F8403C83EA121241
:1070C00082EA00030DF1C00E03F00F030EEB830301
:1070D0000DF1C00E53F8403C199883EA1212189B28
:1070E000D243534003F00F030EEB83030DF1C00EA8
:1070F00053F8403C83EA121282EA000303F00F03C4
:107100000EEB83030DF1C00E53F8403C1E9883EA4A
:107110001212D24382EA010303F00F030EEB830342
:107120000F9953F8403C83EA121282EA01030DF1F1
:10713000C00E03F00F030EEB83030DF1C00E53F8E6
:10714000403C1C9983EA12121B9BD243534003F02C
:107150000F030EEB830307F1140553F8403C83EA59
:10716000121282EA010303F00F030EEB8303FE43C6
:1071700053F8403C83EA12121D9BD243534003F064
:107180000F030EEB830353F8403C83EA121282EAAA
:10719000000303F00F030EEB830353F8403C83EA34
:1071A0001212D2438BEA020303F00F030EEB8303A8
:1071B00053F8403C83EA1212089B534003F00F033C
:1071C0000EEB830353F8403C83EA1213DB433B701E
:1071D00014F8018BA719384612F0E8F880454146AB
:1071E000384601D012F03EF9AC42F1D143F288406A
:1071F0002721C0F2020014F0A9FC4EF20020C2F2D6
:10720000000031B0BDE8F04F15F0B2BBF0B597B05B
:1072100001AD2C4606AE601B12F0C8F804F8010B55
:10722000B442F8D142F6AC65C0F202050FCD0FC4EE
:107230000FCD0FC40FCD0FC495E80F0084E80F00E9
:107240009DF808609DF809509DF80A409DF80B20B4
:107250009DF80C309DF80D009DF80E10F7430DF1D0
:10726000580E07F00F070EEB870757F8407C87F0A2
:107270007047FF4387EA161606F00F060EEB8606E8
:1072800056F8406C86EA1716F64385EA060707F0BB
:107290000F070EEB870757F8407C87EA161787EA37
:1072A000151606F00F060EEB86069DF80F5056F8E1
:1072B000406C86EA1716F64384EA060707F00F07C4
:1072C0000EEB870757F8407C87EA161787EA1416F3
:1072D00006F00F060EEB86069DF8104056F8406C3F
:1072E00086EA1716F64382EA060707F00F070EEB49
:1072F000870757F8407C87EA161787EA121606F0C8
:107300000F060EEB86069DF8112056F8406C86EAB3
:107310001716F64383EA060707F00F070EEB8707F9
:1073200057F8407C87EA161787EA131606F00F060F
:107330000EEB86069DF8123056F8406C86EA17165A
:10734000F64380EA060707F00F070EEB870757F8AA
:10735000407C87EA161787EA101606F00F060EEB38
:10736000860643F2B04056F8406C86EA1716F6439C
:1073700081EA060707F00F070EEB8707C0F202004D
:1073800057F8407C87EA161787EA111606F00F06B1
:107390000EEB8606132156F8406C86EA1716F64364
:1073A00085EA060707F00F070EEB870757F8407CC2
:1073B00087EA161686EA151505F00F050EEB85050A
:1073C00055F8405C85EA1615ED4384EA050606F09B
:1073D0000F060EEB860656F8406C86EA151585EA10
:1073E000141404F00F040EEB840454F8404C84EAA7
:1073F0001514E44382EA040505F00F050EEB85053C
:1074000055F8405C85EA141484EA121202F00F0267
:107410000EEB820252F8402C82EA1412D24383EA25
:10742000020404F00F040EEB840454F8406C86EA66
:10743000121787EA131303F00F030EEB830353F8BD
:10744000406C9DF813309DF814509DF815409DF840
:10745000162086EA1716F64383EA060707F00F0799
:107460000EEB870757F8407C87EA161787EA131652
:1074700006F00F060EEB86069DF8173056F8406CA6
:1074800086EA1716F64385EA060707F00F070EEBA4
:10749000870757F8407C87EA161686EA151505F027
:1074A0000F050EEB850555F8405C85EA1615ED4392
:1074B00084EA050606F00F060EEB860656F8406CC9
:1074C00086EA151585EA141404F00F040EEB840403
:1074D00054F8404C84EA1514E44382EA040505F0AC
:1074E0000F050EEB850555F8405C85EA141484EA17
:1074F000121202F00F020EEB820252F8402C82EAC6
:107500001412D24383EA020404F00F040EEB840445
:1075100054F8404C84EA121484EA131303F00F0366
:107520000EEB830353F8403C83EA141414F00EFB73
:10753000019D4EF20020002310222946C2F20000D5
:1075400015F028FA43F2C4400521C0F2020014F0FD
:10755000FDFAE4434EF200202146C2F2000000236F
:10756000102215F017FAA5421DD14DF68865C2F21A
:10757000000505F114062C46601B11F017FF04F8F6
:10758000010BB442F8D143F2F040C0F202000F21E7
:1075900014F0DCFA4EF20020C2F2000017B0BDE891
:1075A000F04015F0E5B943F2CC402321C0F20200CF
:1075B00014F0CCFAFFF758FAECE700BF2DE9F843D6
:1075C00048F29A69C2F2010943F200502DED028B94
:1075D0000521C0F2020014F0B9FAB9F8003007EE44
:1075E000103A49F69A13C4F2D92308EE903AB8EE4D
:1075F000C77A49F69A13C4F2593308EE103A37EEB7
:10760000287A4EF20024C7EE087AC2F2000448F24B
:107610009467C2F2010748F29868C2F2010848F282
:107620003866C2F201064FF62045C2F2000517EE99
:10763000900A1AF09FF841EC100B0221204615F039
:10764000E9F943F208500D21C0F2020014F07EFA6D
:107650003B8807EE903AF8EEE77A77EEA87A87EE65
:10766000887A17EE100A1AF085F841EC100B022107
:10767000204615F0CFF943F218500821C0F202005D
:1076800014F064FAB8F80010204615F013F943F22C
:1076900024500C21C0F2020014F058FA3188204620
:1076A00015F008F943F234501421C0F2020014F02E
:1076B0004DFA2988204615F0FDF843F24C50092177
:1076C000C0F2020014F042FA40F60453C2F2010381
:1076D0000A2219682046002315F05CF943F258503D
:1076E0000D21C0F2020014F031FA4FF61443C2F239
:1076F00000030A2219682046002315F04BF943F2D3
:1077000068500921C0F2020014F020FA40F69C53A0
:10771000C2F201030A2219682046002315F03AF943
:1077200043F274500C21C0F2020014F00FFA8021D1
:10773000204615F0BFF843F284501021C0F2020039
:1077400014F004FA40F6C953C2F201030A22197870
:107750002046002315F01EF9204615F009F9BDEC6E
:10776000028BB9F80030B8F800203B80002332804B
:107770002B80BDE8F88300BF70B584B0002440F6CC
:10778000645502940194CDF80B40C2F2010506261F
:1077900043F298500221C0F2020014F0D7F94EF2E1
:1077A00000203146C2F2000015F084F843F2F86080
:1077B0000221C0F2020014F0C9F94EF20020C2F218
:1077C000000015F0D5F843F29C505621C0F202009B
:1077D00014F0BCF94EF20020C2F2000015F0C8F817
:1077E0002B6823444EF2002093F830110A22002324
:1077F000C2F2000015F0CEF843F20C600121C0F295
:10780000020014F0A3F92B6823444EF2002093F8F1
:1078100031110A220023C2F2000015F0BBF843F236
:107820000C600121C0F2020014F090F92B6823448F
:107830004EF2002093F832110A220023C2F2000017
:1078400015F0A8F843F20C600121C0F2020014F018
:107850007DF92B6823444EF2002093F833110A225D
:107860000023C2F2000015F095F843F20C600121EC
:10787000C0F2020014F06AF92B6823444EF2002093
:1078800093F834110A220023C2F2000015F082F8A6
:1078900043F20C600121C0F2020014F057F92B688A
:1078A00023444EF2002093F835110A220023C2F23D
:1078B000000015F06FF843F20C600121C0F20200E5
:1078C00014F044F92B6823444EF2002093F836114B
:1078D0000A220023C2F2000015F05CF843F20C60AB
:1078E0000121C0F2020014F031F92B6823444EF25A
:1078F000002093F837110A220023C2F2000015F08D
:1079000049F843F2F4500821C0F2020014F01EF9C5
:107910002B6823444EF2002093F838110A220023EA
:10792000C2F2000015F036F843F200600D21C0F2FB
:10793000020014F00BF92B6823444EF2002093F858
:1079400039110A220023C2F2000015F023F843F295
:1079500000600D21C0F2020014F0F8F82B682344F7
:107960004EF200200A2293F83A11C2F200000023DE
:1079700015F010F84EF20020C2F2000014F0F8FFEB
:1079800043F210605C21C0F2020014F0DFF84EF206
:107990000020C2F2000014F0EBFF43F270600621F9
:1079A000C0F2020014F0D2F82B6823444EF20020FB
:1079B00093F83B110A220023C2F2000014F0EAFF00
:1079C00043F204600921C0F2020014F0BFF82B68F2
:1079D00023444EF2002093F83C110A220023C2F205
:1079E000000014F0D7FF43F204600921C0F2020046
:1079F00014F0ACF82B6823444EF2002093F83D11AC
:107A00000A220023C2F2000014F0C4FF43F2F45033
:107A10000821C0F2020014F099F82B6823444EF2BA
:107A2000002093F83E110A220023C2F2000014F055
:107A3000B1FF43F208600521C0F2020014F086F89D
:107A40002B6823444EF2002093F83F110A220023B2
:107A5000C2F2000014F09EFF43F270600621C0F2F3
:107A6000020014F073F82B6823444EF2002093F8C0
:107A700040110A220023C2F2000014F08BFF43F2EF
:107A800070600621C0F2020014F060F82B682344F5
:107A90004EF2002093F841110A220023C2F20000A6
:107AA00014F078FF43F2F8500421C0F2020014F001
:107AB0004DF82B6823444EF2002093F842110A221D
:107AC0000023C2F2000014F065FF43F208600521B4
:107AD000C0F2020014F03AF82B6823444EF2002062
:107AE00093F843110A220023C2F2000014F052FF5F
:107AF00043F208600521C0F2020014F027F82B6859
:107B000023444EF2002093F844110A220023C2F2CB
:107B1000000014F03FFF4EF200201534C2F20000C6
:107B200014F026FF7E2C06F1FF367FF431AE43F2CF
:107B300078602D21C0F2020014F008F84EF2002007
:107B4000C2F2000014F014FF43F20C60C0F2020015
:107B5000012113F0FBFF2B6823444EF2002093F821
:107B600030110A220023C2F2000014F013FF43F286
:107B700074600134C0F20200022140F6645613F032
:107B8000E5FF862CC2F20106E5D14EF20020C2F2DA
:107B9000000014F0EDFE43F2A8600521C0F20200DF
:107BA00013F0D4FF33684EF2002093F8B6110A2286
:107BB0000023C2F2000014F0EDFE4EF20020C2F2EB
:107BC000000014F0D5FE43F2B0600421C0F20200C0
:107BD00013F0BCFF33684EF2002093F8B7110A226D
:107BE0000023C2F2000014F0D5FE4EF20020C2F2D3
:107BF000000014F0BDFE43F2B8600521C0F202009F
:107C000013F0A4FF33684EF2002093F8B8110A2253
:107C10000023C2F2000014F0BDFE4EF20020C2F2BA
:107C2000000014F0A5FE43F2C0600921C0F202007A
:107C300013F08CFF33684EF2002093F8B9110A223A
:107C40000023C2F2000014F0A5FE4EF20020C2F2A2
:107C5000000014F08DFE43F2CC600921C0F2020056
:107C600013F074FF33684EF2002093F8BA110A2221
:107C70000023C2F2000014F08DFE4EF20020C2F28A
:107C8000000014F075FE43F2D8600921C0F2020032
:107C900013F05CFF33684EF2002093F8BB110A2208
:107CA0000023C2F2000014F075FE4EF20020C2F272
:107CB000000014F05DFE43F2E4600921C0F202000E
:107CC00013F044FF33684EF2002093F8BC110A22EF
:107CD0000023C2F2000014F05DFE4EF20020C2F25A
:107CE000000014F045FE43F2F0600A21C0F20200E9
:107CF00013F02CFF33684EF2002093F8BD110A22D6
:107D00000023C2F2000014F045FE4EF20020C2F241
:107D1000000014F02DFE43F2FC600D21C0F20200C1
:107D200013F014FF33684EF2002093F8BE110A22BC
:107D30000023C2F2000014F02DFE4EF20020C2F229
:107D4000000014F015FE43F20C700921C0F202008D
:107D500013F0FCFE33684EF2002093F8BF110A22A4
:107D60000023C2F2000014F015FE4EF20020C2F211
:107D7000000014F0FDFD43F218700921C0F202006A
:107D800013F0E4FE33684EF2002093F8C0110A228B
:107D90000023C2F2000014F0FDFD4EF20020C2F2FA
:107DA000000014F0E5FD43F224700621C0F2020049
:107DB00013F0CCFE31680A2201F2C11101A81AF0B9
:107DC0006DFD43F24C400121C0F2020013F0BEFEF3
:107DD00001A81AF0F5FC014601A813F0B7FE43F222
:107DE00040200121C0F2020013F0B0FE4EF200204C
:107DF000C2F2000014F0BCFD9B244EF200200023D0
:107E00000A222146C2F2000014F0C4FD43F2F860D9
:107E10000221C0F2020013F099FE2B6823444EF2B7
:107E2000002093F830110A220023C2F2000014F05F
:107E3000B1FD4EF200200134C2F2000014F098FDB2
:107E4000AD2CDAD14EF20020C2F2000014F090FD09
:107E500004B070BD2DE9F0412DED028B40F65C7051
:107E600086B0C2F2010011F00BF940F65C70C2F26C
:107E7000010010F081FF40F65C70C2F2010010F0CA
:107E800073FF40F65C70C2F2010010F00BFE40F68A
:107E90005C70C2F2010010F077FF40F65C70C2F235
:107EA000010010F079FF40F65C70C2F2010010F0A2
:107EB00053FF43F22C73C0F2020393E8070000243F
:107EC0004FF020376B46029703940494CDF80B7063
:107ED0008DF8144003C340F65C701A802146224698
:107EE000C2F2010010F014FF68461AF069FC024665
:107EF00040F65C706946C2F2010014F0C5FC4EF217
:107F0000002023460A222146C2F2000014F042FD5E
:107F100043F25C400121C0F2020013F017FE4EF262
:107F2000002023460A222146C2F2000014F032FD4E
:107F300043F238700321C0F2020013F007FE6846D6
:107F40001AF03EFC0146684613F000FE43F2402062
:107F50000121C0F2020013F0F9FD43F23C764EF22B
:107F60000020C0F20206C2F2000014F001FD96E803
:107F70000300009040F65C70019722468DF80410D3
:107F8000C2F201000B21029703940494CDF80B7008
:107F90008DF8144010F0BCFE68461AF011FC024641
:107FA00040F65C706946C2F2010014F06DFC4EF2BE
:107FB000002023460A222146C2F2000014F0EAFC07
:107FC00043F25C400121C0F2020013F0BFFD4EF20B
:107FD000002023460A220B21C2F2000014F0DAFC32
:107FE00043F238700321C0F2020013F0AFFD68467F
:107FF0001AF0E6FB0146684613F0A8FD43F2402064
:108000000121C0F2020013F0A1FD4EF20020C2F2E5
:10801000000014F0ADFC43F24473C0F202030FCB36
:108020008DE80F0040F65C7021460122C2F201008B
:1080300004948DF8144010F06BFE68461AF0C0FBF3
:10804000024640F65C706946C2F2010014F01CFC66
:108050004EF2002023460A220121C2F2000014F051
:1080600099FC43F25C400121C0F2020013F06EFD66
:108070004EF200200A2223462146C2F2000014F0EC
:1080800089FC43F238700321C0F2020013F05EFD58
:1080900068461AF095FB0146684613F057FD43F217
:1080A00040200121C0F2020013F050FD4EF20020EA
:1080B000C2F2000014F05CFC0221042011F032FE38
:1080C00002211E2011F02EFEDC2011F08DFE43F265
:1080D00058703421C0F2020013F038FD4EF2002037
:1080E000C2F2000014F044FC43F290702E21C0F262
:1080F000020013F02BFD4EF20020C2F2000014F03B
:1081000037FC43F2C0702921C0F2020013F01EFDBB
:108110004EF20020C2F2000014F02AFC43F2EC7090
:108120000921C0F2020013F011FD0521304613F0C1
:108130000DFD4EF20020C2F2000014F019FC43F2D3
:10814000F8700D21C0F2020013F000FD4EF2002085
:10815000C2F2000014F00CFCFFF758F8FCF782F8AC
:108160004EF28813CEF20003012740F2002040F2C5
:108170006C15C2F201051F604FF4E171C1F6FF708A
:1081800013F05AFE28460BF07BFA28460AF0C8FD89
:10819000EA88242122F0100228460AF08DFBEA88A2
:1081A000242122F4807228460AF086FB28460AF031
:1081B00037FDF6EE000AB0EE600A28460BF05AF8DA
:1081C0004CF6CD461D2128460AF09AFEC3F64C56C1
:1081D00028460BF0ADF801EE106A4DF20A76C3F6B0
:1081E000234600EE906A46F26666C3F666763B4624
:1081F00000EE106A3A46394628460BF0E1F8284668
:108200000AF00AFC28460AF089FC022207212846C7
:108210000AF0FCFD28460AF07DFB4CF6CD43C3F680
:108220004C63022200EE903AB7EE000A3946284627
:108230000AF0EAFE43F608001B21C0F2020013F028
:1082400085FC4EF20020C2F2000014F091FB4DF6C6
:10825000A060C2F200000B210CF0D8FB4DF6A0602C
:10826000C2F200000D210CF039FC48F21010C2F2ED
:108270000100FE210CF070FD002840F0A18043F6C3
:1082800024001721C0F2020013F060FC4EF200201F
:10829000C2F2000014F06CFB43F63C03C0F2020390
:1082A00093E8030040F6A05240F65073C2F2010278
:1082B000C2F2010382E8030083E803004DF68866FA
:1082C000C2F2000640F6EC54C2F20104002301EEB3
:1082D000903A237800EE103A0023C4F2964302EE5F
:1082E000103A0023C4F2482301EE103AB8EE400AD7
:1082F000F0EE610A01F056FFB5EEC00AF1EE10FA99
:1083000000F1388347F67903C4F2302307EE103AC0
:10831000F6EE007AE0EE077A4FF4FC53C0F2010368
:10832000FCEEE77A17EE902A9A4240F226831A462C
:108330004FF4107140F2F423C2F20103187EC50716
:1083400000F12481DD8B1A62A94240F0010088BF50
:10835000D9831876237800EE103A002301EE903A84
:1083600040F658440023C4F20C23C2F2010401EE8B
:10837000103AB8EE400A4FF48033F0EE610AB7EEDF
:10838000002AA36101F00EFF4FF47E43C4F2FF63A5
:1083900007EE903AB4EEE70AF1EE10FA00F3BC8073
:1083A0004FF47E43CCF2FF6307EE903AB4EEE70A57
:1083B000F1EE10FA40F1D7820023C8F20103AEE0DB
:1083C00043F644000E21C0F2020013F0BFFB4EF250
:1083D0000020C2F2000014F0CBFA4DF6886640F699
:1083E0003053C2F20103C2F200061F7008F04CFACB
:1083F000327940F6C85EC2F2010E02EB42034FF63C
:10840000244802EB8302C2F2000840F6A0518EF825
:108410000000C2F2010108EB020008F0C3F8307955
:1084200008F0DEF843F654000621C0F2020013F013
:108430008DFB337903EB430503EB850308EB030561
:1084400028461AF0BDF90146284613F07FFB43F297
:108450005C403946C0F2020013F078FB40F6A050B1
:10846000C2F201001AF0ACF9014640F6A050C2F287
:10847000010013F06BFB43F240203946C0F20200CA
:1084800013F064FB4EF20020C2F2000040F6F055FB
:1084900014F06EFAC2F201052FE043F65C000321EE
:1084A000C0F2020013F052FB4EF2002000230A2219
:1084B0002146C2F2000014F06DFA43F24C40012153
:1084C000C0F2020013F042FB28461AF079F9014687
:1084D000284613F03BFB43F240200121C0F202008A
:1084E00013F034FB4EF200200134C2F2000014F00D
:1084F0003FFA202C05F10B0509D0092CCDD843F209
:108500000C600121C0F2020013F020FBC5E7717975
:10851000307908F04DFBD5E60023C7F6FF7340F62F
:108520007075C2F20105002201EE902A2A78E361FB
:1085300000EE102A0022C4F2482201EE102AB8EE02
:10854000400AF0EE610AB7EE002A01F02BFE4FF46C
:108550007E43F7EE007AC4F2FF6337EEC00A07EEFF
:10856000903AB4EEE70AF1EE10FA19DC4FF47E43CC
:10857000CCF2FF6307EE903AB4EEE70AF1EE10FAA0
:1085800040F1EA810023C8F201030CE01D6AAA420F
:1085900040F29881D88B1A62814288BFD983D9E68C
:1085A0000023C7F6FF732A7800EE102A002201EE9E
:1085B000902A40F690440022C4F24822C2F20104FC
:1085C00001EE102AB8EE400AF0EE610AB7EE002A7A
:1085D000A36101F0E7FD4FF47E43C4F2FF6307EEB1
:1085E000903AB4EEE70AF1EE10FA0FDC4FF47E4356
:1085F000CCF2FF6307EE903AB4EEE70AF1EE10FA20
:1086000040F159810023C8F2010302E00023C7F6BC
:10861000FF732A78E36100EE102A002201EE902A0F
:108620000022C4F2482201EE102AB8EE400AF0EE11
:10863000610AB7EE002A01F0B5FD4FF47E43C4F2A3
:10864000FF6307EE903AB4EEE70AF1EE10FA0FDCA2
:108650004FF47E43CCF2FF6307EE903AB4EEE70AA4
:10866000F1EE10FA40F120810023C8F2010302E08C
:108670000023C7F6FF7340F6ED514FF61042C2F2E9
:108680000101C2F2000209781278236207EE901A03
:1086900007EE102A0022C4F2C82208EE102AF8EED3
:1086A000677AB8EE477AC7EE886A40F66453F26894
:1086B000C2F201031B68C7EE087AB7EE007A77EEC4
:1086C000666A77EE677A00EE902AB268C3ED4A6A6E
:1086D00000EE102A83ED4B7AC3ED497AFDF714FBC7
:1086E0000023C4F22C2307EE903A002306EE903AC2
:1086F000B36807EE103A27EE087A27EE277AC7EE1E
:10870000087A77EEA67AFDEEE77A17EE902A9200C5
:1087100072B640F6C843C2F20103DA6062B61A7C50
:10872000012A40F22F8172B6DA6862B64FF618411C
:10873000002AC2F20001B8BF033292100A607179B8
:1087400072B640F6C84289001962C2F2010262B6EE
:1087500093F82410012940F23A8172B6126A62B687
:108760004FF61843002AB8BF0332C2F2000340F6A6
:10877000CC509210C2F201005A6010F033F940F66A
:10878000DC50C2F2010010F02DF948F29A6448F270
:108790009861C2F20104C2F2010148F2946248F207
:1087A0003863C2F20102C2F2010343F66000258879
:1087B0000C8815801821C0F202001C8013F0C6F945
:1087C0004EF2002000230A223179C2F2000014F098
:1087D000E1F843F25C400121C0F2020013F0B6F967
:1087E0004EF2002000230A227179C2F2000014F038
:1087F000D1F843F240200121C0F2020013F0A6F9A3
:108800004EF20020C2F2000014F0B2F8FEF7B4FFFE
:1088100043F67C001421C0F2020013F097F94EF2E7
:1088200000208021C2F2000014F044F843F69400C6
:108830001121C0F2020013F089F94EF2002040F637
:108840005A31C2F2000014F035F843F6A8000321B3
:10885000C0F2020013F07AF94EF20020C2F20000DA
:1088600014F086F8FEF7AAFE40F65C70C2F2010032
:1088700010F092FA01F0D6FE4EF20813CEF2000389
:10888000012243F6AC001A600B21C0F2020013F083
:108890005DF94EF20020C2F2000014F069F806B053
:1088A000BDEC028BBDE8F081F0EE407AFEEEC87AB6
:1088B00017EE903ADFE6F0EE407AFEEEC87A17EE59
:1088C000903AA6E602F17F01C909013100291A6236
:1088D0000A4638BF0022870706D5596A7F31C90981
:1088E00001318A4238BF0A46450706D5996A7F3169
:1088F000C90901318A4238BF0A46010706D5D96A3B
:108900007F31C90901318A4238BF0A46C70606D5F8
:10891000196B7F31C90901318A4238BF0A46850681
:1089200006D5596B7F31C90901318A4238BF0A46E1
:10893000410606D5996B7F31C90901318A4238BF9A
:108940000A46C10906D0D96B7F31C90901318A4273
:1089500038BF0A46DA83FDE4F0EE407AFEEEC87ACC
:1089600017EE903A1FE6F0EE407AFEEEC87A17EE68
:10897000903AD4E501210022DCE402F17F01C9092B
:108980000131D7E472B61A68586811780478587AB9
:108990001A7A044201EA02013AD09A7A02F00302FA
:1089A000002940F0818042F008029110082A997253
:1089B00036D8072A62D2032A4CD046D9042A37D0A7
:1089C000062A7FF4B1AEDA68023ADA60ADE672B632
:1089D000516990690D780478507F117F044201EA53
:1089E000050129D1927F02F0030200295FD1911085
:1089F000082A997732D8072A52D2032A48D041D977
:108A0000042A32D0062A41D11A6A023A1A62A6E62C
:108A10009A7A02F003020029C7D042F00402C4E7A8
:108A20000C2A17D025D8092ACDD00B2A7FF47CAE8A
:108A3000DA68013ADA6078E6927F02F0030209B15F
:108A400042F0040242F00802D1E7012A16D0022ABD
:108A5000EED069E6DA680232DA6066E60C2A17D0F0
:108A60001AD8092AD0D00B2A10D11A6A013A1A62F0
:108A700075E60D2ADCD00E2A7FF456AEDA68013294
:108A8000DA6052E6012A0BD0022AEED01A6A66E6B4
:108A90001A6A02321A6262E60D2AE6D00E2AF5D16F
:108AA0001A6A01321A625AE642F004027BE742F087
:108AB00004029CE72DE9F0479DF82040013CE4B218
:108AC0000F2C03D84EB2002E0D4601DBBDE8F08717
:108AD000E0290FD9F729F9D90835EDB2012303FAB6
:108AE00005F515F0DD0FF1D0806C0368BDE8F047A7
:108AF0001B6818478146806C1F46036846EA0401DC
:108B0000C9B21B6890469847D9F84800036808F036
:108B10007F011B6805F0EF059847C02DD6D0D9F826
:108B20004800036807F07F011B68BDE8F04718475D
:108B3000F8B50446806C03681B69984708B90020A3
:108B4000F8BDA06C03685B699847C3B203F0FB01F2
:108B5000F929F4D0A26D82B994F84D2084F84F30F1
:108B6000150600F19C8040B20028C0F25081002020
:108B700084F84D00A0656065F8BD010667D494F8DF
:108B80004F10F02904EB020140D081F84F30616DA5
:108B90004B1E9A4240D394F84F20F02AE7D0130698
:108BA0003DD4002384F86630B02B4CD0A02B4AD0A3
:108BB000D02B48D0E02B46D0C02B44D0002094F8D6
:108BC000505084F86750032908BF94F8515084F836
:108BD000650018BF002500210120B02B84F86850E3
:108BE000A165616584F8E90000F0B58000F2AC8011
:108BF000902B00F0B080A02B00F0AD80802B00F017
:108C0000AA80002384F84D300120F8BD81F8693036
:108C1000636D013B9A42AAD20132A2658FE702F14D
:108C20000C03DBB2012BBCD902F0FB03F92BB8D04B
:108C3000EF2A00F2DB8002F0F003802B84F866302C
:108C400001D0902BB0D102F00F000130B7E7A3F1B3
:108C5000F701082993D8012505FA01F010F4DD7F0A
:108C600040F0968000298AD194F86930F02B7FF487
:108C70007EAF561C2244F720370A82F8690084F838
:108C8000676084F8687084F8651084F84D10284691
:108C900084F8663084F8E950A1656165F8BD02F199
:108CA0000C05EEB2012E7FF65EAF02F0FB0EBEF1B8
:108CB000F90F3FF458AFEF2A2DD802F0F007802FBC
:108CC0002AD140B20028FFF64FAF012184F84F208F
:108CD00084F85030A165EDB2012D7FF648AFBEF1AA
:108CE000F90F3FF444AFEF2A5FD802F0F003B02B46
:108CF00026D01ED9D02B04D0E02B21D0C02B7FF45E
:108D000036AF022363650121A36D994227D9013350
:108D1000A3650020F8BD174607F0DF06902ED0D0DF
:108D200007F0BF06A02ECCD007F0EF07C02FC8D0A9
:108D300019E7902B04D0A02B02D0802B7FF417AF23
:108D4000032363650221DFE7D02B04D0E02B02D0A0
:108D5000C02B7FF456AF84F84D200120F8BDEF2AD8
:108D600094BF02F0F005154602F00F020023013215
:108D700094F8501084F86520012084F8671084F876
:108D8000683084F86650A365636584F8E900F8BD2F
:108D9000002284F8672084F8682084F8652084F82D
:108DA000663084F8E9502846F8BDF62A0FD007D877
:108DB000F12AA6D01CD9F22AC2D0F32AA1D0D6E635
:108DC000FC2A21D8FA2A02D2F82A7FF4D0AE002356
:108DD000012084F8653084F8673084F8683084F8BE
:108DE0006620A365636584F8E900F8BD1346D9E6FB
:108DF000F02A7FF4BCAE80210023616584F86920ED
:108E000084F84D307F217FE7FE2AE0D2AFE61A4694
:108E10008E4603F10C055EE790F86630F12B7CD0AE
:108E20000ED9FA2B2BD01FD8F32B38D0C0F081806D
:108E3000F62B7AD0F82B40F08B80036BF3B11847F8
:108E4000B02B6ED031D9D02B21D03ED9E02B42D0DF
:108E5000F02B7ED1C3698BB1B0F86710802900F187
:108E6000690028BF80211847FC2B0CD051D3FE2B62
:108E70004BD0FF2B6BD1436C002BE0D17047436B81
:108E8000002BDCD1FAE7C36B002BD8D1F6E743699E
:108E9000002BF3D090F8671090F865001847836AAC
:108EA000002BEBD090F867001847902B29D0A02B0F
:108EB00023D0802BE2D10368002BDFD090F868200C
:108EC00090F8671090F865001847C02B42D10369ED
:108ED000002BDFD1D2E78269002ACFD090F868104A
:108EE00090F8673090F86500C90101F47E5103F0F5
:108EF0007F031943A1F5005110478368002BDDD192
:108F0000BCE74368002BD9D1B8E7036C002B96D19E
:108F1000B4E7836B002B92D1B0E7036A002BC1D179
:108F2000ACE7C368002BC9D1A8E7C36A002B86D180
:108F3000A4E7426A002AA1D090F8683090F8670050
:108F4000DB0103F47E5300F07F00184310477047A5
:108F500070477047704700BF90F86430DA0725D536
:108F600013F0FE0F22D070B590F8665085F08002A5
:108F7000602A82B004461AD9F62D6ED067D8F12D3A
:108F80007ED04FD9F22D2DD0F32D1AD1806C94F8CC
:108F90006760036829461B689847A06C0368DB6C10
:108FA00006F07F0102B0BDE870401847704790F8A6
:108FB00065608E4207D031B15B08012B08D0032BCE
:108FC00027D002B070BD5B08012B01D0022BF8D175
:108FD00094F8683094F86720009629462046FFF7F9
:108FE00069FDEEE7806C94F86730026894F8686079
:108FF0001268294643EAC6159047A06C036805F03D
:109000007F019B6C9847A06C0368C5F3C6119B6CED
:10901000C8E794F8683094F8672000962946FFF76F
:1090200049FDCEE7F02DCCD1B0F86760802E28BF87
:10903000802600F16905002EC3D02E44A06C15F8DF
:10904000011B03681B689847AE42F7D1B9E7FC2DB6
:1090500026D8FA2D01D2F82DB3D105F10803DBB2E1
:10906000072BAED8012202FA03F313F0DD0FA8D0CC
:10907000A06C03681B68294602B0BDE87040184721
:10908000806C94F8672094F86830066812012946CD
:1090900003F00F0302F0700532681D439047E7E7C5
:1090A000FE2D8ED3D9E700BFF0B540F2A41087B0F3
:1090B000C2F201000BF078FB002840F0F88048F283
:1090C0009044C2F2010440F66C7223680193C2F22C
:1090D0000102019B116841F287325B1A934206D963
:1090E00040F6C953C2F201031B78002B3AD040F678
:1090F0007475C2F2010595F84C60102E43D900201A
:1091000012F03CF940F62C5322680292C2F201039D
:10911000029A1868121A48F29041322AC2F20101EA
:109120004ED840F6605322680492C2F20103049ABA
:109130001968521A632A00F2B58040F2842322682B
:109140000592C2F20103059A196841F28730521A5A
:10915000824205D901F59C5108311960FEF72EFABB
:1091600007B0F0BD40F2A013C2F201031B78002B40
:10917000BDD040F67475C2F20105FDF775FC95F897
:109180004C60102EBBD82846FFF7D2FC0028B6D082
:1091900095F86630902B00F00E8183F08003602BF1
:1091A00040F20C8140F67470C2F20100FFF734FE09
:1091B00040F674703146C2F20100FFF7CDFE9EE723
:1091C00040F664560A680392C2F2010640F634552E
:1091D000039A30681A60C2F2010506F0E5FD40F618
:1091E000C953C2F20103AA881870002A40F04381D3
:1091F00040F23815C2F20105AB88002B40F0F08038
:1092000040F2C425C2F20105AB88002B89D0326838
:10921000D2F8241107EE901A296807EE101A77EE9B
:10922000877A43F63010C2ED497A013B0F21C0F234
:109230000200AB8012F08AFC3368D3F8240118F0E6
:1092400099FA41EC100B4EF200200521C2F2000009
:1092500013F0E0FB43F640101521C0F2020012F0BB
:1092600075FC4EF20020A988C2F2000013F022FB28
:1092700043F658101521C0F2020012F067FC28686E
:1092800018F078FA41EC100B4EF200200521C2F2E2
:10929000000013F0BFFB4EF20020C2F2000013F0FA
:1092A00067FB3EE76431196003F01CFB45E740F2C1
:1092B0007814C2F2010410F071FD2368C01AB0F5F1
:1092C000356F7FF6FCAE10F069FD206040F2A4100F
:1092D000C2F201000BF078FA044610F05FFD40F690
:1092E0006453C2F20103054622461868802106F045
:1092F00049F810F053FD40F65A33401B984252D8BB
:109300004FF6204410F04AFDC2F20004401B2388AF
:10931000834260D372B640F27C13C2F201031A7F1B
:1093200002F0FF010AB100221A7762B6A1B372B649
:1093300047F6FF744FF40040B3F91E50B3F92020F4
:10934000DC83188462B685EAE57182EAE273A3EBF6
:10935000E273A1EBE5718B42B8BF0B4607EE903A82
:109360004FF47E43C4F2FF6306EE103AF8EEE77A5C
:1093700047F2A403C7EE866AC3F67D7307EE103A80
:10938000F4EEC76AF1EE10FA06DD40F69C53C2F225
:1093900001031A6801321A6040F2A410C2F20100FF
:1093A0000BF024FA8BE640F60453C2F201031A686C
:1093B00001321A60A4E795F8683043B195F865303A
:1093C0009E423FF4EFAE002E3FF4ECAEF0E6802379
:1093D00085F86630F2E710F0E1FC401B208099E749
:1093E0003268D2F8281107EE901A296807EE101A91
:1093F00077EE877A43F6E400C2ED4A7A013B122108
:10940000C0F20200AB8012F0A1FB3368D3F8280150
:1094100018F0B0F941EC100B4EF200200521C2F219
:10942000000013F0F7FA43F6F8001821C0F202002A
:1094300012F08CFB4EF20020A988C2F2000013F05B
:1094400039FA43F614101821C0F2020012F07EFB24
:10945000286818F08FF941EC100B4EF2002005211E
:10946000C2F2000013F0D6FA4EF20020C2F2000061
:1094700013F07EFAC4E64DF68867C2F20007013A9F
:10948000FB68AA8000EE903ABB6807EE903A2B6822
:1094900007EE103A37EE870AFCF736FC43F6B800C1
:1094A0000821C0F2020012F051FBB86818F062F90E
:1094B00041EC100B4EF200200521C2F2000013F027
:1094C000A9FA43F6C4000E21C0F2020012F03EFBDE
:1094D0004EF20020A988C2F2000013F0EBF943F627
:1094E000D4000E21C0F2020012F030FB286818F000
:1094F00041F941EC100B4EF200200521C2F20000B0
:1095000013F088FA4EF20020C2F2000013F030FA95
:109510006EE600BF2DE9F04F40F67475C2F201050A
:109520008DB00FF0F5FE95F86430002401264EF260
:10953000E01743F001034FF6FF7E66F34703214631
:1095400085F8654085F8664085F8674085F868408D
:1095500085F8E940C2F2000705F169008022C5F8EC
:109560005CE0C5F860E085F86430AF6485F84C4095
:1095700085F84D4085F84E406C65AC6540F65C77EB
:1095800018F0E2FF4DF6682240F689112846C2F233
:109590000002C0F20001C2F201072C606C60AC60F6
:1095A000EC602C616C61AC61EC612C626C62AC6251
:1095B000EC622C636C63AC63EC632C646C6418F039
:1095C00075FC02231022272138460FF05BFA40F683
:1095D000C84042F69C63C0F2020302220321C2F299
:1095E00001003B60FBF758FC40F6DC401D221C21CB
:1095F000C2F20100FBF750FC48F2904340F6CC5019
:10960000C2F2010314220421C2F201001D4602939A
:109610000FF0D0F940F6DC5014221E21C2F20100F6
:109620000FF0C8F92B68069340F66053C2F20103AD
:1096300040F2A419C2F20109069A1A602146224694
:1096400040F27C1B4846FAF7E1FDC2F2010B44F2FE
:109650001433C0F202030BF118023146584689F860
:109660009C40C9F8984089F89D40C9F8003040F204
:10967000F425FAF7CBFD4FF40041C2F2010547F69D
:10968000FF7244F2BC23ABF8201042F69061C0F2A6
:109690000203ABF81E20C0F2020105F51462CBF8FC
:1096A00000302C722346EC6020466E722A612960DD
:1096B0002C4600E0226942F82300697A013340F227
:1096C000F4229942C2F20102F4DC48F23463C2F29D
:1096D00001030393196809B9A8E219464B69002BE5
:1096E000FBD14D614FF00004002140F6584844F290
:1096F000E42340F23430C2F20108C0F2020369618F
:109700004FF41062AC80EC80AC722C76C2F2010097
:109710004FF000042B606C83AC83EC8318F014FFD3
:1097200008F1280204214046FAF770FD4FF4803317
:1097300040F6384440F69047C2F20107C8F81830A6
:10974000C8F81C30C8F82030C8F82430059340F61B
:109750000856234644F2FC2AC2F20106C2F2010373
:10976000C0F2020A07F12802042138461C46C8F854
:1097700000A00493FAF74AFD059B019606F11C022E
:1097800030460121C7F800A0BB61FB613B627B62F0
:10979000FAF73CFD019B44F2F02A9E462246059BC7
:1097A000CEF81830C0F2020A1C320121204640F6E1
:1097B0007C56CEF800A0FAF729FD059BA361C2F202
:1097C000010642F69063C0F2020306F1180100227E
:1097D000022033604FF000033372707231610B4628
:1097E000C4F800A0F2601146304600E0036943F877
:1097F0002210747A013240F67C539442C2F2010383
:10980000F4DC039A126848F23461C2F201010AB929
:109810000EE21A465369002BFBD15661002440F634
:109820007C5040F2482A44F22C73C0F20203C2F288
:10983000010A7461B480F480B472C2F20100336032
:1098400013F0F4FB50468AE8000A8AF808408AF8C8
:109850000940CAF80C408AF8104040F25C2B12F024
:1098600049FC4DF6682240F68D11C2F2010BC2F29E
:109870000002C0F20001504618F018FB5846CBF821
:109880000090CBF804808BF808408BF80940CBF8A7
:109890000C408BF8104040F2702A12F02BFC4DF671
:1098A000682240F68D11C2F2010AC2F20002C0F233
:1098B0000001584618F0FAFA5046CAF800908AF8A3
:1098C00008408AF80940CAF80C408AF81040CAF8E3
:1098D000047040F6F04912F00DFC4DF6682240F697
:1098E0008D11C2F20109C2F20002C0F2000150461D
:1098F00018F0DCFA4FF0010B484689E8200189F89E
:109900000840C9F80C4089F8104089F809B040F2C5
:10991000882A12F0EFFB4DF6682240F68D11C2F254
:10992000010AC2F20002C0F20001484618F0BEFA75
:10993000022350468AF8093005938AE8A0008AF885
:109940000840CAF80C408AF8104040F29C2912F0F6
:10995000D1FB4DF6682240F68D11C2F20109C2F228
:109960000002C0F20001504618F0A0FA4846C9F8BB
:109970000080C9F8045089F8084089F80940C9F8FE
:109980000C4089F8104040F2B02512F0B3FB4DF6C0
:10999000682240F68D11C2F20105C2F20002C0F247
:1099A0000001484618F082FA2846C5F800802C725B
:1099B000EC602C746F6085F809B040F6685812F0BE
:1099C00099FB4DF6682240F68D11C2F20108C2F2F1
:1099D0000002C0F20001284618F068FA019BC8F89E
:1099E0000430404688F8084088F80940C8F80C4020
:1099F00088F81040C8F8007040F2CC2512F07AFBCD
:109A00004DF6682240F68D11C2F20105C2F2000245
:109A1000C0F20001404618F049FA049B6B602846EA
:109A20002C726C72EC602C742F6040F2E02812F003
:109A300061FB4DF6682240F68D11C2F20108C2F2B8
:109A40000002C0F20001284618F030FA4046C8F87B
:109A5000046088F8084088F80940C8F80C4088F885
:109A60001040C8F8007040F2441512F043FB4DF668
:109A7000682240F68D11C2F20105C2F20002C0F266
:109A80000001404618F012FA28466E602C72EC6015
:109A90002C7485F809B02F6040F63C5612F02AFB72
:109AA0004DF6682240F68D11C2F20106C2F20002A4
:109AB000C0F20001284618F0F9F9059B737242F6CE
:109AC000906306F11801C0F202032246336034723B
:109AD000F460204631610B46344600E0236943F8C8
:109AE0002200717A013240F63C539142C2F20103E6
:109AF000F4DC039A126848F23461C2F201010AB937
:109B000098E01A465369002BFBD15661002440F6B9
:109B10003C5044F20833C0F202037461B480F48014
:109B2000B472C2F2010040F25817C2F2010733606A
:109B30000AF0B8FC019B3C72384687E848007C720A
:109B4000FC603C7412F0D6FA4DF6682240F68D1196
:109B5000C0F200013846C2F2000240F6B45518F0D7
:109B6000A5F9C2F20105049A2C720123284685E862
:109B700044006B72EC602C7412F0BCFA4DF6682253
:109B800040F68D11C0F200012846C2F2000218F022
:109B90008DF940F26C13C2F2010344F2C822C0F204
:109BA00002021A604FF40A700A221A7213F04EF879
:109BB0004AF64441064605F05FF9029F3B68079369
:109BC000079D3B680893089C3B68099340F66450E6
:109BD000C2F2010040F66C7140F2442240F6B053EC
:109BE000C2F20101C2F20102C2F201030660099849
:109BF0000D601460186010F0D1F8029F3B680A9362
:109C00000A9D3B680B9340F2781140F62C5240F2CB
:109C10008423C2F20101C2F20102C2F201030B9CD1
:109C2000086015601C600DB0BDE8F08F1A6059E542
:109C30000B60F3E50B6069E74FF07E52002141674E
:109C400002678267704700BF70B507EE901A2DED6E
:109C5000048BB8EEE79AB7EE008A88EE097A4FF4E3
:109C60006043C4F22B730025002604468663056317
:109C70008561C561C56085604560056007EE903A05
:109C800080ED057A87EE897A0562456380ED049A56
:109C900017EE100A17F06EFD41EC100B15F044F8AA
:109CA00051EC100B18F0B2F849F6AB03C3F6B4430D
:109CB00008EE900A07EE903A68EEA77A40F6DB735A
:109CC00088EE277AC4F2490306EE903A2369C4ED80
:109CD000097A05EE903AB6EE006ABAEE040AA5EEED
:109CE000860A636907EE903A20EE260A84ED0A7A26
:109CF00020EE270A14F0C6FD4BF60B43C3F63243A1
:109D000007EE103A0023C4F2FC2307EE903A68EE07
:109D1000878A87EE897A012323660023CBF6807336
:109D200084F854606566A566E364A364C8EE287A87
:109D300038EE478AC4ED168A84ED1B8ABDEC048B8D
:109D400084ED0B0AC4ED177A70BD00BFF8B50B683F
:109D500006EE903A436E07EE903AC36E07EE103A65
:109D6000836E76EEE77A06EE103AE7EE067A02F1B7
:109D70008047012A2DED108B07F1FF37C1ED007AE6
:109D8000C0ED196A19DD01EB87040B465D6807EE2B
:109D9000905A37EEE67A06EE905AC56E06EE105AE5
:109DA0001D6805EE905AA6EE257A17EE105A43F874
:109DB000045FA342C0ED197AE8D1846FBF0007EEBB
:109DC000904ACB19B7EE007AF4EE477A1B688366A7
:109DD000F1EE10FA11D0002A0FDD3C1D0C440B46A9
:109DE00002E0856F07EE905A1D6807EE105A67EE85
:109DF000277AE3EC017AA342F3D1036F07EE903A9E
:109E0000B7EE007AF4EE477AF1EE10FA00F0FB803C
:109E1000C36C07EE103A436FF4EE477AF1EE10FA96
:109E200016460D46044600EE103A40F0EF80836C73
:109E300007EE903AB4EE670AF1EE10FA40F0E680D1
:109E4000C36B0CEE903AF7EE00BA3CEEABDA002EA4
:109E50008CEE8DBA40F3D78040F6DB73C4F2490331
:109E60000437A66B2F440AEE103A2BEE0B8A46F20B
:109E70006663C3F6E6630DEE903A28EE0B8A4CF665
:109E80007743C3F22B2309EE903A8BEE8D9AF2EED4
:109E90000E8A28EE0B8A10E0022E00F02981032E94
:109EA00040F02281F0EE6B7AECEE2D7A67EEAA7A22
:109EB000E5EC017AAF4200F0A6802B6807EE903AFD
:109EC000E36905EE903AA36906EE103AE36A04EE00
:109ED000103A23680AEE903A63680EEE103AA368CF
:109EE0000FEE103AE3680EEE903A236A0CEE103A49
:109EF000636907EE103A27EE287A37EEE55A27EE27
:109F00000A7AF0EE4E3A25EE075A37EE2B7AEBEE50
:109F10002A3A636AC5EE076AB0EE4F7A75EEA65A22
:109F2000ABEE237AE5EEED7A74EE2B4A77EEC67A45
:109F3000B0EE6E5A67EE847AABEE075A87EEA47ADB
:109F400029EE455A36EE076AF0EE6B3AF0EE467AA5
:109F5000E5EE0C7AECEE083A76EEA55AC7EEA36A67
:109F600037EE066A76EEA96A07EE903A76EEEA6A6E
:109F7000C4ED075AEBEE26AA84ED066AB0EE6A0A33
:109F8000ABEE260A20EE270A14F006FB7AEECE7A14
:109F9000A36A67EEAC7A07EE103A27EE000A87EE66
:109FA0008D7A012E84ED000A77EE0E7A37EECF6AB5
:109FB00037EE277A26EE2C6A84ED017AC6EE0D6A1A
:109FC00036EE8F7A77EE6E5A76EE876A65EEAC5A89
:109FD000C4ED026A85EE8D6A76EE2E6A36EE266A4A
:109FE00084ED036A74D03FF757AF002E7CD1636BCA
:109FF00006EE103A66EE077A3BEEC66AE6EE267A81
:10A00000F0EE67AA4EE7BDEC108BF8BD4BF61423BB
:10A01000B7EE008AC4F23F0309EE103A38EE400A68
:10A02000F3EE038A20EE090A14F0DEFE30EE480A51
:10A030004BF22D2380EE286AC3F67D7307EE103AAB
:10A04000002307EE903AE6EE077A236FF0EE0C6AF3
:10A0500077EE677A06EE103A27EEA67A26EE090A20
:10A06000C4ED107A84ED087A14F0BEFE30EE480A92
:10A070004FF4784380EE286AC4F2936306EE903A78
:10A080000023C4F2702307EE903A40F6DB73C4F26B
:10A090004903E6EE267A07EE103A636906EE903A37
:10A0A00027EEA60A20EE070A14F0ECFB216C226FC3
:10A0B000636F84ED0F0A07EE901A38EE678AF0EEB0
:10A0C00040CABDEEC88AE264A36484ED188ABAE689
:10A0D000636B06EE903A66EEA77A7BEEE66AE6EEF2
:10A0E000877AF0EE67AADDE600230AEE903AD9E619
:10A0F000636B06EE903A6AEEA6AA7BEEE66AE6EE9F
:10A10000A7AACFE610B4036841681A780C78417AA0
:10A11000037A0C4202EA03021AD0837A03F00303A3
:10A120000AB143F0040343F008039A10082B82722B
:10A130002AD8072B22D2032B2ED011D9042B13D0CF
:10A14000062B14D1C3685DF8044B023BC360704713
:10A15000837A03F00303002AE7D043F00403E4E723
:10A16000012B0BD0022B02D1C368013BC3605DF809
:10A17000044B70470D2BF7D00E2BF8D1C3685DF858
:10A18000044B0133C36070470C2B05D0F2D8092B68
:10A19000D8D00B2BE8D0EAE7C3685DF8044B023354
:10A1A000C360704730EE600A32EE612A31EE601A09
:10A1B00020EE022A82EE010A30EE210A704700BF2B
:10A1C00000B583B00FF0A4F848F29042C2F2010249
:10A1D00041F2600312680192C2F20103019A1A600F
:10A1E00003B05DF804FB00BF2DE9F0434DF688682D
:10A1F000C2F200082DED028BD8ED027A9FED748A31
:10A200009FED746AF6EE008AF0EE686AE7EE886AFF
:10A2100048F29043C2F20103B2EE0E7A26EE877A3C
:10A220004FF61147C7EE087A91B0C2F200071B68DB
:10A2300003933A78039941F26003C2F20103012AC1
:10A24000196077EE867AFCEEE77ACDED017A9DF81B
:10A25000046000F0E08140F65C70C2F201000EF094
:10A260009BFD43F67013C0F2020393E803000AACAF
:10A2700000254FF020336360A360E5602561A38172
:10A2800025750A9040F65C702A46ADF82C10C2F293
:10A29000010029460EF03CFD204618F091FA0246D6
:10A2A00040F65C702146C2F2010012F0EDFA4EF267
:10A2B00000202B460A222946C2F2000012F06AFB57
:10A2C00043F25C400121C0F2020011F03FFC4EF26B
:10A2D00000202B460A222946C2F2000012F05AFB47
:10A2E00043F238700321C0F2020011F02FFC204627
:10A2F00018F066FA0146204611F028FC43F240208F
:10A300000121C0F2020011F021FC4EF20020C2F245
:10A31000000012F02DFB40F65C702A23012231462A
:10A32000C2F201000A956560A560E56025612575AA
:10A330008DF828300EF0ECFC204618F041FA024669
:10A3400040F65C702146C2F2010012F09DFA4EF216
:10A3500000202B460A220121C2F2000012F01AFB53
:10A3600043F25C400121C0F2020011F0EFFB4EF21B
:10A3700000202B460A223146C2F2000012F00AFBEE
:10A3800043F238700321C0F2020011F0DFFB2046D7
:10A3900018F016FA0146204611F0D8FB43F240208F
:10A3A0000121C0F2020011F0D1FB4EF20020C2F2F6
:10A3B000000012F0DDFAD8ED027AF0EE686A41F2A0
:10A3C0006408E7EE886AC2F2010888F8006003E0DA
:10A3D0000000C84200000000FDEEE67A0A2217EEF7
:10A3E000900A04A917F0B4FD054618F0E9F9C0B2C7
:10A3F0000328024628BF0322C2F1030043F23003C0
:10A40000C0F230032946204400250A956560A56006
:10A41000E56025612575ADF82830A37018F03EFA87
:10A4200040F65C702A460D21C2F201000EF070FC6D
:10A43000204618F0C5F9024640F65C702146C2F28B
:10A44000010012F021FA4EF200202B460A22294682
:10A45000C2F2000012F09EFA43F25C400121C0F209
:10A46000020011F073FB4EF200202B460A220D2150
:10A47000C2F2000012F08EFA43F238700321C0F2EB
:10A48000020011F063FB204618F09AF901462046BD
:10A4900011F05CFB43F240200121C0F2020011F0F8
:10A4A00055FB4EF20020C2F2000012F061FA98F85B
:10A4B000003041F26408B342C2F2010800F0A48007
:10A4C00040F65C702A2301223146C2F201000A954F
:10A4D0006560A560E560256125758DF828300EF072
:10A4E00017FC204618F06CF9024640F65C702146D5
:10A4F000C2F2010012F0C8F94EF200202B460A22E7
:10A500000121C2F2000012F045FA43F25C40012141
:10A51000C0F2020011F01AFB4EF200202B460A2274
:10A520003146C2F2000012F035FA43F238700321CE
:10A53000C0F2020011F00AFB204618F041F9014672
:10A54000204611F003FB43F240200121C0F202003B
:10A5500011F0FCFA4EF20020C2F2000012F008FAEC
:10A5600098F800900A9540F65C7020234946012235
:10A57000C2F201006560A560E560256125758DF872
:10A5800028300EF0C5FB204618F01AF9024640F6B6
:10A590005C702146C2F2010012F076F94EF2002002
:10A5A0002B460A220121C2F2000012F0F3F943F215
:10A5B0005C400121C0F2020011F0C8FA4EF2002006
:10A5C0002B460A224946C2F2000012F0E3F943F298
:10A5D00038700321C0F2020011F0B8FA204618F0DA
:10A5E000EFF80146204611F0B1FA43F24020012174
:10A5F000C0F2020011F0AAFA4EF20020C2F20000EE
:10A6000012F0B6F988F8006001233B7011B0BDEC80
:10A61000028BBDE8F08341F26408C2F201080AAC83
:10A62000DAE600BF2DE9F0434FF61147C2F200070A
:10A630008DB03B78002B40F094854DF68866C2F2D1
:10A64000000669460A22307917F082FC044618F0A9
:10A65000B7F8C0B20228024628BF0222C2F10200A7
:10A6600006AB21461844002443F2300306940794B5
:10A67000ADF81830089409940A948DF82C4018F01D
:10A680000DF940F65C7022462146C2F201000EF040
:10A690003FFB06A818F094F8024640F65C7006A945
:10A6A000C2F2010012F0F0F84EF2002023460A2216
:10A6B0002146C2F2000012F06DF943F25C40012124
:10A6C000C0F2020011F042FA4EF2002023460A22A4
:10A6D0002146C2F2000012F05DF943F23870032106
:10A6E000C0F2020011F032FA06A818F069F801462B
:10A6F00006A811F02BFA43F240200121C0F202001B
:10A7000011F024FA4EF20020C2F2000012F030F9EB
:10A7100040F65C7022460221C2F201004FF020098F
:10A7200006940794089409940A948DF82C408DF8A7
:10A7300018900EF0EDFA06A818F042F8024640F61E
:10A740005C7006A9C2F2010012F09EF84EF20020E1
:10A7500023460A222146C2F2000012F01BF943F2FE
:10A760005C400121C0F2020011F0F0F94EF200202D
:10A7700023460A220221C2F2000012F00BF943F232
:10A7800038700321C0F2020011F0E0F906A818F0B9
:10A7900017F8014606A811F0D9F943F2402001212B
:10A7A000C0F2020011F0D2F94EF20020C2F2000015
:10A7B00012F0DEF833794FF6244003EB43024DF6F6
:10A7C000866803EB8203C2F2000040F6A051C2F299
:10A7D00000081844C2F2010105F0E4FE98F80050A8
:10A7E00040F65C7015F0FD05C2F2010000F0D08269
:10A7F0002246022106940794089409940A948DF83D
:10A800002C408DF818900EF083FA06A817F0D8FFA8
:10A81000024640F65C7006A9C2F2010012F034F85C
:10A820004EF2002023460A222146C2F2000012F016
:10A83000B1F843F25C400121C0F2020011F086F948
:10A840004EF2002023460A220221C2F2000012F03A
:10A85000A1F843F238700321C0F2020011F076F93A
:10A8600006A817F0ADFF014606A811F06FF943F2F4
:10A8700040200121C0F2020011F068F94EF20020E0
:10A88000C2F2000012F074F840F6A050C2F20100CB
:10A8900017F096FFC2B2082A40F6A05128BF08223E
:10A8A0004FF02033C2F2010106A8069307940894E2
:10A8B000CDF81B3009940A948DF82C4017F0EEFF68
:10A8C00040F65C7022460321C2F201000EF020FA2D
:10A8D00006A817F075FF024640F65C7006A9C2F2A2
:10A8E000010011F0D1FF4EF2002023460A2221463A
:10A8F000C2F2000012F04EF843F25C400121C0F2B7
:10A90000020011F023F94EF2002023460A2203210F
:10A91000C2F2000012F03EF843F238700321C0F298
:10A92000020011F013F906A817F04AFF014606A825
:10A9300011F00CF943F240200121C0F2020011F0A5
:10A9400005F94EF20020C2F2000012F011F840F6B4
:10A950005C7022460B21C2F2010006940794089411
:10A9600009940A948DF82C408DF818900EF0D0F9C7
:10A9700006A817F025FF024640F65C7006A9C2F251
:10A98000010011F081FF4EF2002023460A222146E9
:10A99000C2F2000011F0FEFF43F25C40C0F2020080
:10A9A000012111F0D3F823464EF200200A220B2198
:10A9B000C2F2000011F0EEFF43F238700321C0F242
:10A9C000020011F0C3F806A817F0FAFE014606A827
:10A9D00011F0BCF843F240200121C0F2020011F056
:10A9E000B5F84EF20020C2F2000011F0C1FF7079FC
:10A9F00069460A22013017F0ABFA044617F0E0FE70
:10AA0000C0B20228024628BF0222C2F1020006ABF1
:10AA100021461844002443F2300306940794ADF80D
:10AA20001830089409940A948DF82C4017F036FFDA
:10AA300040F65C7021460122C2F201000EF068F976
:10AA400006A817F0BDFE024640F65C7006A9C2F2E9
:10AA5000010011F019FF4EF2002023460A220121C5
:10AA6000C2F2000011F096FF43F25C400121C0F2F7
:10AA7000020011F06BF84EF2002023460A22214614
:10AA8000C2F2000011F086FF43F238700321C0F2D9
:10AA9000020011F05BF806A817F092FE014606A826
:10AAA00011F054F843F240200121C0F2020011F0ED
:10AAB0004DF84EF20020C2F2000011F059FF40F6AE
:10AAC0005C7001220221C2F2010020250694079445
:10AAD000089409940A948DF82C408DF818500EF0C3
:10AAE00017F906A817F06CFE024640F65C7006A93E
:10AAF000C2F2010011F0C8FE4EF2002023460A22E5
:10AB00000121C2F2000011F045FF43F25C40012137
:10AB1000C0F2020011F01AF84EF2002023460A2279
:10AB20000221C2F2000011F035FF43F23870032118
:10AB3000C0F2020011F00AF806A817F041FE014623
:10AB400006A811F003F843F240200121C0F20200F0
:10AB500010F0FCFF4EF20020C2F2000011F008FFDE
:10AB600098F8008008F0FD084DF6886640F65C70A5
:10AB7000B8F1010FC2F20006C2F2010000F0E78155
:10AB80000122022106940794089409940A948DF8EE
:10AB90002C408DF818500EF0BBF806A817F010FEE8
:10ABA000024640F65C7006A9C2F2010011F06CFE8C
:10ABB0004EF2002023460A220121C2F2000011F0C9
:10ABC000E9FE43F25C400121C0F2020010F0BEFF3A
:10ABD0004EF2002023460A220221C2F2000011F0A8
:10ABE000D9FE43F238700321C0F2020010F0AEFF2C
:10ABF00006A817F0E5FD014606A810F0A7FF43F2EE
:10AC000040200121C0F2020010F0A0FF4EF200200F
:10AC1000C2F2000011F0ACFE727940F6F05302EB84
:10AC2000820602EB4606C2F201031E44304617F0CC
:10AC3000C7FDC2B20A2A28BF0A224FF0203331468C
:10AC400006A806930793089409940A948DF82C405B
:10AC50008DF8205017F022FE40F65C70012203218F
:10AC6000C2F201000EF054F806A817F0A9FD024642
:10AC700040F65C7006A9C2F2010011F005FE4EF22A
:10AC8000002023460A220121C2F2000011F082FEB8
:10AC900043F25C400121C0F2020010F057FF4EF277
:10ACA000002023460A220321C2F2000011F072FEA6
:10ACB00043F238700321C0F2020010F047FF06A8EB
:10ACC00017F07EFD014606A810F040FF43F2402039
:10ACD0000121C0F2020010F039FF4EF20020C2F252
:10ACE000000011F045FE40F65C7001220E21C2F218
:10ACF000010006940794089409940A948DF82C4056
:10AD00008DF818500EF004F806A817F059FD024609
:10AD100040F65C7006A9C2F2010011F0B5FD4EF2DA
:10AD2000002023460A220121C2F2000011F032FE67
:10AD300043F25C400121C0F2020010F007FF4EF226
:10AD4000002023460A220E21C2F2000011F022FE4A
:10AD500043F238700321C0F2020010F0F7FE06A89B
:10AD600017F02EFD014606A810F0F0FE43F2402039
:10AD70000121C0F2020010F0E9FE4EF20020C2F202
:10AD8000000011F0F5FD00233B700DB0BDE8F0832D
:10AD90005B232A460221069507958DF81830089501
:10ADA00009950A958DF82C500DF0B2FF06A817F002
:10ADB00007FD024640F65C7006A9C2F2010011F0E0
:10ADC00063FD4EF200202B460A222946C2F2000003
:10ADD00011F0E0FD43F25C400121C0F2020010F0EE
:10ADE000B5FE4EF200202B460A220221C2F20000DC
:10ADF00011F0D0FD43F238700321C0F2020010F0D0
:10AE0000A5FE06A817F0DCFC014606A810F09EFE81
:10AE100043F240200121C0F2020010F097FE4EF2F2
:10AE20000020C2F2000011F0A3FD40F6A050C2F2D3
:10AE3000010017F0C5FCC2B2082A40F6A05128BF95
:10AE400008224FF02033C2F2010106A806930795AD
:10AE50000895CDF81B3009950A958DF82C5017F000
:10AE60001DFD40F65C702A460321C2F201000DF080
:10AE70004FFF06A817F0A4FC024640F65C7006A936
:10AE8000C2F2010011F000FD4EF200202B460A2212
:10AE90002946C2F2000011F07DFD43F25C40012121
:10AEA000C0F2020010F052FE4EF200202B460A22A1
:10AEB0000321C2F2000011F06DFD43F2387003214E
:10AEC000C0F2020010F042FE06A817F079FC01461D
:10AED00006A810F03BFE43F240200121C0F2020020
:10AEE00010F034FE4EF20020C2F2000011F040FDDE
:10AEF00040F65C705D232A460B21C2F201000695E4
:10AF000007958DF81830089509950A958DF82C50FD
:10AF10000DF0FEFE06A817F053FC024640F65C70EA
:10AF200006A9C2F2010011F0AFFC4EF200202B4640
:10AF30000A222946C2F2000011F02CFD43F25C40C7
:10AF4000C0F20200012110F001FE2B462CE55B232C
:10AF500042460221069407948DF81830089409940B
:10AF60000A948DF82C400DF0D3FE06A817F028FCAB
:10AF7000024640F65C7006A9C2F2010011F084FCA2
:10AF80004EF2002023460A224146C2F2000011F090
:10AF900001FD43F25C404146C0F2020010F0D6FDD4
:10AFA0004EF2002023460A220221C2F2000011F0D4
:10AFB000F1FC43F238700321C0F2020010F0C6FD2C
:10AFC00006A817F0FDFB014606A810F0BFFD43F2EE
:10AFD00040204146C0F2020010F0B8FD4EF20020C1
:10AFE000C2F2000011F0C4FC727940F6F05302EB9B
:10AFF000820602EB4606C2F201031E44304617F0F9
:10B00000DFFBC2B20A2A28BF0A224FF020333146A2
:10B0100006A806930793089409940A948DF82C4087
:10B020008DF8205017F03AFC40F65C704246032140
:10B03000C2F201000DF06CFE06A817F0C1FB02463B
:10B0400040F65C7006A9C2F2010011F01DFC4EF240
:10B05000002023460A224146C2F2000011F09AFC69
:10B0600043F25C404146C0F2020010F06FFD4EF228
:10B07000002023460A220321C2F2000011F08AFCBC
:10B0800043F238700321C0F2020010F05FFD06A801
:10B0900017F096FB014606A810F058FD43F2402039
:10B0A0004146C0F2020010F051FD4EF20020C2F203
:10B0B000000011F05DFC40F65C705D2342460E21FD
:10B0C000C2F20100069407948DF818300894099490
:10B0D0000A948DF82C400DF01BFE06A817F070FBAB
:10B0E000024640F65C7006A9C2F2010011F0CCFBEA
:10B0F0004EF2002023460A224146C2F2000011F01F
:10B1000049FC43F25C404146C0F2020010F01EFDD3
:10B110004EF2002023460A220E21C2F2000011F056
:10B1200039FC43F238700321C0F2020010F00EFD2A
:10B1300006A817F045FB014606A810F007FD43F2EC
:10B1400040204146C0F2020010F000FD4EF2002007
:10B15000C2F2000011F00CFC00233B700DB0BDE802
:10B16000F08340F65C70C2F201000DF015FEFFF7AF
:10B1700064BA00BF2DE9F0414FF61146C2F2000655
:10B180008CB03378032B00F03E8340F65C70C2F243
:10B1900001000DF001FE43F67813C0F2020393E8BC
:10B1A000030006AC00254FF02033A3606360E56028
:10B1B0002561C4F80B302575069040F65C702A4670
:10B1C000ADF81C10C2F2010029460DF0A1FD204689
:10B1D00017F0F6FA024640F65C702146C2F2010012
:10B1E00011F052FB4EF200202B460A222946C2F2F1
:10B1F000000011F0CFFB43F25C400121C0F20200DD
:10B2000010F0A4FC4EF200202B460A222946C2F27E
:10B21000000011F0BFFB43F238700321C0F20200BE
:10B2200010F094FC204617F0CBFA0146204610F0AF
:10B230008DFC43F240200121C0F2020010F086FC98
:10B240004EF20020C2F2000011F092FB46F252537F
:10B2500040F65C70C3F6732329460122C2F2010056
:10B260006560A560E5602561257506930DF050FDCC
:10B27000204617F0A5FA024640F65C702146C2F25D
:10B28000010011F001FB4EF200202B460A220121A1
:10B29000C2F2000011F07EFB43F25C400121C0F2DB
:10B2A000020010F053FC4EF200202B460A222946E1
:10B2B000C2F2000011F06EFB43F238700321C0F2BD
:10B2C000020010F043FC204617F07AFA01462046AF
:10B2D00010F03CFC43F240200121C0F2020010F0CB
:10B2E00035FC4EF20020C2F2000011F041FB47F2A3
:10B2F000435340F65C70C3F6742301220821C2F266
:10B3000001006560A560E5602561257506930DF077
:10B31000FFFC204617F054FA024640F65C702146C6
:10B32000C2F2010011F0B0FA4EF200202B460A22C0
:10B330000121C2F2000011F02DFB43F25C4001211B
:10B34000C0F2020010F002FC4EF200202B460A224E
:10B350000821C2F2000011F01DFB43F238700321F6
:10B36000C0F2020010F0F2FB204617F029FA014665
:10B37000204610F0EBFB43F24020C0F20200012116
:10B3800010F0E4FB4EF20020C2F2000011F0F0FADF
:10B3900040F6ED53C2F201034FF2CB081B7803EBEA
:10B3A000830303EB8303C2F68D089B0088FB032015
:10B3B000DB17C3EB201069460A2216F0C9FD0546CB
:10B3C00017F0FEF9C0B20228024628BF0222C2F1DD
:10B3D0000200294643F230070025204406956560A7
:10B3E000A560E56025612575ADF8187017F056FA6F
:10B3F00040F65C7001220521C2F201000DF088FCCC
:10B40000204617F0DDF9024640F65C702146C2F294
:10B41000010011F039FA4EF200202B460A220121D8
:10B42000C2F2000011F0B6FA43F25C400121C0F212
:10B43000020010F08BFB4EF200200A222B46052161
:10B44000C2F2000011F0A6FA43F238700321C0F2F4
:10B45000020010F07BFB204617F0B2F901462046AF
:10B4600010F074FB43F240200121C0F2020010F002
:10B470006DFB4EF20020C2F2000011F079FA4FF697
:10B480001043C2F2000369461B7803EB830303EB0E
:10B4900083039B0088FB0320DB17C3EB20100A22E9
:10B4A00016F056FD804617F08BF9C0B2022802460E
:10B4B00028BF0222C2F10200414620440695656081
:10B4C000A560E56025612575ADF8187017F0E6F9FF
:10B4D00040F65C7001220D21C2F201000DF018FC53
:10B4E000204617F06DF9024640F65C702146C2F224
:10B4F000010011F0C9F94EF200202B460A22012169
:10B50000C2F2000011F046FA43F25C400121C0F2A1
:10B51000020010F01BFB4EF200202B460A220D21E8
:10B52000C2F2000011F036FA43F238700321C0F283
:10B53000020010F00BFB204617F042F901462046AE
:10B5400010F004FB43F240200121C0F202004DF64E
:10B55000866710F0FBFAC2F200074EF20020C2F23A
:10B56000000011F005FA97F8008040F65C70B8F121
:10B57000040FC2F2010000F04881012204214FF0C3
:10B58000200806956560A560E560256125758DF844
:10B5900018800DF0BDFB204617F012F9024640F668
:10B5A0005C702146C2F2010011F06EF94EF20020EB
:10B5B0002B460A220121C2F2000011F0EBF943F2FE
:10B5C0005C400121C0F2020010F0C0FA4EF20020EF
:10B5D0000A222B460421C2F2000011F0DBF943F2EB
:10B5E00038700321C0F2020010F0B0FA204617F0C4
:10B5F000E7F80146204610F0A9FA43F24020012165
:10B60000C0F2020010F0A2FA4EF20020C2F20000D6
:10B6100011F0AEF940F65C700695C2F2010065606B
:10B62000A560E56025612575012207218DF8188048
:10B630000DF06EFB204617F0C3F8024640F65C7032
:10B640002146C2F2010011F01FF94EF200202B46F4
:10B650000A220121C2F2000011F09CF943F25C4081
:10B660000121C0F2020010F071FA4EF200202B46C8
:10B670000A220721C2F2000011F08CF943F238705F
:10B680000321C0F2020010F061FA204617F098F88A
:10B690000146204610F05AFA43F240200121C0F240
:10B6A000020010F053FA4EF20020C2F2000011F036
:10B6B0005FF93B7840F65C70052B4FF00005C2F255
:10B6C000010000F0FE8001220C2120270695656014
:10B6D000A560E560256125758DF818700DF018FBE3
:10B6E000204617F06DF8024640F65C702146C2F223
:10B6F000010011F0C9F84EF200202B460A22012168
:10B70000C2F2000011F046F943F25C400121C0F2A0
:10B71000020010F01BFA4EF200200A222B460C21E8
:10B72000C2F2000011F036F943F238700321C0F282
:10B73000020010F00BFA204617F042F801462046AE
:10B7400010F004FA43F240200121C0F2020010F090
:10B75000FDF94EF20020C2F2000011F009F940F6A6
:10B760005C700695C2F201006560A560E560256128
:10B77000257501220F218DF818700DF0C9FA2046A9
:10B7800017F01EF8024640F65C702146C2F2010036
:10B7900011F07AF84EF200202B460A220121C2F263
:10B7A000000011F0F7F843F25C400121C0F2020002
:10B7B00010F0CCF94EF200202B460A220F21C2F2E3
:10B7C000000011F0E7F843F238700321C0F20200E4
:10B7D00010F0BCF9204616F0F3FF0146204610F0A9
:10B7E000B5F943F240200121C0F2020010F0AEF999
:10B7F0004EF20020C2F2000011F0BAF803233370B9
:10B800000CB0BDE8F08106ACC2E55B2301224146E5
:10B8100006956560A560E560256125758DF8183091
:10B820000DF076FA204616F0CBFF024640F65C702B
:10B830002146C2F2010011F027F84EF200202B46FB
:10B840000A220121C2F2000011F0A4F843F25C4088
:10B850000121C0F2020010F079F94EF200202B46CF
:10B860000A224146C2F2000011F094F843F2387007
:10B870000321C0F2020010F069F9204616F0A0FF83
:10B880000146204610F062F943F240200121C0F247
:10B89000020010F05BF94EF20020C2F2000011F03D
:10B8A00067F840F65C705D230695C2F201006560A2
:10B8B000A560E56025612575012207218DF8183006
:10B8C000B6E65B2301220C2106956560A560E56064
:10B8D000256125758DF818300DF01AFA204616F0FE
:10B8E0006FFF024640F65C702146C2F2010010F084
:10B8F000CBFF4EF200202B460A220121C2F20000AB
:10B9000011F048F843F25C400121C0F2020010F04F
:10B910001DF94EF200202B460A220C21C2F2000033
:10B9200011F038F843F238700321C0F2020010F031
:10B930000DF9204616F044FF0146204610F006F9A6
:10B9400043F240200121C0F2020010F0FFF84EF255
:10B950000020C2F2000011F00BF840F65C705D238D
:10B960000695C2F201006560A560E5602561257558
:10B9700001220F218DF81830FFE600BFF0B548F224
:10B980009043C2F201034FF611468FB0C2F2000697
:10B990001B6801933278019941F26003C2F20103FE
:10B9A000022A196000F0D18040F65C70C2F20100FA
:10B9B0000DF0F2F943F68013C0F2020393E807009A
:10B9C00008AC00254FF02033E560C4F80B3084E864
:10B9D000070040F65C702A462946C2F20100256144
:10B9E00025750DF095F9204616F0EAFE024640F660
:10B9F0005C702146C2F2010010F046FF4EF20020BA
:10BA00002B4629460A22C2F2000010F0C3FF43F27F
:10BA10005C400121C0F2020010F098F84EF20020C4
:10BA20002B460A222946C2F2000010F0B3FF43F26F
:10BA300038700321C0F2020010F088F8204616F09A
:10BA4000BFFE0146204610F081F843F2402001215C
:10BA5000C0F202004DF6886710F078F8C2F20007D5
:10BA60004EF20020C2F2000010F082FF3D7C002D5B
:10BA700073D00A2202A9284616F06AFA054616F083
:10BA80009FFEC0B20228024628BF0222C2F1020075
:10BA900043F2300329462044002508956560A560DF
:10BAA000E56025612575ADF8203016F0F7FE40F60B
:10BAB0005C7029460122C2F201000DF029F92046EE
:10BAC00016F07EFE024640F65C702146C2F201008E
:10BAD00010F0DAFE4EF200202B460A220121C2F2BB
:10BAE000000010F057FF43F25C400121C0F2020059
:10BAF00010F02CF84EF200202B460A222946C2F202
:10BB0000000010F047FF43F238700321C0F202003A
:10BB100010F01CF8204616F053FE0146204610F0A7
:10BB200015F843F240200121C0F2020010F00EF897
:10BB30004EF20020C2F2000010F01AFF3F7C012FED
:10BB400060D0022333700FB0F0BD4DF68867C2F2AB
:10BB5000000708AC3D7C002D8BD144F64F5340F6D6
:10BB60005C70C4F64E1329460122C2F201006560E2
:10BB7000A560E5602561257508930DF0C9F820469C
:10BB800016F01EFE024640F65C702146C2F201002D
:10BB900010F07AFE4EF200202B460A220121C2F25A
:10BBA000000010F0F7FE43F25C400121C0F20200F9
:10BBB0000FF0CCFF4EF200202B460A222946C2F29B
:10BBC000000010F0E7FE43F238700321C0F20200DB
:10BBD0000FF0BCFF204616F0F3FD014620460FF0A3
:10BBE000B5FF43F240200121C0F202000FF0AEFF8A
:10BBF0004EF20020C2F2000010F0BAFE02233370B1
:10BC00000FB0F0BD40F65C7042F220033A460221CC
:10BC1000C2F2010008956560A560E56025612575A3
:10BC2000ADF820300DF074F8204616F0C9FD02463C
:10BC300040F65C702146C2F2010010F025FE4EF283
:10BC400000202B460A223946C2F2000010F0A2FE64
:10BC500043F25C403946C0F202000FF077FF4EF22B
:10BC600000202B460A220221C2F2000010F092FEB0
:10BC700043F238700321C0F202000FF067FF204644
:10BC800016F09EFD014620460FF060FF43F2402073
:10BC90003946C0F202000FF059FF4EF20020C2F206
:10BCA000000010F065FE022333700FB0F0BD00BF3E
:10BCB0002DE9F0414FF61146C2F200068CB0337800
:10BCC000042B00F0F88440F65C70C2F201000DF025
:10BCD00063F843F69013C0F2020393E8030006AC46
:10BCE00000256560A560E56025612575069040F634
:10BCF0005C702A468DF81C10C2F2010029460DF036
:10BD000007F8204616F05CFD024640F65C702146BE
:10BD1000C2F2010010F0B8FD4EF200202B460A22BC
:10BD20002946C2F2000010F035FE43F25C400121CA
:10BD3000C0F202000FF00AFF4EF200202B460A224A
:10BD40002946C2F2000010F025FE43F238700321AC
:10BD5000C0F202000FF0FAFE204616F031FD014657
:10BD600020460FF0F3FE43F240200121C0F2020012
:10BD70000FF0ECFE4EF20020C2F2000010F0F8FDD1
:10BD800040F65C7043F654232A460621C2F20100B5
:10BD900006956560A560E56025612575ADF81830EC
:10BDA0000CF0B6FF204616F00BFD024640F65C7024
:10BDB0002146C2F2010010F067FD4EF200202B4632
:10BDC0000A222946C2F2000010F0E4FD43F25C4072
:10BDD0000121C0F202000FF0B9FE4EF200202B4606
:10BDE0000A220621C2F2000010F0D4FD43F238709E
:10BDF0000321C0F202000FF0A9FE204616F0E0FC7D
:10BE0000014620460FF0A2FE43F240200121C0F27D
:10BE100002000FF09BFE4EF20020C2F2000010F074
:10BE2000A7FD40F65C7047F26D332A460E21C2F240
:10BE3000010006956560A560E56025612575ADF892
:10BE400018300CF065FF204616F0BAFC024640F6AA
:10BE50005C702146C2F2010010F016FD4EF2002087
:10BE60002B460A222946C2F2000010F093FD43F24D
:10BE70005C400121C0F202000FF068FE4EF200208B
:10BE80002B460A220E21C2F2000010F083FD43F27D
:10BE900038700321C0F202000FF058FE204616F061
:10BEA0008FFC014620460FF051FE43F24020012155
:10BEB000C0F202000FF04AFE4EF20020C2F2000073
:10BEC00010F056FD43F69813C0F2020340F65C7082
:10BED0001B6806951F0C29460122C2F2010065600D
:10BEE000A560E56025612575ADF818308DF81A70EC
:10BEF0000CF00EFF204616F063FC024640F65C7024
:10BF00002146C2F2010010F0BFFC4EF200202B4689
:10BF10000A220121C2F2000010F03CFD43F25C4015
:10BF20000121C0F202000FF011FE4EF200202B465C
:10BF30000A222946C2F2000010F02CFD43F23870AC
:10BF40000321C0F202000FF001FE204616F038FC7B
:10BF5000014620460FF0FAFD43F240200121C0F2D5
:10BF600002000FF0F3FD4EF20020C2F2000010F0CC
:10BF7000FFFC46F6567340F65C70C3F66C23012254
:10BF80000821C2F201006560A560E56025612575A4
:10BF900006930CF0BDFE204616F012FC024640F659
:10BFA0005C702146C2F2010010F06EFC4EF20020DF
:10BFB0002B460A220121C2F2000010F0EBFC43F2F2
:10BFC0005C400121C0F202000FF0C0FD4EF20020E3
:10BFD0002B460A220821C2F2000010F0DBFC43F2DB
:10BFE00038700321C0F202000FF0B0FD204616F0B9
:10BFF000E7FB014620460FF0A9FD43F24020C0F2C6
:10C00000020001210FF0A2FD4EF20020C2F200005A
:10C0100010F0AEFC40F24012C2F201024FF49663FF
:10C02000107848F21F57C5F2EB1703FB00F387FBAC
:10C030000320DB17C3EB201069460A2215F088FFA6
:10C04000054616F0BDFBC0B20428024628BF0422F4
:10C05000C2F104004FF030332946204400256560CA
:10C06000A560E56025612575069316F017FC40F67E
:10C070005C702A460921C2F201000CF049FE2046FC
:10C0800016F09EFB024640F65C702146C2F20100AB
:10C0900010F0FAFB4EF200202B460A222946C2F28B
:10C0A000000010F077FC43F25C400121C0F2020076
:10C0B0000FF04CFD4EF200200A222B460921C2F25D
:10C0C000000010F067FC43F238700321C0F2020058
:10C0D0000FF03CFD204616F073FB014620460FF0A2
:10C0E00035FD43F240200121C0F202000FF02EFD89
:10C0F0004EF20020C2F2000010F03AFC40F6EC5381
:10C10000C2F201034AF2EB001B7803EB430303EB9B
:10C110004313CEF60E2080FB03201844DB17C3EB3D
:10C12000601069460A2215F013FF804616F048FB9E
:10C13000C0B20228024628BF0222C2F102004146D4
:10C14000204443F2300806956560A560E5602561EE
:10C150002575ADF8188016F0A1FB40F65C70012241
:10C160000421C2F201000CF0D3FD204616F028FB9A
:10C17000024640F65C702146C2F2010010F084FBDA
:10C180004EF200202B460A220121C2F2000010F0DC
:10C1900001FC43F25C400121C0F202000FF0D6FC2A
:10C1A0004EF200200A222B460421C2F2000010F0B9
:10C1B000F1FB43F238700321C0F202000FF0C6FC1D
:10C1C000204616F0FDFA014620460FF0BFFC43F270
:10C1D00040200121C0F202000FF0B8FC4EF2002016
:10C1E000C2F2000010F0C4FB40F67073C2F201030B
:10C1F00069461B7803EB430303EB431387FB0320E0
:10C20000DB17C3EB20100A2215F0A2FE074616F03A
:10C21000D7FAC0B20228024628BF0222C2F10200A9
:10C220003946204406956560A560E5602561257561
:10C23000ADF8188016F032FB40F65C7001220D213B
:10C24000C2F201000CF064FD204616F0B9FA024675
:10C2500040F65C702146C2F2010010F015FB4EF270
:10C2600000202B460A220121C2F2000010F092FBAE
:10C2700043F25C400121C0F202000FF067FC4EF275
:10C2800000202B460A220D21C2F2000010F082FB92
:10C2900043F238700321C0F202000FF057FC204631
:10C2A00016F08EFA014620460FF050FC43F2402073
:10C2B0000121C0F202004DF686670FF047FCC2F282
:10C2C00000074EF20020C2F2000010F051FB3B7854
:10C2D00040F65C70062BC2F2010000F04A822A464A
:10C2E00008214FF0200806956560A560E56025618E
:10C2F00025758DF818800CF00BFD204616F060FABD
:10C30000024640F65C702146C2F2010010F0BCFA11
:10C310004EF200202B460A222946C2F2000010F0FD
:10C3200039FB43F25C400121C0F202000FF00EFC29
:10C330004EF200200A222B460821C2F2000010F023
:10C3400029FB43F238700321C0F202000FF0FEFB1C
:10C35000204616F035FA014620460FF0F7FB43F26F
:10C3600040200121C0F202000FF0F0FB4EF200204D
:10C37000C2F2000010F0FCFA40F65C700695C2F2C2
:10C3800001006560A560E560256125752A460D21DF
:10C390008DF818800CF0BCFC204616F011FA02460D
:10C3A00040F65C702146C2F2010010F06DFA4EF2C8
:10C3B00000202B460A222946C2F2000010F0EAFAB9
:10C3C00043F25C400121C0F202000FF0BFFB4EF2CD
:10C3D00000202B460A220D21C2F2000010F0DAFAEA
:10C3E00043F238700321C0F202000FF0AFFB204689
:10C3F00016F0E6F9014620460FF0A8FB43F2402074
:10C400000121C0F202000FF0A1FB4EF20020C2F2A7
:10C41000000010F0ADFA3B7840F65C70072B4FF04F
:10C420000005C2F2010000F04881012203214FF013
:10C43000200806956560A560E560256125758DF885
:10C4400018800CF065FC204616F0BAF9024640F65A
:10C450005C702146C2F2010010F016FA4EF2002084
:10C460002B460A220121C2F2000010F093FA43F297
:10C470005C400121C0F202000FF068FB4EF2002088
:10C480000A222B460321C2F2000010F083FA43F285
:10C4900038700321C0F202000FF058FB204616F05E
:10C4A0008FF9014620460FF051FB43F24020012155
:10C4B000C0F202000FF04AFB4EF20020C2F2000070
:10C4C00010F056FA40F65C700695C2F20100656005
:10C4D000A560E56025612575012206218DF818808B
:10C4E0000CF016FC204616F06BF9024640F65C7024
:10C4F0002146C2F2010010F0C7F94EF200202B468F
:10C500000A220121C2F2000010F044FA43F25C401A
:10C510000121C0F202000FF019FB4EF200202B4661
:10C520000A220621C2F2000010F034FA43F23870F9
:10C530000321C0F202000FF009FB204616F040F97B
:10C54000014620460FF002FB43F240200121C0F2D9
:10C5500002000FF0FBFA4EF20020C2F2000010F0D1
:10C5600007FA3B7840F65C70082B4FF00005C2F2EA
:10C57000010000F05A8101220C21202706956560F8
:10C58000A560E560256125758DF818700CF0C0FB7D
:10C59000204616F015F9024640F65C702146C2F2BC
:10C5A000010010F071F94EF200202B460A22012101
:10C5B000C2F2000010F0EEF943F25C400121C0F23B
:10C5C00002000FF0C3FA4EF200200A222B460C2183
:10C5D000C2F2000010F0DEF943F238700321C0F21D
:10C5E00002000FF0B3FA204616F0EAF801462046A2
:10C5F0000FF0ACFA43F240200121C0F202000FF02C
:10C60000A5FA4EF20020C2F2000010F0B1F940F697
:10C610005C700695C2F201006560A560E560256169
:10C62000257501220F218DF818700CF071FB204642
:10C6300016F0C6F8024640F65C702146C2F20100D0
:10C6400010F022F94EF200202B460A220121C2F2FC
:10C65000000010F09FF943F25C400121C0F202009B
:10C660000FF074FA4EF200202B460A220F21C2F27C
:10C67000000010F08FF943F238700321C0F202007D
:10C680000FF064FA204616F09BF8014620460FF0A2
:10C690005DFA43F240200121C0F202000FF056FA89
:10C6A0004EF20020C2F2000010F062F90423337051
:10C6B0000CB0BDE8F08106ACACE45B2301220321A1
:10C6C00006956560A560E560256125758DF81830D3
:10C6D0000CF01EFB204616F073F8024640F65C7024
:10C6E0002146C2F2010010F0CFF84EF200202B4696
:10C6F0000A220121C2F2000010F04CF943F25C4022
:10C700000121C0F202000FF021FA4EF200202B4668
:10C710000A220321C2F2000010F03CF943F2387003
:10C720000321C0F202000FF011FA204616F048F87B
:10C73000014620460FF00AFA43F240200121C0F2E0
:10C7400002000FF003FA4EF20020C2F2000010F0D7
:10C750000FF940F65C705D230695C2F2010065603A
:10C76000A560E56025612575012206218DF8183048
:10C77000B6E65B232A46082106956560A560E5605C
:10C78000256125758DF818300CF0C2FA204616F098
:10C7900017F8024640F65C702146C2F2010010F024
:10C7A00073F84EF200202B460A222946C2F20000FE
:10C7B00010F0F0F843F25C400121C0F202000FF0EB
:10C7C000C5F94EF200202B460A220821C2F20000D1
:10C7D00010F0E0F843F238700321C0F202000FF0CD
:10C7E000B5F9204615F0ECFF014620460FF0AEF9F2
:10C7F00043F240200121C0F202000FF0A7F94EF2EF
:10C800000020C2F2000010F0B3F840F65C705D2327
:10C810000695C2F201006560A560E5602561257599
:10C820002A460D218DF81830B4E55B2301220C2136
:10C8300006956560A560E560256125758DF8183061
:10C840000CF066FA204615F0BBFF024640F65C701D
:10C850002146C2F2010010F017F84EF200202B46DC
:10C860000A220121C2F2000010F094F843F25C4069
:10C870000121C0F202000FF069F94EF200202B46B0
:10C880000A220C21C2F2000010F084F843F2387042
:10C890000321C0F202000FF059F9204615F090FF75
:10C8A000014620460FF052F943F240200121C0F228
:10C8B00002000FF04BF94EF20020C2F2000010F01F
:10C8C00057F840F65C705D230695C2F20100656082
:10C8D000A560E5602561257501220F218DF81830CE
:10C8E000A3E600BF2DE9F04F2DED068B48F29047EF
:10C8F000C2F2010789B041F260023B680493C2F2C0
:10C900000102049B116840F6B7325B1A934207D9C3
:10C910004FF61143C2F200031B78002B40F0488110
:10C9200040F6C848C2F2010840F66C733A680592B6
:10C93000C2F2010341F287321968059B5B1A9342E8
:10C9400008D94DF68663C2F200031A78911E0129B8
:10C9500040F2E28040F6C844C2F2010440F6CC53F3
:10C960004FF618464BF6836A04F10C02C2F201033B
:10C970009FEDD08A9FEDD09ADFEDD08A9FEDD0AAAF
:10C98000DFEDD09ACDF80480C2F200060093C2F623
:10C99000A07A0025904603EB051B58460CF022F8C0
:10C9A00058465FFA85F90CF063F838B13B68069396
:10C9B00040F6B053C2F20103069A1A6058460CF0D2
:10C9C0004DF8A0B340F6B0533A680792C2F20103A3
:10C9D0001A68079B9B1AB3F5FA7F00F223814FF682
:10C9E0001143C2F20003B9F1010F1B7800F0D580AA
:10C9F000012B00F07284C0F01183022B00F08784B9
:10CA0000AB4643F6C8100721C0F202000FF09EF8B3
:10CA10004EF200205946C2F2000000230A220FF015
:10CA2000B9FF4EF20020C2F200000FF0A1FF237CFC
:10CA3000012B40F2498172B6E36862B6002B56F8CA
:10CA4000042BB8BF0333B2EBA30F5CD0B9F1010FD5
:10CA50006DD14FF61142C2F200021378012B00F0A3
:10CA6000AE82C0F06983032B00F0FA81042B0FD152
:10CA70004DF68663C2F200031B78072B00F0E986AF
:10CA8000082B00F0CB84062B00F05387FFF710F93A
:10CA900043F614300821C0F202000FF057F84EF2AE
:10CAA000002000230A222946C2F200000FF072FF84
:10CAB00043F2F860C0F2020002210FF047F8237C35
:10CAC000012B40F2068372B6E16862B60029B8BF56
:10CAD00003314EF200208910C2F200000FF0EAFE8E
:10CAE0004EF20020C2F200000FF042FF237C012B27
:10CAF00040F2C48272B6E36862B6002BB8BF03335B
:10CB00009B1046F8043C0135022D04F1140408F191
:10CB1000140807D0009B3EE7032A40F00081012261
:10CB20001A7017E709B0BDEC068BBDE8F08F4FF621
:10CB30001143C2F200031B78012B40F2F380022B59
:10CB4000A6D1237C012B40F2D28772B6E36862B68D
:10CB5000032B40F35185237C012B41F2508072B6A8
:10CB6000E36862B63F2B03DD72B64023E36062B632
:10CB7000237C012B40F28F8772B6E36862B64DF6D4
:10CB80008862002BC2F20002B8BF03339B101374FB
:10CB9000F9F754FFFEF7F2FE7AE7002B00F0298246
:10CBA000033B012B4FF0040140F23883CB4628E7CA
:10CBB000033B012B7FF6B4AE4DF68863C2F200034F
:10CBC00093ED027ADFED3B6ADFED3B7A9FED3B6A46
:10CBD00027EE267A27EE277AC7EE267A77EE867A30
:10CBE000FDEEE77A17EE903A9B0072B640F6C84821
:10CBF000C2F20108C8F80C3062B698F81030012B68
:10CC000040F2388372B6D8F80C3062B64FF618424C
:10CC1000002BC2F20002B8BF03339B101360FDF774
:10CC200001FD81E643F69C102921C0F202000EF0BE
:10CC30008DFF4EF2002000230A222946C2F2000096
:10CC40000FF0A8FE4EF20020C2F200000FF090FE9E
:10CC5000B9F1010FAB467FF4D4AE4FF61143C2F2E7
:10CC600000031B78032B00F0FC84042B00F0DA8413
:10CC7000002B7FF4C6AE4DF6866240F6ED53C2F24D
:10CC80000002C2F20103042111701B7872B69B00EE
:10CC9000E36062B6237C012B41F2158372B6E36830
:10CCA00062B6002BB8BF03339B103360FEF762FA05
:10CCB000A7E600BF0000C84200002C4200000000B0
:10CCC00000000C4200FEFF4672B694E80C0010789B
:10CCD0001978637A227A194202EA000200F0B780DA
:10CCE000A37A03F003030AB143F0040343F00803FB
:10CCF0009A10082BA27200F21482072B80F0348362
:10CD0000032B00F0368340F2AF81042B00F0B28198
:10CD1000062B7FF491AEE368023BE3608DE60022D0
:10CD20001A7017E6237C012B40F2898672B6E368FD
:10CD300062B6032B40F36684237C012B40F28B8781
:10CD400072B6E36862B6AB2B03DD72B6AC23E36068
:10CD500062B6237C012B40F2228772B6E36862B68A
:10CD6000002B227CB8BF03339B10012A46F8043CF9
:10CD700040F2E98672B6E36862B6002BB8BF0333AF
:10CD80009A10642303FB02F38AFB0312DB17C3EB45
:10CD9000E20307EE903AF8EEE77A4DF6886387EE05
:10CDA000887AC2F2000340F63459C2F2010943F610
:10CDB000D01014221C21C0F20200A9F80420029312
:10CDC000D3ED027A77EE677AF3EE046A87EEA67AFD
:10CDD00089ED007A0EF0BAFE029B986814F0CAFC46
:10CDE00041EC100B4EF200200521C2F200000FF0C2
:10CDF00011FE43F6F0100E21C0F202000EF0A6FE66
:10CE00004EF20020B9F80410C2F200000FF052FDFB
:10CE100043F600200E21C0F202000EF097FED9F872
:10CE2000000014F0A7FC41EC100B4EF2002005218D
:10CE3000C2F200000FF0EEFD4EF20020C2F2000040
:10CE40000FF096FDF9F7FAFDFDF7CEF920E6A37A8B
:10CE500003F00303002A3FF44BAF43F0040347E71A
:10CE60004DF68663C2F200031B78042B00F0208489
:10CE7000052B40F0A180237C012B41F2E68272B6A3
:10CE8000E36862B6032B40F3E887237C012B41F271
:10CE9000AB8472B6E36862B6B3F5C87F04DB72B6E2
:10CEA0004FF4C873E36062B6237C012B41F2A18288
:10CEB00072B6E36862B6002B227CB8BF03339B10C6
:10CEC000012A46F8043C41F2688272B6E36862B611
:10CED0004FF61042002B217CB8BF0333C2F2000290
:10CEE0009B100129137041F2528272B6E36862B658
:10CEF000002BB8BF03339B1007EE903AB8EEE77AE9
:10CF000040F6645BC7EE087AC2F2010B40F2C42916
:10CF1000DBF80030C2F2010943F67020142223210D
:10CF2000C0F20200A9F80420B7EE007A37EE677A63
:10CF3000D3ED497A77EE677AF3EE046A87EEA67A44
:10CF400089ED007A0EF002FEDBF80030D3F8240100
:10CF500014F010FC41EC100B4EF200200521C2F23F
:10CF600000000FF057FD43F694201521C0F2020097
:10CF70000EF0ECFD4EF20020B9F80410C2F20000F1
:10CF80000FF098FC43F6AC20C0F2020015210EF021
:10CF9000DDFDD9F8000014F0EDFB41EC100B4EF272
:10CFA0000020C2F2000005210FF034FD4EF20020F7
:10CFB000C2F200000FF0DCFCFEF7DCF868E54DF68D
:10CFC000886340F65C70C2F200030021C2F20100E7
:10CFD0000293039311700BF0DFFE029B5B7972B634
:10CFE000019A9B00136262B6F9F728FDFDF71AFB60
:10CFF0004EE54DF68662C2F200021378012B00F076
:10D000001484C0F0E182022B00F0DE82032B00F0DA
:10D010000C84FDF707FB4FF0010BF2E44DF688633B
:10D02000C2F2000393ED027A27EE087A27EE097A1E
:10D03000C7EE087A77EEA87AFDEEE77A17EE903A17
:10D040009B0072B6E36062B6237C012B40F210872E
:10D0500072B6E36862B6002BB8BF03339B1033602F
:10D06000AB46FDF7C1F8CCE4012B00F07D81022B2B
:10D070007FF4E2ACE368013BE360DEE472B694E87F
:10D080000C0010781978637A227A194202EA0002B9
:10D0900000F09680A37A03F003030AB143F004037F
:10D0A00043F008039A10082BA27200F2A880072B05
:10D0B00080F0AF81032B00F0B08240F26681042B38
:10D0C00000F0A880062B7FF416ADE368023BE36016
:10D0D00012E572B694E80C0010781978637A227A17
:10D0E000194202EA000274D0A37A03F003030AB1E2
:10D0F00043F0040343F008039A10082BA27270D87F
:10D10000072B80F07B81032B00F0828240F2368176
:10D11000042B70D0062B7FF4D7ACE1680239E160B4
:10D12000D3E40C2B00F0258100F21881092B3FF489
:10D13000F2AD0B2B9ED07FE44DF68663C2F2000366
:10D140001A78012A00F05785C0F0FB81022A00F00E
:10D15000FA81032A31D1237C012B40F2B18772B6C8
:10D16000E36862B6032B40F31586237C012B41F262
:10D17000A38272B6E36862B67F2B4DF68863C2F273
:10D18000000307DD1A79622A41F2A68172B67C2279
:10D19000E26062B6227C012A40F2BC8772B6E26885
:10D1A00062B6002AB8BF0332C2F38702114618796B
:10D1B0005A7103F0FDFCF9F741FCFDF733FA67E41F
:10D1C000A37A03F00303002A3FF46CAF43F0040397
:10D1D00068E7A37A03F00303002A8DD043F0040329
:10D1E0008AE70C2B00F0148200F20281092B94D004
:10D1F0000B2B7FF469ACE1680139E16065E40C2B2D
:10D2000000F00B8200F2FF80092B3FF45EAF0B2B86
:10D210007FF471ACE368013BE3606DE44DF6866337
:10D22000C2F200031A78062A00F0558500F2BD808C
:10D23000042A00F05785052A40F0F38240F6ED52AB
:10D24000C2F201021970137872B69B00E36062B6F5
:10D25000237C012B41F25B8272B6E36862B6002B3D
:10D26000B8BF03339B1033604FF0010BFDF782FF13
:10D27000FFF7C7BB72B6D8F80030D8F804101A7898
:10D28000087898F8091098F80830084202EA030272
:10D2900000F0828098F80A3003F003030AB143F0EB
:10D2A000040343F008039A10082B88F80A2000F2C0
:10D2B0008D82072B80F00185032B00F0058540F25D
:10D2C0003585042B00F08D82062B7FF49CACD8F8BA
:10D2D0000C30023BC8F80C3097E44DF68863C2F27C
:10D2E00000031B7C72B69B00E36062B6237C012BBB
:10D2F00040F2218672B6E36862B6002BB8BF0333F2
:10D300009B103360AB46FEF739FBFFF77ABB4DF657
:10D310008863C2F2000393ED027A27EE087A27EEC3
:10D32000097AC7EE087A77EEA87AFDEEE77A17EE6B
:10D33000903A9B0072B6E36062B6237C012B40F208
:10D34000CD8572B6E36862B6002BB8BF03339B107D
:10D350003360AB46FDF766F9FFF753BB0D2B3FF487
:10D3600089AE0E2B7FF468ABE3680133E360FFF70F
:10D3700064BBE3680233E360FFF75FBB012B3DD082
:10D38000022B3FF438AFFFF79FBB012B41D0022B9C
:10D390003FF440AFFFF7AFBB98F80A3003F0030348
:10D3A000002A80D043F004037DE7072A00F02082A2
:10D3B000082A40F0368240F24012C2F201020621F1
:10D3C0001278197072B69300E36062B6237C012B69
:10D3D00041F2808172B6E36862B6002BB8BF0333B6
:10D3E0009B1033604FF0010BFEF762FCFFF709BBA7
:10D3F0000D2B3FF400AF0E2B7FF466ABE1680131DB
:10D40000E160FFF762BB0D2B3FF404AF0E2B7FF4FE
:10D4100072ABE3680133E360FFF76EBB237C012B43
:10D4200041F2CC8172B6E36862B6032B40F3DE852D
:10D43000237C012B41F2308272B6E36862B6CB2BBB
:10D4400003DD72B6C823E36062B6237C012B41F290
:10D45000AF8172B6E36862B6002BB8BF0333C3F383
:10D46000870307EE903A9FED907AF8EE676A40F6F0
:10D470007079C6EE877AC2F2010989F80030B7EEFA
:10D48000007A77EEA87A37EE677AB4EEE97AF1EEB1
:10D4900010FA00F33B84DFED826AB4EEE67AF1EE37
:10D4A00010FA00F1F585F0EE476AFEEEC86A16EE56
:10D4B000903A40F69042C2F20102F4EEE97AF1EEBF
:10D4C00010FA936100F31D849FED757AF4EEC77A2C
:10D4D000F1EE10FA00F1EA85B0EE677ABEEEC87A96
:10D4E00017EE103AF4EEE97AF1EE10FAD36101F397
:10D4F0009E849FED6B7AF4EEC77AF1EE10FA00F19C
:10D50000D085B0EE677ABEEEC87A17EE103A43F6D1
:10D51000F8201921C0F2020013620EF017FB4EF240
:10D52000002099F8001000230A22C2F200000FF038
:10D5300031FA4EF20020C2F200000FF019FAFFF7A4
:10D54000A5BA02221A70237C012B40F2388672B6EB
:10D55000E36862B6032B40F32A8440F6C859237C63
:10D56000C2F20109012B99F800B041F2F68072B6BF
:10D57000E36862B6002BB8BF0333BBEBA30F06DC36
:10D5800099F80030013B9B0072B6E36062B6237CE1
:10D59000012B40F2EA8572B6E36862B61A1EB8BF84
:10D5A00003324DF68863C2F38702C2F200031046CD
:10D5B0001A71029303F014F8029B5979187903F059
:10D5C000F7FAF9F73BFAF8E54DF68863C2F2000383
:10D5D00001215B79117072B69B00E36062B6237C17
:10D5E0008B4240F2318172B6E36862B6002BB8BF5D
:10D5F00003339B1033600CE572B60023E36062B620
:10D60000FFF7B6BA72B60023E36062B6FFF7A1BBBC
:10D61000E1680231E160FFF758BAE3680233E36082
:10D62000FFF76ABA4DF686624DF68863C2F20002D1
:10D63000C2F2000382F800905B7972B69B00E3604F
:10D6400062B6237C012B40F2118672B6E36862B6A3
:10D65000002BB8BF03339B103360FCF7E3FFFFF7E9
:10D66000D0B94DF6866240F24013C2F20002C2F217
:10D670000103062111701B7872B69B00E36062B64D
:10D68000237C012B40F2C58572B6E36862B6002B9D
:10D69000B8BF03339B103360FEF70AFBFFF7B1B945
:10D6A00000FEFFC6000096440000484279783042F0
:10D6B000237C012B40F23F8672B6E36862B6032BEF
:10D6C00040F3D183237C012B41F24D8072B6E36895
:10D6D00062B6B3F5C87F04DB72B64FF4C873E3607B
:10D6E00062B6237C012B40F2788772B6E36862B69B
:10D6F000002B227CB8BF03339B10012A46F8043C60
:10D7000040F2138772B6E36862B640F6ED52002B22
:10D71000217CB8BF0333C2F201029B1001291370B0
:10D7200040F22F8772B6E36862B6002BB8BF0333AE
:10D730009B1007EE903AF8EEE77A40F6645B87EECE
:10D74000887AC2F2010B40F23819DBF80030C2F2DD
:10D75000010943F6102014222621C0F20200A9F884
:10D760000420F7EE007A37EEC77AD3ED4A7A77EEE7
:10D77000677AF3EE046A87EEA67A89ED007A0EF0F6
:10D78000E5F9DBF80030D3F8280113F0F3FF41ECA2
:10D79000100B4EF200200521C2F200000FF03AF902
:10D7A00043F638201821C0F202000EF0CFF94EF2F5
:10D7B0000020B9F80410C2F200000FF07BF843F625
:10D7C0005420C0F202001821FFF7E1BB0C2B00F03F
:10D7D0007B8200F26C82092B3FF479AD0B2B7FF436
:10D7E00012AAD8F80C30013BC8F80C30FFF70DBA7C
:10D7F00040F67072C2F2010208211278197072B6F6
:10D800009300E36062B6237C012B41F27F8172B604
:10D81000E36862B6002BB8BF03339B103360FEF79A
:10D8200047FA4FF0010BFFF7ECB84DF68863C2F2F0
:10D83000000300211B79117072B69B00E36062B691
:10D84000237C012B3FF6CFAE72B62046FCF75AFC84
:10D85000CAE6237C012B40F28C8772B6E36862B67D
:10D86000032B40F3CD83237C012B41F23D8072B624
:10D87000E36862B68F2B03DD72B68C23E36062B679
:10D88000237C012B40F28E8772B6E36862B6002BD0
:10D89000B8BF0333C3F3870307EE903AB8EE677A55
:10D8A00040F6EC59C7EE0A7AC2F2010989F8003055
:10D8B00077EEA87AF4EEE97AF1EE10FA00F31D8221
:10D8C0001FED897AF4EEC77AF1EE10FA00F1E583E4
:10D8D000B0EE677ABEEEC87A17EE103A40F65842BC
:10D8E000C2F2010243F6DC201B21C0F20200D36128
:10D8F0000EF02CF999F8003007EE903AF8EE677ABE
:10D9000087EE8A7A77EE287A17EE900A13F032FFC4
:10D9100041EC100B4EF200200221C2F200000FF089
:10D9200079F84EF20020C2F200000FF021F8FFF764
:10D93000ADB8237C012B40F22F8772B6E36862B644
:10D94000032B40F34E83237C012B40F2DC8772B61D
:10D95000E36862B6CB2B03DD72B6C823E36062B620
:10D96000237C012B40F2128772B6E36862B6002B6B
:10D97000B8BF0333C3F3870307EE903AB8EE677A74
:10D980005FEDB87A5FEDB86A67EE277A40F240192A
:10D9900087EEA67AC2F2010989F8003077EE287A7C
:10D9A000F5EEC07AF1EE10FA00F126835FEDC16A60
:10D9B000B6EE007AA7EEA67A4FF4FC53C0F201034C
:10D9C000FCEEC77A17EE90EA9E4540F274839E46BD
:10D9D0004FF4107040F2F423C2F201031A7ED10713
:10D9E00000F19981D98BC3F820E0814242F0010215
:10D9F00038BFD8831A7643F6C4201721C0F202003C
:10DA00000EF0A4F899F800104FF4966348F21F52F4
:10DA100003FB01F3C5F2EB1282FB03124EF200206E
:10DA2000D917C1EB2211C2F200000EF043FF4EF2F3
:10DA30000020C2F200000EF09BFFFFF727B872B67D
:10DA400094E80C0010781978637A227A194202EA75
:10DA5000000200F08481A37A03F003030AB143F0CB
:10DA6000040343F008039A10082BA27200F2A58168
:10DA7000072B80F02785032B00F0528540F2148697
:10DA8000042B00F0A581062B7FF451A9E368023B2B
:10DA9000E360FFF74DB972B694E80C00107819787E
:10DAA000637A227A194202EA000200F04F81A37AD7
:10DAB00003F003030AB143F0040343F008039A1090
:10DAC000082BA27200F29981072B80F0F084032BBF
:10DAD00000F0BA8540F2F685042B00F09981062B00
:10DAE0007FF44BA8E368023BE360FFF747B872B6E8
:10DAF00094E80C0010781978637A227A194202EAC5
:10DB0000000200F03E81A37A03F003030AB143F060
:10DB1000040343F008039A10082BA27200F27D81DF
:10DB2000072B80F0F384032B00F0E58440F2058698
:10DB3000042B00F07D81062B7FF408A8E368023BEC
:10DB4000E360FFF704B872B694E80C001078197817
:10DB5000637A227A194202EA000200F00981A37A6C
:10DB600003F003030AB143F0040343F008039A10DF
:10DB7000082BA27200F23181072B80F06085032B05
:10DB800000F0A58440F2AC85042B00F03181062B17
:10DB90007FF4F1A8E368023BE360FFF7EDB872B6EB
:10DBA00094E80C0010781978637A227A194202EA14
:10DBB000000200F0C280A37A03F00303002A41F0C0
:10DBC0003B8143F008039A10082BA27200F23581C2
:10DBD000072B80F0AB83032B00F09D8440F2B585CA
:10DBE000042B00F03581062B7FF4B8A8E368023BD4
:10DBF000E360FFF7B4B803221A70FFF7ACBA72B64D
:10DC000094E80C0010781978637A227A194202EAB3
:10DC1000000200F0BD81A37A03F003030AB143F0D0
:10DC2000040343F008039A10082BA27200F2B98192
:10DC3000072B80F0E585032B00F0E78540F2FC859B
:10DC4000042B00F0B981062B7EF48AAFE368023B17
:10DC5000E360FEF786BF72B694E80C00107819787E
:10DC6000637A227A194202EA000200F02E81A37A36
:10DC700003F003030AB143F0040343F008039A10CE
:10DC8000082BA27200F29D81072B80F0A385032B45
:10DC900000F0A58540F2D785042B00F09D81062B6E
:10DCA0007FF44FA8E368023BE360FFF74BB80D2B0E
:10DCB0003FF497AD0E2B7EF4A6AFD8F80C300133AD
:10DCC000C8F80C30FEF7A1BFD8F80C300233C8F802
:10DCD0000C30FEF79ABF40F6EC52C2F20102072167
:10DCE000FFF76EBB4FF61042C2F200020521127818
:10DCF000197072B69300FFF7A9BA0023C7F6FF7335
:10DD0000ECE50023C7F6FF73D36100E40023C7F6F8
:10DD1000FF73FFF7CEBB196A8E4540F27681DA8B2E
:10DD2000C3F820E0824238BFD88364E6012BC4D018
:10DD3000022B3FF456ADFEF766BFA37A03F0030350
:10DD4000002A3FF440AF43F004033CE7A37A03F01A
:10DD50000303002A3FF4B3AE43F00403AFE6A37A13
:10DD600003F00303002A3FF47EAE43F004037AE697
:10DD7000A37A03F00303002A3FF4F9AE43F004034F
:10DD8000F5E6A37A03F00303002A3FF4C4AE43F0A0
:10DD90000403C0E64DF68863C2F200031A79002A34
:10DDA00040F0ED8472B6E26062B6FFF7F3B972B686
:10DDB0000023E36062B6FFF7EABB0C2B00F0B083F0
:10DDC00000F27A83092B3FF461AE0B2B7EF4AFAFE8
:10DDD000E368013BE360FEF7ABBF0C2B00F07783F9
:10DDE00000F22784092B3FF4D5AE0B2B7EF4C3AF92
:10DDF000E368013BE360FEF7BFBF0C2B00F0248417
:10DE000000F24F83092B3FF46DAE0B2B7EF4B5AEC1
:10DE1000E368013BE360FEF7B1BE0C2B00F06B83BF
:10DE200000F26E83092B3FF489AE0B2B7EF48EAE8D
:10DE3000E368013BE360FEF78ABE0C2B00F06B83C6
:10DE400000F26E82092B3FF4D1AE0B2B7EF486AF2D
:10DE5000E368013BE360FEF782BF72B60023E36034
:10DE600062B6FFF721B872B60023E36062B638E409
:10DE700072B658F80C2C636810781978637A227A95
:10DE8000194202EA000200F0ED83A37A03F00303D3
:10DE9000002A40F0E58743F008039A10082BA2728D
:10DEA00000F2F283072B80F05586032B00F03B86AF
:10DEB00040F23286042B00F0F283062B7FF4C9A8CF
:10DEC000E368023BE360FFF7C5B8A37A03F00303FE
:10DED000002A3FF4D4AE43F00403D0E672B658F8FB
:10DEE0000C2C636810781978637A227A194202EA56
:10DEF000000200F0AE83A37A03F003030AB143F0FB
:10DF0000040343F008039A10082BA27200F2058460
:10DF1000072B80F04186032B00F0338640F22A86DF
:10DF2000042B00F00584062B7FF40CAAE368023B67
:10DF3000E360FFF708BA72B658F80C2C63681078E3
:10DF40001978637A227A194202EA000200F0938378
:10DF5000A37A03F003030AB143F0040343F0080378
:10DF60009A10082BA27200F2C283072B80F0FD8565
:10DF7000032B00F0E48540F2DB85042B00F0C28324
:10DF8000062B7FF4B8A9E368023BE360FFF7B4B95E
:10DF9000A37A03F00303002A3FF445AE43F00403E1
:10DFA00041E60C2B00F0318400F22484092B3FF46D
:10DFB0004DAE0B2B7EF4D4ADE368013BE360FEF77E
:10DFC000D0BD0C2B00F00B8400F2FE83092B3FF434
:10DFD00069AE0B2B7EF4B5AEE368013BE360FEF760
:10DFE000B1BE72B60023E36062B6B9E472B6002334
:10DFF000E36062B6FFF729BA01204FF0000EE9E4B2
:10E0000072B60023E36062B63AE49107C3F820E0F9
:10E0100006D5596A7F31C9090131884238BF08469F
:10E02000510706D5996A7F31C9090131884238BF45
:10E030000846110706D5D96A7F31C90901318842DE
:10E0400038BF0846D10606D5196B7F31C9090131A1
:10E05000884238BF0846910606D5596B7F31C909F9
:10E060000131884238BF0846510606D5996B7F3189
:10E07000C9090131884238BF0846D20906D0DA6B97
:10E080007F32D2090132904238BF1046D883B2E4C1
:10E090000023C8F20103FFF70CBA0023C8F2010302
:10E0A0001CE40023C8F20103FFF731BA0023C8F2D1
:10E0B0000103FFF717BA0EF17F00C009013089E4B0
:10E0C00072B694E80C0010781978637A227A1942B3
:10E0D00002EA000240F0BE83A37A03F00303002AA1
:10E0E00040F0C2869A10082BA27200F21284072B0D
:10E0F00080F01086032B00F0DC8540F2D385042BE2
:10E1000000F01284062B7FF42BA8E368023BE36047
:10E11000FFF727B872B694E8060091F800E010788F
:10E12000627A217A10420EEA010140F07383A27AEA
:10E1300002F00302002940F083869110082AA172A0
:10E1400000F2F783072A80F0CF85032A00F0358696
:10E1500040F22C86042A00F0F783062A7FF41FA8D9
:10E16000E268023AE260FFF71BB872B694E80C006E
:10E1700010781978637A227A194202EA000240F094
:10E180005283A37A03F00303002A40F05D869A10BD
:10E19000082BA27200F27083072B80F07285032B8C
:10E1A00000F07B8540F27285042B00F07083062B13
:10E1B0007FF4F2A9E368023BE360FFF7EEB972B6C1
:10E1C00094E80C0010781978637A227A194202EAEE
:10E1D000000240F04883A37A03F00303002A40F0D2
:10E1E00047869A10082BA27200F26E83072B80F0EC
:10E1F000B185032B00F0238540F21985042B00F034
:10E200006E83062B7FF4A4A9E368023BE360FFF76B
:10E21000A0B972B658F80C2C636810781978637A34
:10E22000227A194202EA000200F04583A37A03F041
:10E2300003030AB143F0040343F008039A10082BC8
:10E24000A27200F22384072B80F0C084032B00F01D
:10E25000C98440F2C084042B00F02384062B7FF491
:10E2600014AAE368023BE360FFF710BA72B658F8ED
:10E270000C2C636810781978637A227A194202EAC2
:10E28000000200F00F83A37A03F003030AB143F006
:10E29000040343F008039A10082BA27200F2CD8306
:10E2A000072B80F07385032B00F0658540F25C85B9
:10E2B000042B00F0CD83062B7FF4C8A9E368023B52
:10E2C000E360FFF7C4B972B658F80C2C6368107895
:10E2D0001978637A227A194202EA000200F00A836E
:10E2E000A37A03F003030AB143F0040343F00803E5
:10E2F0009A10082BA27200F24583072B80F0AA84A3
:10E30000032B00F0B38440F2AA84042B00F0458371
:10E31000062B7EF4C4ACE368023BE360FEF7C0BCAE
:10E320000D2B3FF495AD0E2B7EF418ADE368013351
:10E33000E360FEF714BD72B694E80C00107819780B
:10E34000637A227A194202EA000200F0BF83A37ABC
:10E3500003F00303002A40F07B8543F008039A1082
:10E36000082BA27200F2A283072B80F04684032BB5
:10E3700000F0F58440F22685042B00F0A283062BE2
:10E380007FF49BA9E368023BE360FFF797B972B69D
:10E390002046FBF7B7FEFEF7A9BD72B694E80C0065
:10E3A00010781978637A227A194202EA000200F0A2
:10E3B000D082A37A03F00303002A40F04D8543F096
:10E3C00008039A10082BA27200F2CC82072B80F06F
:10E3D0007B84032B00F07D8440F20A85042B00F03F
:10E3E000CC82062B7EF472ADE368023BE360FEF75D
:10E3F0006EBD72B694E80C0010781978637A227AB0
:10E40000194202EA000200F03883A37A03F0030302
:10E410000AB143F0040343F008039A10082BA272D8
:10E4200000F21B83072B80F08584032B00F0878488
:10E4300040F2D084042B00F01B83062B7EF439AD10
:10E44000E368023BE360FEF735BD72B694E80C006A
:10E4500010781978637A227A194202EA000200F0F1
:10E46000E382A37A03F003030AB143F0040343F009
:10E4700008039A10082BA27200F2C682072B80F0C4
:10E480003E84032B00F04B8440F2AB84042B00F05D
:10E49000C682062B7EF4F4ACE368023BE360FEF731
:10E4A000F0BC0D2B3FF4B4AC0E2B7EF466ABE368EE
:10E4B0000133E360FEF762BB0D2B3FF489AC0E2BFA
:10E4C0007EF435ACE3680133E360FEF731BCE3680A
:10E4D0000233E360FEF750BC72B60022E26062B61F
:10E4E0001A790132D2B210461A71029302F078F80A
:10E4F000029BFEF74FBEE3680233E360FEF727BBE3
:10E500000D2B3FF495AC0E2B7EF420ABE36801336A
:10E51000E360FEF71CBBE3680233E360FEF71FBC59
:10E52000E3680233E360FEF703BC72B694E80C00C4
:10E5300010781978637A227A194202EA000200F010
:10E54000CE82A37A03F003030AB143F0040343F03D
:10E5500008039A10082BA27200F22482072B80F085
:10E560005783032B00F0598340F25184042B00F0B1
:10E570002482062B7FF4C7A8E368023BE360FFF721
:10E58000C3B872B694E80C0010781978637A227ACE
:10E59000194202EA000200F02E82A37A03F003037C
:10E5A0000AB143F0040343F008039A10082BA27247
:10E5B00000F29E82072B80F0FE82032B00F0F18296
:10E5C00040F22D84042B00F09C82062B7FF4ABA834
:10E5D000E368023BE360FFF7A7B872B694E80C006B
:10E5E00010781978637A227A194202EA000200F060
:10E5F000F981A37A03F003030AB143F0040343F063
:10E6000008039A10082BA27200F2DC81072B80F01D
:10E61000C883032B00F0068340F2F283042B00F042
:10E62000DC81062B7FF462A8E368023BE360FFF71E
:10E630005EB80D2B3FF4DCAB0E2B7EF49CABE36895
:10E640000133E360FEF798BBE3680233E360FEF753
:10E6500095BAA37A03F00303002A3FF454AC43F0C5
:10E66000040350E4A37A03F00303002A3FF415AC3B
:10E6700043F0040311E4A37A03F00303002A3FF4F8
:10E680006FAC43F004036BE40C2B00F04C8200F2FF
:10E690005B82092B3FF414AC0B2B7EF4DAACE368FD
:10E6A000013BE360FEF7D6BC012B3FF40BAF022B1E
:10E6B0003FF48EABFEF73BBB72B62046FBF722FD64
:10E6C000FEF758BD012B3FF4F2AE022B3FF4A0AB96
:10E6D000FEF753BA72B62046FBF714FDFEF77BBE79
:10E6E000012BACD0022B3FF483ABFEF744BB0C2BC9
:10E6F00000F0258200F23382092B3FF444AC0B2B4F
:10E700007EF4F9ADE368013BE360FEF7F5BD72B658
:10E710002046FBF7F7FCFEF7A0BD0C2B00F0318282
:10E7200000F23482092B3FF401AC0B2B7EF40AAECD
:10E73000E368013BE360FEF706BE012B3FF4E6AE63
:10E74000022B3FF475ABFEF701BA012B3FF4EEAD9F
:10E75000022B3FF47DABFEF701BB72B62046FBF700
:10E76000D1FCFEF705BF72B62046FBF7CBFCFEF7E7
:10E77000AEBF72B62046FBF7C5FCFFF76FB872B6A6
:10E780007C22E26062B61A79013AABE672B62046A4
:10E79000FBF7B8FCFFF7E9B872B62046FBF7B2FC0E
:10E7A000FFF7CCB872B62046FBF7ACFCFFF76DB8AC
:10E7B00072B62046FBF7A6FCFEF74CBE72B62046AA
:10E7C000FBF7A0FCFEF72FBE0D2B3FF405AC0E2B84
:10E7D0007EF4B7AAE3680133E360FEF7B3BAE368F7
:10E7E0000233E360FEF7AEBA72B62046FBF78AFC4E
:10E7F000FEF750BB0D2B3FF4DFAB0E2B7EF4B0A920
:10E80000E3680133E360FEF7ACB9E3680233E36029
:10E81000FEF7A7B9A27A02F0030209B142F004029E
:10E8200042F0080289E4A37A03F003030AB143F03B
:10E83000040343F00803AAE4012BE1D0022B3FF4C8
:10E84000BBABFEF78DB9012BC4D0022B3FF4C4AB98
:10E85000FEF777BAA37A03F003030AB143F0040387
:10E8600043F008033EE4A37A03F003030AB143F044
:10E87000040343F00803B4E40C2B00F00E8200F212
:10E88000FA81092B3FF496AC0B2B7EF485AEE3683E
:10E89000013BE360FEF781BE72B62046FBF732FC17
:10E8A000FEF7CBBDA37A03F00303002A3FF4F3ACD9
:10E8B00043F00403EFE4A37A03F00303002A3FF4D8
:10E8C000BDAC43F00403B9E40C2B00F0B88100F2B6
:10E8D0003B82092B3FF498AC0B2B7EF439AEE368F6
:10E8E000013BE360FEF735BE72B62046FBF70AFC3B
:10E8F000FEF7BEBFA37A03F00303002A3FF4F8AC8F
:10E9000043F00403F4E472B62046FBF7FBFBFFF789
:10E910001FB80C2B00F0CD8100F2F681092B3FF4DB
:10E92000F4AB0B2B7EF41CACE368013BE360FEF719
:10E9300018BC0C2A00F0418200F2D081092A3FF471
:10E940000FAC0B2A7EF42BACE268013AE260FEF7D2
:10E9500027BCA37A03F00303002A3FF432AD43F04F
:10E9600004032EE50C2B00F0B48100F2A781092BE3
:10E970003FF43AAD0B2B7EF4A9AAE368013BE360B8
:10E98000FEF7A5BA0C2B00F0718100F25D81092B16
:10E990003FF4C1AC0B2B7EF482A9E368013BE3603A
:10E9A000FEF77EB90C2B00F0388100F22B81092B89
:10E9B0003FF4E2AD0B2B7EF4A6AEE368013BE360CF
:10E9C000FEF7A2BE0C2B00F02D8100F2E481092B92
:10E9D0003FF42AAE0B2B7EF489AEE368013BE36083
:10E9E000FEF785BEA37A03F00303002A3FF409AEC5
:10E9F00043F0040305E6A37A03F00303002A3FF47F
:10EA0000D4AD43F00403D0E50C2B00F0888100F274
:10EA10007081092B3FF440AD0B2B7EF431AAE368E3
:10EA2000013BE360FEF72DBAA37A03F00303002A4B
:10EA30003FF41FAD43F004031BE50C2B00F09B815A
:10EA400000F29E81092B3FF439AC0B2B7EF4FEAD16
:10EA5000E368013BE360FEF7FABD0C2B00F06F8129
:10EA600000F26281092B3FF4EBAC0B2B7EF421AA60
:10EA7000E368013BE360FEF71DBAA37A03F00303EA
:10EA8000002A3FF4CAAC43F00403C6E40C2B00F0A8
:10EA9000A98000F29580092B3FF4E3AB0B2B7EF4A9
:10EAA000F4ADE368013BE360FEF7F0BD0C2B00F032
:10EAB000568100F29C80092B3FF464AC0B2B7EF452
:10EAC000FCADE368013BE360FEF7F8BDA37A03F019
:10EAD0000303002A3FF443AC43F004033FE4A37A6A
:10EAE00003F00303002A3FF434AD43F0040330E5A0
:10EAF0000C2B56D05AD8092B3FF46AAD0B2B7EF461
:10EB000012AEE368013BE360FEF70EBE72B620462C
:10EB1000FBF7F8FAFEF77CBE012B1BD0022B3FF46B
:10EB2000BEADFEF796BAE3680233E360FEF792BA31
:10EB3000012B1AD0022B3FF4E5ADFEF7DCBBE368F6
:10EB40000233E360FEF7D8BB0D2B3FF4A8AD0E2BCC
:10EB50007EF47FAAE3680133E360FEF77BBA0D2BF6
:10EB60003FF4D0AD0E2B7EF4C6ABE3680133E36017
:10EB7000FEF7C2BB012B0FD0022B3FF4D9ADFEF73D
:10EB8000E1BBE3680233E360FEF7DDBB0D2B3FF42E
:10EB9000CFAD0E2B7EF4D6ABE3680133E360FEF716
:10EBA000D2BBE3680233E360FEF7BEBD0D2BA8D0F5
:10EBB0000E2B7EF4B8ADE3680133E360FEF7B4BD1D
:10EBC0000D2B3FF46EAF0E2B7EF45FADE368013387
:10EBD000E360FEF75BBD012BF8D0022B3FF461AF81
:10EBE000FEF753BDE3680233E360FEF74FBD0D2B24
:10EBF0003FF467AF0E2B7EF460ADE3680133E36052
:10EC0000FEF75CBD0D2B3FF4D8AE0E2B7EF47BAD32
:10EC1000E3680133E360FEF777BDE3680233E36046
:10EC2000FEF772BDE3680233E360FEF760BD012BBF
:10EC300000F09080022B3FF452AEFEF789BCE368EF
:10EC40000233E360FEF785BC0D2B3FF4A6AE0E2B1E
:10EC50007EF425A8E3680133E360FEF721B8012BB9
:10EC6000F8D0022B3FF499AEFEF719B8E3680233EF
:10EC7000E360FEF715B80D2B3FF409AE0E2B7EF4C2
:10EC80008BACE3680133E360FEF787BC012BF8D05F
:10EC9000022B3FF4FCADFEF77FBCE3680233E36078
:10ECA000FEF77BBC012B35D0022B3FF43DAEFEF7C7
:10ECB00057BAE3680233E360FEF753BA0D2B3FF413
:10ECC0005CAE0E2B7EF402A9E3680133E360FEF72D
:10ECD000FEB8E3680233E360FEF7F9B80D2A3FF4AB
:10ECE00033AE0E2A7EF45BAAE2680132E260FEF7E0
:10ECF00057BA0D2B3FF493AE0E2B7EF4C1A8E368F8
:10ED00000133E360FEF7BDB80D2B3FF40DAE0E2BC3
:10ED10007EF426AAE3680133E360FEF722BAE368D3
:10ED20000233E360FEF7ADB80D2B3FF4A1AE0E2B1E
:10ED30007EF4BFA8E3680133E360FEF7BBB8E36885
:10ED40000233E360FEF7B6B80D2B3FF4C8AD0E2BCF
:10ED50007EF4FEABE3680133E360FEF7FABBE368E1
:10ED60000233E360FEF7AABC012B0FD0022B3FF465
:10ED70006FAEFEF76BBCE3680233E360FEF767BC7F
:10ED80000D2B3FF465AE0E2B7EF460ACE3680133CF
:10ED9000E360FEF75CBC0D2B3FF41FAE0E2B7EF440
:10EDA000A5ACE3680133E360FEF7A1BC012A9BD068
:10EDB000022A3FF4C9ADFEF7F2B9E2680232E2601E
:10EDC000FEF7EEB9012B3FF418AF022B3FF479AEFA
:10EDD000FEF773BC012BADD0022B3FF449AEFEF71A
:10EDE00068B8012B8BD0022B3FF419AEFEF748B860
:10EDF000012B3FF469AF022B3FF4BFADFEF766B8BD
:10EE0000012BCED0022B3FF4E8ADFEF76FBC012BF7
:10EE10003FF4FEAE022B3FF4D0ADFEF774BC012BE5
:10EE20003FF4C9AE022B3FF46CAEFEF77CBC00236E
:10EE3000C7F6FF73FEF76BBB43F00403FEF7C1BEDA
:10EE400042F00402FFF779B943F00403FFF79FB9DA
:10EE500043F00403FFF781BA43F00403FFF7AFBAAE
:10EE600043F00403FFF717B843F00403FFF73AB980
:10EE700043F00403FFF7B5B92DE9F0432DED028B04
:10EE80000446002683B000F1B405284684F89D604E
:10EE900084F89E6084F89F6084F8A06084F8A16084
:10EEA00084F8A26084F8A36084F8A46084F8A56064
:10EEB00084F8A66084F8A76084F8A86084F8A96044
:10EEC00084F8AA6084F8AB6084F8AC6084F8906041
:10EED00084F8916084F892600191FAF7ADFE43F6F0
:10EEE0002031AD22C0F2020104F598700AF0DAF880
:10EEF0000B2384F8DD3102F0C9FE02F017FF03F0A6
:10EF0000DDFBDDED017AB8EEE78AA046B0EE480AF7
:10EF100003F0D4F9B0EE480A03F01CFAB0EE480A48
:10EF200003F0F8FAB0EE480A02F0B2FC0199284664
:10EF3000FAF78AFE4FF409700DF088FE0546F1F7E6
:10EF40009FFAC4F820524FF409700DF07FFE42F68C
:10EF50007863C0F202030360C4F824024FF409701E
:10EF60000DF074FE43F6E063C0F20203C4F81C0225
:10EF7000036004F1840925464FF425700DF066FE08
:10EF800007460C3501F010FF45F8047C05F80A6CC3
:10EF900005F8096C05F8086CA9454FF00003EBD1A2
:10EFA00094F89D209FEDD26ADFEDD26A84F8DE31BD
:10EFB00007EE902AB8EEE77A94F89F20C4F88830DC
:10EFC00067EE067A0B2067EEA67A4FF40051FCEE4E
:10EFD000E77AC4F88C30CDED017A84F8963084F865
:10EFE000953084F8943084F8933084F8923084F823
:10EFF000913084F8903084F8DD019DF80430C4F835
:10F0000084100AB184F8903094F89E200AB184F8F4
:10F01000913094F8A0200AB184F8923094F8A53089
:10F020009FEDB36ADFEDB36A94F8A71007EE903A4C
:10F03000B8EEE77A67EE067A67EEA67AFCEEE77A34
:10F04000CDED017A9DF8043031B194F890109942D9
:10F0500038BF194684F8901094F8A61031B194F88E
:10F060009110994238BF194684F8911094F8A8007D
:10F0700030B194F892108B4238BF0B4684F892302E
:10F0800094F8A1309FED9A6ADFED9A6A94F8A31084
:10F0900007EE903AB8EEE77A67EE067A67EEA67A60
:10F0A000FCEEE77ACDED017A9DF8043031B194F8A9
:10F0B0009010994238BF194684F8901094F8A21025
:10F0C00031B194F89110994238BF194684F89110E3
:10F0D00094F8A41031B194F89250AB4238BF2B464B
:10F0E00084F8923094F8A9309FED816ADFED816A4F
:10F0F00094F8AB5007EE903AB8EEE77A67EE067AEE
:10F1000067EEA67AFCEEE77ACDED017A9DF8043041
:10F1100035B194F890509D4238BF1D4684F8905008
:10F1200094F8AA5035B194F891509D4238BF1D46CD
:10F1300084F8915094F8AC5035B194F89260B34291
:10F1400038BF334684F892302AB921B918B915B9B5
:10F150007F2384F892303F23002584F89C30C4F844
:10F16000985004F2B91104F5017003F009F994F80C
:10F17000E0310BB184F8E05194F8E231002584F8D5
:10F18000DF51002B00F0F780D4F81C3284F8E251F4
:10F19000C4F8B03098F804305BB1D8F8083088F87B
:10F1A0000250184688F8045088F803500BB102F05A
:10F1B00055FB08F10C08C145ECD194F89D309FED4A
:10F1C0004C6A94F89F1007EE903A94F89630B8EE97
:10F1D000E77A06EE903A67EE067AF8EEE66A0022E3
:10F1E00067EEA67A84F89220FCEEE77A84F8912004
:10F1F000CDED017A9DF8043084F8902009B184F8AF
:10F20000903094F89E200AB184F8913094F8A020B0
:10F210000AB184F8923094F8A5309FED356A94F8DD
:10F22000A71007EE903A94F89430B8EEE77A06EE1D
:10F23000903A67EE067AF8EEE66A67EEA67AFCEE9A
:10F24000E77ACDED017A9DF8043031B194F8901051
:10F25000994238BF194684F8901094F8A61031B13D
:10F2600094F89110994238BF194684F8911094F897
:10F27000A80030B194F892108B4238BF0B4684F846
:10F28000923094F8A1309FED1A6A94F8A31007EE1B
:10F29000903A94F89530B8EEE77A06EE903A67EE39
:10F2A000067AF8EEE66A67EEA67AFCEEE77ACDED2E
:10F2B000017A9DF8043031B194F89010994238BF2A
:10F2C000194684F8901094F8A21031B194F8911076
:10F2D000994238BF194684F8911094F8A41069B186
:10F2E00094F89250AB4238BF2B4684F8923005E038
:10F2F0000AD7233C000000000AD7233C94F8A93029
:10F300001FED036A94F8AB5007EE903A94F89330EF
:10F31000B8EEE77A06EE903A67EE067AF8EEE66A1D
:10F3200067EEA67AFCEEE77ACDED017A9DF804301F
:10F3300035B194F890509D4238BF1D4684F89050E6
:10F3400094F8AA5035B194F891509D4238BF1D46AB
:10F3500084F8915094F8AC5035B194F89260B3426F
:10F3600038BF334684F892302AB921B918B915B993
:10F370007F2384F89230204603B0BDEC028BBDE8B9
:10F38000F08300BF2DE9F04F2DED028B8B00CDB047
:10F390000A3302AF23F007037961ADEB030D90F858
:10F3A000E1117A6002AB06463B6139B390F8DD317A
:10F3B000DBB1002400F5987503E00134A4B2A34248
:10F3C00013D904EB440206EB820108790028F4D03B
:10F3D0004B78886816F82220294602F005F8013497
:10F3E00096F8DD31A4B2A342EBD806F2B91106F5C6
:10F3F000017002F0C5FF002386F8E1317B69002B24
:10F4000000F0AB8007F127084FF6144406F50173AE
:10F410009FED588ABB6028F00F08C2F200044FF03D
:10F42000000A3B694FF4807203EB8A0900214046D1
:10F4300013F08AF800214FF48072484613F084F8E4
:10F44000BD68284602F0DEFF8346284603F034F804
:10F4500096F8DD11002955D0C7F80CA0002582468A
:10F4600003E00135EDB28D424AD205EB450306EBD0
:10F4700083031A79002AF4D0986806F18403009374
:10F480005A465346414601F067FEA8F1040308F1CD
:10F49000FC0E4A46F7EE006ABFEE006A00200DE05F
:10F4A000216801312160B7EE007AD2ED007A186050
:10F4B00037EE877A7345A2EC017A1BD053F8041F0C
:10F4C000091121F35721491007EE901AF8EEE77A57
:10F4D00087EE887AB4EEE67AF1EE10FAE0DCB4EE6C
:10F4E000C67AF1EE10FAE0D5216801312160BFEE55
:10F4F000007ADAE796F8DD110135EDB28D42B4D32A
:10F50000D7F80CA07B690AF1400A1FFA8AFA534522
:10F5100087D83C691D4606F1B4001A462146FAF721
:10F5200015FC7A689FED137A681E80B202EB4000EA
:10F530002146023AF1EC017A67EE877AFDEEE77A2E
:10F5400017EE903A22F8023F8242F3D107F5967700
:10F55000BD46BDEC028BBDE8F08F39691A4606F155
:10F56000B400FAF7F3FB07F59677BD46BDEC028BC6
:10F57000BDE8F08F00FEFF462DE9F843064690F8FF
:10F58000C03190F8DD51002A00F0B080183BCF1850
:10F5900090F8DE81FFB2002D00F09F804FEA48090D
:10F5A00009EB080300EB830341469C78CE46002C10
:10F5B0006ED0002402E08378002B69D00131013441
:10F5C00091FBF5F305FB1311E4B24FEA410E0EEB8C
:10F5D0000100AC4206EB80005FFA81F8EBD196F8AF
:10F5E000E031002B4BD096F8DD31002B47D032793B
:10F5F000002A40F06281012B41D9327C002A40F080
:10F600005E81022B3BD0327F002A40F06281032BC7
:10F6100035D096F82820002A40F05D81042B2ED0AA
:10F6200096F83420002A40F04C81052B27D096F81C
:10F630004020002A40F04781062B20D096F84C202D
:10F64000002A40F04281072B19D096F85820002A52
:10F6500040F03D81082B12D096F86420002A40F03B
:10F660003C81092B0BD096F87020002A40F037819E
:10F670000A2B04D096F87C30002B40F0E9804FEA4A
:10F680004809C84406EB880601233371BDE8F883B6
:10F690008E444FEA8E0E013106EB0E0991FBF5F315
:10F6A00005FB131586F8DE5106F80E7089F8012067
:10F6B00096F8DF3189F803300121134689F80210EA
:10F6C000D9F808003A4606F5987101F087FB96F8DC
:10F6D000B831002B53D1002C81D106F5017002F016
:10F6E00011FF96F8E031002BC9D07CE7183BCF180A
:10F6F000FBB2002D41D0017899427BD0012D3CD93D
:10F70000327B9A4271D0022D37D0327E9A4267D036
:10F71000032D32D096F824209A425BD0042D2CD0B1
:10F7200096F830209A424FD0052D26D096F83C20EE
:10F730009A4243D0062D20D096F848209A4237D0DE
:10F74000072D1AD096F854209A422BD0082D14D0A9
:10F7500096F860209A421FD0092D0ED096F86C20A2
:10F760009A4213D00A2D08D096F878209A4204D1F4
:10F7700096F87A30002B40F08280BDE8F883D9F803
:10F78000080002F06BF8002CA7D028E796F86E204E
:10F79000002AE7D0092773E096F86220002ADBD020
:10F7A00008276DE096F85620002ACFD0072767E09B
:10F7B00096F84A20002AC3D0062761E096F83E203A
:10F7C000002AB7D005275BE096F83220002AABD09C
:10F7D000042755E096F82620002A9FD003274FE003
:10F7E000B27E002A94D002274AE0B27B002A8AD057
:10F7F000012745E08178002980D082701746804635
:10F8000096F8E031E3B14FF0000E734671464FF0C9
:10F81000FF3203EB430306EB8304481CA4782CB1AE
:10F8200016F823309342C4BF5AB28E4641B2A94261
:10F830000B46EEDB013203D098F80430002B50D198
:10F8400096F8DF3183B3012388F80330BDE8F883ED
:10F850000A2303EB43039B00F2189178C1B1F35CD8
:10F86000BB428AD24FEA480909EB080306EB83033F
:10F87000002111719868916801F09CFF01E70A2747
:10F8800007EB470806EB8808002388F80230B7E743
:10F890004FEA480909EB080306EB830311719868E6
:10F8A000916801F0A7FFECE607EB470206EB820642
:10F8B000B068BDE8F84301F083BD0023C9E7012328
:10F8C000C7E70423C5E70523C3E70623C1E70723EA
:10F8D000BFE70223BDE70323BBE70823B9E70923FA
:10F8E000B7E70EEB4E0E07EB470206EB8E03002147
:10F8F00006EB820288F8041001211971986891685A
:10F9000001F058FF9CE700BFF8B590F8C03190F8BF
:10F91000DD41183B1944002C40D00378C9B28B421A
:10F920003DD0012C3AD9037B8B4200F09D80022C04
:10F9300034D0037E8B4200F09180032C2ED090F8BF
:10F9400024308B4200F08380042C27D090F8303094
:10F950008B4276D0052C21D090F83C308B426AD077
:10F96000062C1BD090F848308B425ED0072C15D067
:10F9700090F854308B4252D0082C0FD090F8603061
:10F980008B4246D0092C09D090F86C308B423AD08B
:10F990000A2C03D090F878308B422ED0F8BD8378B3
:10F9A000002BBED000258570064690F8E031074652
:10F9B000E3B100231A469C464FF0FF3E03EB43039E
:10F9C00007EB8300511C807830B117F82330734562
:10F9D000C4BF4FFA83FE94464AB2A2421346EDDBFF
:10F9E000BEF1FF3F02D03379002B52D197F8DF31BF
:10F9F000002B45D00123F370F8BD90F87A30002B2E
:10FA0000CCD00A2535E090F86E30002BC0D0092507
:10FA10002FE090F86230002BB4D0082529E090F850
:10FA20005630002BA8D0072523E090F84A30002B51
:10FA30009CD006251DE090F83E30002B90D0052587
:10FA400017E090F83230002B84D0042511E090F8B4
:10FA50002630002B3FF478AF03250AE0837E002B8D
:10FA60003FF46BAF022504E0837B002B3FF45FAFD4
:10FA7000012505EB450600EB86060023B37094E7ED
:10FA800005EB450507EB8500BDE8F840806801F00F
:10FA900097BC0CEB4C0C05EB450207EB8C030021EB
:10FAA00007EB82023171012119719868916801F0A8
:10FAB00081FE9BE7012380F8E131704790F8E03147
:10FAC0008B4218BF80F8E011704700BF90F8DF311B
:10FAD0008B4218BF80F8DF11704700BF90F8DF013C
:10FAE000704700BF70B5044600F1840600252379F5
:10FAF0003BB1A368A57018462571E5700BB101F004
:10FB0000ADFE0C34B442F2D170BD00BF90F89D3010
:10FB10009FED6C6ADFED6C6A90F89F1007EE903AEB
:10FB2000B8EEE77A70B467EE067A83B067EEA67A2D
:10FB30000023FCEEE77A4FF40052CDED017AC0F8D5
:10FB40008420C0F888309DF80420C0F88C3080F8FC
:10FB5000963080F8953080F8943080F8933080F8B3
:10FB6000923080F8913080F8903009B180F8902080
:10FB700090F89E300BB180F8912090F8A01009B158
:10FB800080F8922090F8A5309FED4E6ADFED4E6A26
:10FB900090F8A72007EE903AB8EEE77A67EE067A7B
:10FBA00067EEA67AFCEEE77ACDED017A9DF8043097
:10FBB00032B190F890209A4238BF1A4680F89020CF
:10FBC00090F8A62032B190F891209A4238BF1A4698
:10FBD00080F8912090F8A84034B190F89220934298
:10FBE00038BF134680F8923090F8A1309FED356A07
:10FBF000DFED356A90F8A32007EE903AB8EEE77A89
:10FC000067EE067A67EEA67AFCEEE77ACDED017A2A
:10FC10009DF8043032B190F890209A4238BF1A46CD
:10FC200080F8902090F8A22032B190F891209A426A
:10FC300038BF1A4680F8912090F8A42032B190F88D
:10FC40009250AB4238BF2B4680F8923090F8A930E2
:10FC50009FED1C6ADFED1C6A90F8AB5007EE903AFE
:10FC6000B8EEE77A67EE067A67EEA67AFCEEE77AF8
:10FC7000CDED017A9DF8043035B190F890509D4259
:10FC800038BF1D4680F8905090F8AA5035B190F8D2
:10FC900091509D4238BF1D4680F8915090F8AC506D
:10FCA00035B190F89260B34238BF334680F8923055
:10FCB00029B922B91CB915B97F2380F8923003B055
:10FCC00070BC70470AD7233C00000000037913B1D1
:10FCD0008378002B60D1037C13B1837B002B58D138
:10FCE000037F13B1837E002B50D190F828301BB1D5
:10FCF00090F82630002B45D190F8343013B190F8AD
:10FD00003230DBBB90F8403013B190F83E308BBB03
:10FD100090F84C3013B190F84A303BBB90F8583013
:10FD200013B190F85630EBB990F8643013B190F8F5
:10FD300062309BB990F8703013B190F86E304BB9C7
:10FD400090F87C302BB190F87A3013B1002380F812
:10FD50007A307047002380F86E30F1E7002380F896
:10FD60006230E7E7002380F85630DDE7002380F8B3
:10FD70004A30D3E7002380F83E30C9E7002380F8FB
:10FD80003230BFE7002380F82630B5E700238376C2
:10FD9000ABE700238373A3E7002383709BE700BFD7
:10FDA00090F8DD01704700BF2DE9F04F054690F84F
:10FDB000B611D0F8B00085B002F0F4F895F8DD1176
:10FDC000002900F0C780C0F3C0030093C0F3001304
:10FDD00000260193C0F34013344600F00108C0F33D
:10FDE000400BC0F3800A029305F5F27703E001347B
:10FDF000E4B2A1427CD904EB440305EB830999F8F2
:10FE00000420002AF3D000212022384612F09CFB67
:10FE10003946D9F8080001F08FFCB8F1000F6BD01B
:10FE2000D5F8E41140F22D42914269D895F8FC11C1
:10FE3000A1F10401B1FA81F1022049090122BBF1CB
:10FE4000000F0AD0D5F8E82140F22D4E724503D8B4
:10FE500095F8FD21042A57D00246BAF1000F0DD0C3
:10FE6000D5F8EC0140F22D4E01327045D2B205D8E2
:10FE700095F8FE01042804BF0131C9B2009B6BB1A3
:10FE8000D5F8F00140F22D4E01327045D2B205D8BE
:10FE900095F8FF01042804BF0131C9B2019B6BB181
:10FEA000D5F8F40140F22D4E01327045D2B205D89A
:10FEB00095F80002042804BF0131C9B2029B6BB15E
:10FEC000D5F8F80140F22D4E01327045D2B205D876
:10FED00095F80102042804BF0131C9B2914217D03C
:10FEE00095F8DD110134E4B20136A142F6B282D8B0
:10FEF000304605B0BDE8F08F0120424641469EE7FE
:10FF00000220012200219AE70131C9B20246A4E78A
:10FF1000002243F6D03089F8042089F8032089F8BC
:10FF200002201021C0F2020003920BF00FFE039A90
:10FF30004EF20020134621460A22C2F200000CF0C5
:10FF400029FD4EF20020C2F200000CF011FD95F8E0
:10FF5000DD114CE70E46CBE72DE9F04100F5987333
:10FF600084B004460A4600F5D775106856685E608E
:10FF700018601089967A9E721881D07A00F0030674
:10FF8000C0F38100DE721873107BC0F3C30600F06B
:10FF900007001E755873507BC0F3820600F0030003
:10FFA000DE739873907B1874D07BC0F3440600F026
:10FFB00001009E745874107CD87415339D4202F170
:10FFC0001102D2D10B460A4653F8660FDFEDD75A1D
:10FFD0005B68C4F8AE016B6091F86E3003F01F03EC
:10FFE00084F8B63191F86F30C3F3C00003F0070313
:10FFF00084F8B80184F8B7310B6FC4F8B93191F8BF
:020000021000EC
:100000007430C3F30115C3F3420003F0010384F815
:10001000BF5184F8BE0184F8BD3191F8753084F881
:10002000C03152F8761F04F2C1175368C4F8C111E9
:100030007B6013893B8163220123072184F8CB3144
:1000400084F8CC3184F8CD2184F8CF2184F8D121F3
:1000500084F8D32184F8CE1184F8D01184F8D21119
:1000600084F8D41194F8941084F8D63106EE101A5E
:1000700094F8961084F8D73106EE901A94F89510FB
:1000800084F8D831B8EEC66AF8EEE66A07EE101AC0
:1000900094F8931084F8D93126EE256A66EEA56AA5
:1000A00007EE901AB8EEC77ABCEEC66AFCEEE66AB6
:1000B000F8EEE77A27EE257A8DED016ACDED026A3A
:1000C0009DF804009DF8081084F8DA3167EEA57AEF
:1000D000BCEEC77A88428DED037AFCEEE77A38BF32
:1000E00008469DF80C10CDED017A88429DF8045029
:1000F00084F8DB3138BF0846A842C4F88830C4F819
:100100008C3084F89D2084F89E3084F89F3084F8E9
:10011000A03084F8A12084F8A23084F8A33084F8B9
:10012000A43084F8A52084F8A63084F8A73084F899
:10013000A83084F8A92084F8AA3084F8AB3084F879
:10014000AC30237938BF284600210B253F2284F8A4
:10015000900084F8D511C4F8981084F8DC5184F824
:10016000910084F8920084F89C201BB1A378002BA6
:1001700040F08381237C1BB1A37B002B40F07A816C
:10018000237F1BB1A37E002B40F0718194F82830AF
:1001900023B194F82630002B40F0658194F8343078
:1001A00023B194F83230002B40F0598194F840305C
:1001B00023B194F83E30002B40F04D8194F84C3040
:1001C00023B194F84A30002B40F0418194F8583024
:1001D00023B194F85630002B40F0358194F8643008
:1001E00023B194F86230002B40F0298194F87030EC
:1001F00023B194F86E30002B40F01D8194F87C30D0
:1002000023B194F87A30002B40F011810B2384F84D
:10021000DD31254604F1840800262B793BB1AB681B
:10022000AE7018462E71EE700BB101F017FB0C3555
:100230004545F2D194F89D309FED3D6A94F89F10AA
:1002400007EE903A94F89630B8EEE77A06EE903AD8
:1002500067EE067AF8EEE66A002267EEA67A84F880
:100260009220FCEEE77A84F89120CDED017A9DF89A
:10027000043084F8902009B184F8903094F89E20DE
:10028000002A40F0148194F8A0200AB184F892303A
:1002900094F8A5309FED266A94F8A71007EE903ADF
:1002A00094F89430B8EEE77A06EE903A67EE067A64
:1002B000F8EEE66A67EEA67AFCEEE77ACDED017A13
:1002C0009DF8043031B194F89010994238BF194626
:1002D00084F8901094F8A610002940F0E08094F87B
:1002E000A81031B194F89200834238BF034684F8D5
:1002F000923094F8A1309FED0E6A94F8A30007EEB7
:10030000903A94F89530B8EEE77A06EE903A67EEB8
:10031000067AF8EEE66A67EEA67AFCEEE77ACDEDAD
:10032000017A9DF8043060B104E000BFA3707D3F06
:100330000AD7233C94F89000984238BF184684F8B6
:10034000900094F8A200002840F0A18094F8A40046
:1003500030B194F89250AB4238BF2B4684F89230BB
:1003600094F8A9301FED0E6A94F8AB5007EE903A5E
:1003700094F89330B8EEE77A06EE903A67EE067A94
:10038000F8EEE66A67EEA67AFCEEE77ACDED017A42
:100390009DF8043035B194F890509D4238BF1D4609
:1003A00084F8905094F8AA50002D68D194F8AC507D
:1003B00035B194F89260B34238BF334684F8923036
:1003C0002AB920B919B915B97F2384F892300125CB
:1003D00040F650700A22394684F8E151C2F2010019
:1003E00012F05CFA43F2D4300721C0F202000BF0A5
:1003F000ADFB40F65070C2F2010012F0E1F9014687
:1004000040F65070C2F201000BF0A0FB43F2DC306A
:100410000921C0F202000BF099FB4EF20020C2F25B
:1004200000000CF0A5FA284604B0BDE8F0810023D6
:1004300084F87A30EAE6002384F86E30DEE60023A2
:1004400084F86230D2E6002384F85630C6E60023F2
:1004500084F84A30BAE6002384F83E30AEE6002342
:1004600084F83230A2E6002384F8263096E6002392
:10047000A3768BE60023A37382E6A1707AE694F854
:1004800091509D4238BF1D4684F891508EE794F8F4
:100490009100984238BF184684F8910056E794F8C6
:1004A0009110994238BF194684F8911017E784F8E3
:1004B0009130E8E610B5044612F082F90146204674
:1004C000BDE810400BF042BB10B5044612F078F9BD
:1004D000014620460BF03AFB04464EF20020C2F2E1
:1004E00000000CF045FA204410BD00BF2DE9F0419A
:1004F00000262F270C468E600E604E60C1F80B6000
:100500000A2201F8017B804611F022FD204612F0FC
:1005100057F908EB48054FF62442C2F2000208EBF7
:1005200085051544431C27542946E01812F0D8F8D5
:100530004EF2002743F6E430C2F200072121C0F258
:1005400002000BF003FB33460A22414638460CF00A
:1005500021FA43F608400A21C0F202000BF0F6FA35
:10056000284612F02DF9014628460BF0EFFA43F227
:1005700038700321C0F202000BF0E8FA204612F0B6
:100580001FF9014620460BF0E1FA43F24020C0F289
:10059000020001210BF0DAFA3846BDE8F0410CF018
:1005A000E7B900BF10B584B00C460146684612F0AA
:1005B00097F843F270316846C0F2020112F0A2F9D6
:1005C00028B10146204612F08BF804B010BD43F666
:1005D0001443C0F2020303CB2060616004B010BD7D
:1005E0002DE9F04194B0044604A804F085FB40F6E0
:1005F000F050C2F201004FF4B072002111F0A4FFDC
:1006000040F63053C2F201031B7833B904A804F05A
:1006100081FB002014B0BDE8F08148F21F53C5F201
:10062000EB13A3FB04235B09642000FB1340C0B25F
:100630006946FFF75BFF43F61C401E21C0F2020033
:100640000BF084FA684612F0BBF8014668460BF0DE
:100650007DFA43F240200121C0F202000BF076FA4D
:100660004EF20020C2F200000CF082F948F21011A4
:1006700001236A460CA8C2F2010104F019FC14AB74
:100680009DF8344053F8131DCDF81D105A689E682C
:100690001D7B0E99CDF82120139B9DF83C20CDF8B1
:1006A00025600CA88DF829508DF8144006918DF81E
:1006B0001C200B9304F02EFB04A804F045FB00283B
:1006C000A4D004A804F03CFB41F2080398420DD0EA
:1006D00043F63C401A21C0F202000BF037FA4EF20A
:1006E0000020C2F200000CF043F98FE704A804F0E8
:1006F00073FAF0280DD043F658401F21C0F20200D3
:100700000BF024FA4EF20020C2F200000CF030F997
:100710007CE704A804F060FA43280DD043F6784043
:100720001C21C0F202000BF011FA4EF20020C2F2BE
:1007300000000CF01DF969E741F2070104A804F07C
:10074000F5FA04A804F048FAF72806D043F69840D2
:10075000C0F20200FFF7B8FE58E7032104A804F036
:10076000E5FA04A804F038FA092806D043F6B840A0
:10077000C0F20200FFF7A8FE48E741F2060104A814
:1007800004F0D4FA04A804F027FA062146B204A81B
:1007900004F0CCFA04A804F01FFA002740F6F05544
:1007A00002463C46B846C2F2010516E004F014FACF
:1007B00004F07F0108EB880308EB43030246A1F134
:1007C000760009282B449CBF5B1803F8762C7F2900
:1007D00004BF08F101085FFA88F80134A4B2D2B26C
:1007E000B4F5805F04A8A7EB0207DFD143F6D84039
:1007F000C0F20200FFF75EFE07F07F074EF2002016
:10080000394600231022C2F200000CF0C3F843F670
:10081000EC40C0F20200FFF74DFE4EF20020002334
:1008200010223146C2F200000CF0B4F843F240202E
:10083000C0F20200FFF748FEB7423FF4E7AE43F6CE
:10084000F440C0F20200FFF735FE4EF200203946B8
:1008500000231022C2F200000CF09CF843F6145062
:10086000C0F20200FFF726FE4EF2002031460023C0
:100870001022C2F200000CF08DF84EF20020C2F2FD
:1008800000000CF075F8C1E62DE9F04192B002A825
:1008900004F032FA4FF62440C2F2000040F2145243
:1008A000002111F051FE40F63053C2F201031C78D2
:1008B000002C00F09E804FF62446C2F20006002471
:1008C00008E00AA804F026FA02A804F03DFA00287D
:1008D00000F08F802F2300250A220DF1050120460C
:1008E00001958DF8043011F033FB48F21011C2F27B
:1008F0000101012301AA0AA804F0DAFA9DF82CE00C
:100900000C9D9DF834709DF836009DF837109DF8C9
:1009100038209DF839309DF83AC09DF835808DF823
:100920000CE004959DF83BE08DF814709DF83D5067
:100930009DF83C708DF816008DF817109DF83E005C
:100940009DF83F108DF818208DF819309DF8402043
:100950009DF841308DF81F108DF820208DF81AC0B9
:100960008DF81BE08DF81E008DF815808DF81C7039
:100970008DF81D508DF821300AA8119B099304F0C1
:10098000C9F902A804F0E0F9012202A988B30AA873
:1009900004F006FB0AA804F0C1F9002891D10AA8C6
:1009A00004F0BAF904EB440504EB8505354401462F
:1009B000284611F095FE43F61C500C21C0F20200AF
:1009C0000BF0C4F8284611F0FBFE014628460BF058
:1009D000BDF843F240200121C0F202000BF0B6F84E
:1009E0004EF20020C2F2000001340BF0C1FFE4B26D
:1009F00067E702A804F08EF9204612B0BDE8F08146
:100A00002DE9F0470E469046054604F099F941F26B
:100A1000080398420FD043F63C40C0F202001A216E
:100A20000BF094F84EF20020C2F200000BF0A0FF91
:100A30000020BDE8F087284604F0CEF8F02805D065
:100A400043F65840C0F202001F21E9E7284604F0AF
:100A5000C3F8432805D043F67840C0F202001C21B9
:100A6000DEE741F20701284604F060F9284604F069
:100A7000B3F8F72805D043F69840C0F202001D21D4
:100A8000CEE70321284604F051F9284604F0A4F8E3
:100A9000092804D043F6B840C0F20200EFE741F263
:100AA0000601284604F042F9284604F095F806218C
:100AB0004FFA80F9284604F039F906F1010A0024BA
:100AC0004FEACA1AF6012746284604F085F8B442D0
:100AD000C3B2A7EB030704DBA31B5445B8BF08F858
:100AE00003000134B4F5805FEED143F6D840122103
:100AF000C0F202000BF02AF807F07F074EF2002048
:100B0000002310223946C2F200000BF043FF43F6E7
:100B1000EC400421C0F202000BF018F84EF2002065
:100B2000002310224946C2F200000BF033FF43F2CB
:100B300040200121C0F202000BF008F84EF2002024
:100B4000C2F200000BF014FF4F4508D14FF62043CE
:100B5000C2F2000300221A800120BDE8F08743F6AC
:100B6000F4401F21C0F202000AF0F0FF4EF2002014
:100B7000394600231022C2F200000BF00BFF43F6AF
:100B800014500621C0F202000AF0E0FF4EF20020ED
:100B9000494600231022C2F200000BF0FBFE4EF289
:100BA0000020C2F200000BF0E3FE0020BDE8F08759
:100BB00030B540F63052C2F20102B5B01378002BC6
:100BC00000F09C80044604A80D4604F095F848F215
:100BD0001F53C5F2EB13A3FB04235B09642000FB46
:100BE0001340C0B26946FFF781FC48F2101101239F
:100BF0006A4614A8C2F2010104F05AF934AB9DF818
:100C0000544053F8732DCDF81D2059689A681B7B0A
:100C1000CDF82110CDF8252016999DF85C208DF88F
:100C2000293014A81B9B8DF8144006918DF81C20C8
:100C30000B9304F06FF804A804F086F8044600BB98
:100C400043F62C501021C0F202000AF07FFF6846E4
:100C500011F0B6FD014668460AF078FF43F64050B1
:100C6000C0F2020008210AF071FF4EF20020C2F229
:100C700000000BF07DFE04A804F04CF8204635B0CF
:100C800030BDDDF82130DDF81D20CDF84130DDF834
:100C90002530CDF84530CDF83D209DF82930069A15
:100CA0008DF849300E929DF814308DF8343044F2AE
:100CB000B4329DF81C308DF83C30C0F2020205F0D1
:100CC0001F050B9B0C9229460CA814AA1393FFF73F
:100CD00097FE04460CA804F01DF804BB43F65C50D4
:100CE0001A21C0F202000AF031FF4EF20020C2F2D7
:100CF00000000BF03DFE04A804F00CF843F6785019
:100D00001321C0F202000AF021FF4EF20020C2F2CD
:100D100000000BF02DFE0024204635B030BD0A2225
:100D20000DF1C6010CA811F0B9FD43F64C500E218F
:100D3000C0F202000AF00AFF684611F041FD0146C8
:100D400068460AF003FF43F658000221C0F2020091
:100D50000AF0FCFE05EB850340F6F05005EB430579
:100D6000C2F201000544284611F02AFD014628463A
:100D70000AF0ECFE43F240200121C0F202000AF02A
:100D8000E5FE4EF20020C2F200000BF0F1FD40F64D
:100D90006453C2F2010314A91868FFF7DDF8044692
:100DA00069E700BF08F0B4BA0022C0F8A421C0F877
:100DB0009C21C0F8B421C0F8AC21C0F8C421C0F80F
:100DC000BC21C0F8D421C0F8CC21C0F8E421C0F87F
:100DD000DC21C0F8F421C0F8EC2170472DE9F04F78
:100DE00045F255541646C0F2150404FB06F49A4623
:100DF00004F142732DED088B08EE903A4FF04E53FC
:100E00000AEE103A4CF28303CBF6CA6309EE903A2D
:100E100043F27A63C3F6AB4309EE103A4DF20A731C
:100E2000C3F623430BEE103A4AF63B23C4F6B8331D
:100E300045F256550AEE903A18EE903AC5F25555DD
:100E400093B085FB022703F231733246A7EBE677B6
:100E500043F6D45B08EE903A4FEA6A030395814665
:100E6000073F08930C460546C0F2020B0026099185
:100E700090464EE0BAF1000F00F30F816FF0EE01E3
:100E800001FB02F20732D21000EB0213002F23EA1B
:100E9000E373627B40F3FF801F2FCCBFC2EB421293
:100EA0007A43D21000920AA90EAA09EB060000F0BC
:100EB00007FD627CA37CE17C207D002A7AD003F0D0
:100EC000030C4FF0640E40F678031EFB0C11C0F2C9
:100ED000440303FB01F307284FEAE301C3BF0738CC
:100EE00043F29143434300230B44C5F86C22C5F8F9
:100EF0003032A37B03F0030344365BF82330C5F89C
:100F00005432B6F5CC7F04F1150405F1040500F068
:100F1000D48020782179627863790A90A0780E9144
:100F20000B92A179E2780F930C90E379207C0D92DB
:100F30001193109100F01EFE237AC3EB0803B3F166
:100F4000110200F18680039A217B94F80AE0103B9D
:100F500082FB03C2A2EBE37301B303291ED01F2B54
:100F6000DBBF43F66462C0F20202FA23D35C03FBE8
:100F70000EFE40F2491303FB0EF301294FEAE3335F
:100F800016DD18447F28A8BF7F20BAF17F0F4FEAF3
:100F90004010E27B7FF76EAF0F2171E703FB0EF38A
:100FA00040F2491202FB03F301294FEA2333E8DC44
:100FB0005B42E6E7B8EEE88A079028EE0A0A069157
:100FC00020EE290A059304920DF00EFF20EE090A87
:100FD000F1EE0C7A80EE277A0798059B0699073880
:100FE00043F6E45E03F01F03C0F2020E5EF8233006
:100FF00007EE900A27EE087AF8EEE77AA7EE278A3E
:10100000BDEEC88A18EE102A1A441346049A002925
:101010003FF46BAF07EE901AF8EEE77AB7EE000AEE
:10102000A7EE8B0A05930DF061FFF6EE007AE0EE75
:101030002A7A17EE900A10F09DFB41EC100B0DF090
:10104000AFF951EC100B10F099FE059B049A034484
:101050004BE7039B94F809C0C2F10101E27A83FBDC
:10106000013EAEEBE17102B3032A1ED01F29DBBFA4
:1010700043F6646EC0F2020EFA211EF8011040F22F
:10108000491301FB0CF103FB01F3DB13012A3FF7CA
:1010900078AF5B4275E7002204E743F68C53C0F259
:1010A00002030899595CEF39EAE601FB0CF140F2C2
:1010B000491303FB01F31B13E8E7DDF8248098F8DC
:1010C0007E5098F8824098F87F3098F8830098F81E
:1010D00080600A950E9498F8845098F881400B939C
:1010E0000F9098F8853011930EAA0AA909F5FC70A3
:1010F0000C9610950D9401F029FA98F88630C9F8ED
:10110000883298F887302BB3C3F10803C9F85032FE
:1011100098F88B3003EB830303EB43139B11C9F85F
:101120008C3298F88F3043F6CC52C0F2020203F0B2
:101130000703D35CC9F8903298F88C3003EB830333
:1011400003EB43139B11C9F8843213B0BDEC088B39
:10115000BDE8F08F1023D9E72DE9F04F2DED048B7A
:1011600089B0D0F89052DDF8588007918146D0F8C8
:101170008C0298F80DE09B46A2F5000305FB03F5F1
:1011800000FB0BF0A0FB0567EB1700FB0377144691
:101190008EFB0523900B40EA8340FE1186EAE6733E
:1011A00080EAE072A2EBE072A3EBE6739342B8BF71
:1011B000134609F5FC701E4601F000FAD8F800301D
:1011C000002DB4BF4FF0FF320122B3F5005A06FBE9
:1011D00002001AD0D8F80820002A40F0D980D8F8A8
:1011E00004304FEACA2A07EE90AA07EE103AF8EE4A
:1011F000E77AB8EEC77AF2EE086A67EE877A87EE8A
:10120000A67AFDEEC77A17EE90AA4FF05A5309EE70
:10121000103A45F62943C3F68F53D9F8842298F83B
:101220000C1008EE903A43F23333C4F2431308EE45
:10123000103A82FB0B23C4F180744FEA122B4BEA65
:10124000036BE3170BFB03F298F80E30002704FB47
:1012500007225B04ABFB046781FB0445C3F57E0BEF
:10126000E30943EA45635B4517444FEA166138BF1B
:101270005B4641EA0721D8F814208B4238BF0B4661
:1012800092449B4600EB0A0305934E4609F50C7405
:101290004F46002514E0504401F040F8C6F8A00184
:1012A000384600F065FB626A02BBC6F8980101355A
:1012B000062D07F1440706F1100604F1040452D08C
:1012C00098F818302B4113F0010344D0E36B2068E9
:1012D000002BE0D1059B184401F020F8C6F8A001CE
:1012E000384600F045FB626A002ADED0D117ABFB1E
:1012F0000223CDE90223039A06900BFB01230393FB
:10130000DDE90201020E42EA012207EE902AF8EE20
:10131000677AB0EE480A67EE897AA7EEA80A0DF060
:1013200063FDFCEEC07A069817EE901AC3174FEAD9
:10133000011E0EFB03F3090F00FB0131AEFB00237E
:10134000CDE902230B440393029B1A0F039B42EA4D
:101350000312801AA9E73846029300F009FB029BAA
:10136000C6F89831A3E7D8F82C00D9F850120268D3
:10137000D9F88832019109F51271009194680799A2
:1013800009F5CC72A04709B0BDEC048BBDE8F08F25
:1013900021230C21C8F2040391FBF2F202FB0AFAAA
:1013A00083FB0A1353444FEAEA7ACAEB233A41F625
:1013B000FF7393FBF2F303FB0AFA4FEACA2A24E70E
:1013C00070B50646044600F5CC752046002144342D
:1013D00000F080FBAC42F8D106F5FC700021BDE8BE
:1013E000704001F039B900BF2DE9F04F45F2555476
:1013F0009246C0F2150404FB0AF4994604F14273C4
:101400002DED088B08EE903A4FF04E530AEE103A4D
:101410004CF28303CBF6CA6309EE903A43F27A6347
:10142000C3F6AB4309EE103A4DF20A73C3F62343F9
:101430000BEE103A4AF63B23C4F6B83345F2565544
:101440000AEE903A18EE903AC5F2555593B085FBE6
:101450000A2803F23173A8EBEA7843F6D45B08EE6E
:10146000903A4FEA69030295074607900891A8F160
:10147000070809930C460546C0F2020B00262AE035
:10148000B9F1000F00F312816FF0EE0101FB02F2DF
:101490000732D21000EB0213B8F1000F23EAE37316
:1014A000627B40F30181B8F11F0FCCBFC2EB421247
:1014B00008FB02F2D2100092384601360EAA0AA9A1
:1014C00000F062FB062E04F1150405F1040507F196
:1014D000440700F0FB80627CA37CE17C207D002A35
:1014E00071D003F0030C4FF0640E40F678031EFB3E
:1014F0000C11C0F2440303FB01F307284FEAE30198
:10150000C3BF073843F29143434300230B44C5F85C
:101510003032A37BC5F86C2203F003035BF8233061
:10152000C5F8543220782179627863790A90A078DE
:101530000E910B92A179E2780F930C90E379207CC5
:101540000D921193109100F015FB237AC3EB0A035F
:10155000B3F1110200F18680029A217B94F80AE02F
:10156000103B82FB03C2A2EBE37301B303291ED03D
:101570001F2BDBBF43F66462C0F20202FA23D35C86
:1015800003FB0EFE40F2491303FB0EF301294FEA61
:10159000E33316DD18447F28A8BF7F20B9F17F0F01
:1015A0004FEA4010E27B7FF76BAF0F216EE703FB42
:1015B0000EF340F2491202FB03F301294FEA2333F1
:1015C000E8DC5B42E6E7B8EEE88A069028EE0A0A15
:1015D000059120EE290A049303920DF005FC20EEFC
:1015E000090AF1EE0C7A80EE277A0698049B059999
:1015F000073843F6E45E03F01F03C0F2020E5EF804
:10160000233007EE900A27EE087AF8EEE77AA7EE85
:10161000278ABDEEC88A18EE102A1A441346039A88
:1016200000293FF474AF07EE901AF8EEE77AB7EEB0
:10163000000AA7EE8B0A04930DF058FCF6EE007A30
:10164000E0EE2A7A17EE900A10F094F841EC100BB5
:101650000CF0A6FE51EC100B10F090FB049B039ACB
:10166000034454E7029B94F809C0C2F10101E27AF5
:1016700083FB013EAEEBE17102B3032A1ED01F29AA
:10168000DBBF43F6646EC0F2020EFA211EF80110B1
:1016900040F2491301FB0CF103FB01F3DB13012AB8
:1016A0003FF778AF5B4275E7002204E743F68C53BF
:1016B000C0F202030999595CEF39E7E601FB0CF12E
:1016C00040F2491303FB01F31B13E8E7089A07995B
:1016D00092F88630C1F8883292F887303BB3C3F174
:1016E000080308461446C0F8503294F88B3003EBD8
:1016F000830303EB43139B11C0F88C3294F88F30B3
:1017000043F6CC52C0F2020203F00703D35CC0F8E8
:10171000903294F88C3003EB830303EB43139B115B
:10172000C0F8843213B0BDEC088BBDE8F08F1023F5
:1017300008461446D7E700BF2DE9F84F43F2680A80
:10174000804689460646A1F1040B01F1180500F117
:1017500060070446C2F2010AD4F8981101F17241FF
:101760004A1340F2FE731340581C5AF823205AF8CB
:101770002000C1F30D0382FB0323920B42EA834254
:101780000916C1F1060102440A41304629461034C7
:101790004BF8042F00F050FAA74205F1010506F1BD
:1017A0004406D9D109F11E0108F5FC70BDE8F84FD7
:1017B00000F080BF2DE9F04104460F4600F5CC78DB
:1017C00006460D463946204600F03AFAD5F89C31D7
:1017D000C6F89C314434D5F8A431C6F8A431444548
:1017E00007F1440705F1100506F11006EAD1BDE83E
:1017F000F08100BFD1F8AC31D1F8A42110B4D1F8F8
:101800009C41C0F89C41C0F8A421C0F8AC31D1F88B
:10181000B431C0F8B431D1F8BC31C0F8BC31D1F822
:10182000C431C0F8C431D1F8CC31C0F8CC31D1F8D2
:10183000D431C0F8D431D1F8DC31C0F8DC31D1F882
:10184000E431C0F8E431D1F8EC31C0F8EC31D1F832
:10185000F431C0F8F4315DF8044B70470023C0F850
:101860009C31C0F8A431C0F8AC31C0F8B431C0F834
:10187000BC31C0F8C431C0F8CC31C0F8D431C0F8A4
:10188000DC31C0F8E431C0F8EC31C0F8F431704715
:101890004FF48843C4F22C7307EE103A87EE000A27
:1018A0004FF0974307EE903A20EE270A4DF69C63DF
:1018B000BCEEC00AC2F2000383ED000A704700BF0D
:1018C00030B40C680460146804614D684560556864
:1018D00045618D68856095688561C968C160D26819
:1018E000C261132C4FF0000282624263DBBF43F6F9
:1018F0008862C0F202021C3452F824400362641071
:1019000003EB8413A3F58553026802994162102BFF
:1019100002EB8204B8BF102302EBC4021B04002BAD
:1019200001EBA212D4BF0024012401253E2A80F835
:101930004050C36280F8304016DC02F0030392107E
:101940000433083203FA02F2D3174DF69C61C2F257
:1019500000010968A1FB024501FB0355230E43EA80
:101960000523836330BC70474FF060720023ECE7BF
:10197000426B022AF0B4034605DD032A66D190F8D3
:101980004010002962D193F8301071B9986A996BB0
:10199000DC6A401AA042986259DC511C03299C62FF
:1019A00059635BDD2046F0BC70474FF6FF70996AC3
:1019B000C0F2B36081424CDDC1F1885000169D6BCE
:1019C000DC6A05FB0010A042986240DB511C032931
:1019D0009C625963E6DC03EB820251691329DBBF89
:1019E00043F68860C0F2020001F11C0550F8215056
:1019F000196A586A6D1001EB8511A1F585511029FE
:101A0000B8BF102109048C42ACBF00250125D96262
:101A100083F83050526802EB820102EBC10200EB06
:101A2000A2123E2A4CDD4FF0607600274DF69C62F4
:101A3000C2F2000220461268A2FB064502FB0755CF
:101A4000220E42EA05229A63F0BC7047986AF0BC05
:101A500070470021C0F2B4610A20B0E703EB8202B4
:101A600051691329DBBF43F68860C0F2020001F11F
:101A70001C0550F82150196A586A6D1001EB851148
:101A8000A1F585511029B8BF102109048C42ACBFC3
:101A900000250125D96283F83050526802EB82019B
:101AA00002EBC10200EBA2103E28BCDC00F00306F2
:101AB00080100436083006FA00F00646C717B5E76E
:101AC00002F0030692100436083206FA02F21646B5
:101AD000D717ABE790F840308B4241D000290CBFBC
:101AE0000323002330B49D00421980F84010436363
:101AF0001369816A132BDBBF43F68862C0F20202CE
:101B000003F11C0452F82340036A426A641003EB99
:101B10008413A3F58553102BB8BF10231B048B42ED
:101B2000D4BF0021012180F83010C362435903EB78
:101B3000830103EBC10302EBA3123E2A11DD4FF038
:101B4000607200234DF69C61C2F200010968A1FB9E
:101B5000024501FB0355230E43EA052330BC836392
:101B6000704702F0030392100433083203FA02F2C2
:101B7000D317E7E71328DBBF43F68863C0F20203FD
:101B80001C3053F82000704730B40C6804601468AF
:101B900004614C684460546844618C688460946853
:101BA0008461C968C16090F84010D568029AC56127
:101BB00003624262002934D0132CDBBF43F68861F4
:101BC000C0F202011C3451F824408568816A641017
:101BD00003EB8413A3F58553102BB8BF102305EB3B
:101BE00085041B0405EBC4058B4202EBA512D4BF90
:101BF0000021012102243E2AC36280F83010446390
:101C000011DD4FF0607200234DF69C61C2F20001BD
:101C10000968A1FB024501FB0355230E43EA052396
:101C2000836330BC704702F003032241043308325F
:101C300003FA02F2D317E7E7436B0B70704700BF5C
:101C40000A680B69036102604B6843604B6943613A
:101C50008B6883608B698361CB68C360F0B5CB69A7
:101C6000C3610B6A4F6A8E6ACD6A91F830E04C6BA3
:101C70008A6B036291F8403047628662C56280F8E1
:101C800030E04463826380F84030F0BD70B54FF0BF
:101C90009D432DED048B08EE103A41F23063002194
:101CA00043F26804C3F680730020C4F2D01108EE3A
:101CB000903AC2F201040025B6EE009A0BE078EEED
:101CC000097A17EE900A0FF055FD41EC100B0CF05D
:101CD00067FB51EC100B6E0010F050F80136013527
:101CE000B5F5806F28EE288A44F82600E7D1002356
:101CF00040F2FF355A00D11C501C54F8211054F802
:101D000020000133091AAB4243F2680044F8221064
:101D1000C2F20100EED141F6FC73BDEC048BC35856
:101D200041F6F872C3F10043835070BD002207EE04
:101D3000902A4FF0974202EE102A4FF06C5204EEB8
:101D4000902A4FF06E5202EE902A4AF6AB22C3F66A
:101D50002A2241F2680303EE102AC2F20103002294
:101D6000F6EE003AB7EE006AB0EE004AF0EE465AE0
:101D7000E7EEE75A03EBC2010132B0EE677AA5EE57
:101D8000A47AB2F5806FB0EE465AA7EE475AF0EE4D
:101D9000636AE7EE826AB0EE677AA5EE247AFDEE1A
:101DA000E66AC1ED016AF0EE466AE7EE476AB0EE18
:101DB000677AA6EEA27A76EE856AB0EE465AA7EE6C
:101DC000475A35EE257AA6EE847AE7EE037ACDD12E
:101DD00030B4002240F2FF355100C81C4C1C53F8AF
:101DE000200053F824400132001BAA4241F268044B
:101DF00043F82100C2F20104EED14FF0974306EE02
:101E0000903AB6EE007AA7EEA67A41F6FC7341F658
:101E1000F872E358FDEEC77A17EE901ACB1AA3506A
:101E200030BC7047704700BF2DE9F04F43F6EC64BB
